:100000000C9491080C94C2080C94C2080C94C20879
:100010000C94C2080C94C2080C94C2080C94C20838
:100020000C94C2080C94C2080C94C2080C94C20828
:100030000C94C2080C94FB860C94C2080C94C20861
:100040000C94C2080C94C2080C94C2080C94C20808
:100050000C94C2080C94C2080C94C2080C94CA8D6B
:100060000C94C2080C9436510C940D510C94C20897
:100070000C94C2080C94C2080C94C2080C94C208D8
:100080000C94C2080C94C2080C94C2080C94C208C8
:100090000C94E3500C94BA500C94C2080C940E8843
:1000A0000C94C2080C94C2080C94C2080C94C208A8
:1000B0000C94C2080C94C2080C94C2080C94C20898
:1000C0000C94C2080C94C2080C94C2080C94905072
:1000D0000C9467500C94C2080C943D500C9414502E
:1000E0000C94C2088A35833565354F362136213662
:1000F00021362136213621362136213621364B2331
:10010000602668263728EE280A2ABE2BBA2C322D04
:10011000472D4B2D21368D2D992D062FC030DA30ED
:10012000FC315B3237334C3353333C342136213688
:100130002136213621362136213621362136213607
:100140007B342136213621362136213621364F3671
:100150006D89508AF08A0E8B238B388B4D8B6B8B7D
:10016000808B958BB38BC88BD78BEC8B568C598C33
:10017000488C4C8C528C908C5D8C618C678C6B8C19
:100180006F8C758C798C7D8C908C838C878C8B8C10
:10019000084AD73B3BCE016E84BCBFFDC12F3D6CEE
:1001A00074319ABD56833DDA3D00C77F11BED9E454
:1001B000BB4C3E916BAAAABE000000803F07634281
:1001C00036B79BD8A71A39685618AEBAAB558C1DEE
:1001D0003CB7CC5763BD6DEDFD753EF6177231BF70
:1001E000000000803F08000000BE922449123EAB90
:1001F000AAAA2ABECDCCCC4C3E00000080BEABAA41
:10020000AAAA3E00000000BF000000803F000000DE
:100210000000084178D3BB4387D1133D190E3CC37E
:10022000BD4282AD2B3E68EC8276BED98FE1A93EFD
:100230004C80EFFFBE01C4FF7F3F000000000000C4
:100240004E414E494E495459494E46CDCCCC3D0ABB
:10025000D7233C17B7D13877CC2B329595E6241F9E
:10026000B14F0A000020410000C84200401C462057
:10027000BCBE4CCA1B0E5AAEC59D7400407A10F32A
:100280005A00A0724E18090010A5D4E80000E876C4
:1002900048170000E40B54020000CA9A3B0000001B
:1002A000E1F505000080969800000040420F000034
:1002B00000A08601000000102700000000E80300F5
:1002C0000000006400000000000A000000000001BF
:1002D00000000000002C76D888DC674F0823DFC1BF
:1002E000DFAE59E1B1B796E5E3E453C63AE651997A
:1002F0007696E8E6C28426EB898C9B62ED407C6FA3
:10030000FCEFBC9C9F40F2BAA56FA5F490055A2A59
:10031000F75C936B6CF9676DC11BFCE0E40D47FE65
:10032000F520E6B500D0ED902E030094357705005A
:1003300080841E080000204E0A000000C80C3333E1
:1003400033330F986E12831141EF8D2114893BE6F0
:100350005516CFFEE6DB18D1844B381BF77C1D9079
:100360001DA4BBE424203284725E228100C9F124E2
:10037000ECA1E53D27696E707574204453546361A8
:100380006C6962726174653A0020766F6C746167A3
:10039000653D0023547572626964697479205570F3
:1003A000706572204C696D69743A200020766F6C1C
:1003B000746167653D00235475726269646974797C
:1003C000204C6F776572204C696D69743A20002368
:1003D000547572626964697479204C6F7765722014
:1003E0004C696D69742056696E663A200023434F4C
:1003F00032204D415820766F6C7420280023434FE3
:1004000032207A65726F20766F6C74202800234F3B
:10041000322063616C6962726174696F6E3A2000A8
:1004200023547572626964697479204C6F776572C0
:10043000204C696D69742056313A2000576946692D
:100440002049503A00234D5320456E61626C65642B
:1004500000234D532044697361626C6564004D6FE5
:1004600074696F6E004D6F74696F6E005556204948
:100470006E742E00555620496E74656E73697479DA
:10048000004F3220436F6E6300434F3220436F6E44
:10049000630053656E736F72206572726F72210014
:1004A000234E6F2073656E736F722100434F3220AD
:1004B000436F6E63004D6561737572696E670023EB
:1004C0004E6F2073656E736F7220666F7220504D91
:1004D00021004E6F2073656E736F722100206E676E
:1004E0002F4C00504D313A322E353A3130004D65A7
:1004F00061737572696E672E2E00234E6F20544211
:100500002073656E736F723F00234E6F2073656EAC
:10051000736F722100536F756E64204C6576656C45
:10052000004D6561737572696E672E2E00234E6FE4
:100530002073656E736F722100536F756E64204C6B
:100540006576656C00234E6F2073656E736F722045
:10055000666F722074656D7020262068756D696401
:1005600069747921004E6F2053656E736F7221009C
:1005700020666F722074656D7020262068756D6925
:100580006469747921002353656E736F722045721C
:10059000726F72200053656E736F72204572726FB6
:1005A0007221002357726F6E672073656E736F72CE
:1005B00020666F722074656D7020262068756D69E5
:1005C00064697479210057726F6E672053656E738A
:1005D0006F72210054656D702048756D696469748F
:1005E00079004C6967687420496E74656E7369742C
:1005F0007900466C616D6520495200234E6F207072
:10060000482073656E736F72210070482076616CAC
:10061000756500496E76616C6964206B65792100AF
:10062000204D756C746973656E736F7273004D75D0
:100630006C746973656E736F727300446973616281
:100640006C6500456E61626C6500237265706C6953
:1006500065733D002353657474696E6773206F661C
:1006600020616C6C2073656E736F72733A00436126
:100670006C6962726174696F6E2050726573737514
:1006800072653D00536561206C6576656C2050286D
:1006900063616C63293D00234572726F723A707218
:1006A00065737375726520424D503038352C206368
:1006B0006865636B20776972696E67210049522013
:1006C00054656D702073656E736F7220666F756E02
:1006D0006400504D322E352073656E736F72206C3E
:1006E000696B656C7920666F756E64005769466941
:1006F0002049503A00456455484B205345534C6FB0
:10070000676765720053656E736F7220736C6F74E8
:1007100020616E6420747970653A0057656C636F70
:100720006D6520746F20456455484B0067657453B0
:10073000656C665465737442697428293A200069AF
:1007400073496E74657272757074456E61626C6522
:10075000642831293A2000676574496E74657272A5
:100760007570744D617070696E672831293A200088
:10077000676574496E74657272757074536F7572C3
:1007800063652831293A2000676574496E74657283
:1007900072757074536F7572636528293A2000670B
:1007A00065745261746528293A20332E313431350D
:1007B000393F00616363656C2E69734C6F77506FCE
:1007C00077657228293A2000616363656C2E69732E
:1007D00041736C65657028293A2000616363656C1C
:1007E0002E6973546170536F757263654F6E5A282A
:1007F000293A2000616363656C2E697354617053FC
:100800006F757263654F6E5928293A2000616363E2
:10081000656C2E6973546170536F757263654F6EAA
:100820005828293A2000616363656C2E697341631F
:10083000746976697479536F757263654F6E5A285F
:10084000293A2000616363656C2E697341637469A2
:1008500076697479536F757263654F6E5928293ABA
:10086000200069734163746976697479536F757296
:1008700063654F6E5828293A2000697354617044AB
:100880006574656374696F6E4F6E5A28293B2066E4
:10089000616C73653F2000697354617044657465D1
:1008A0006374696F6E4F6E5A28293B2074727565A8
:1008B0003F20006973546170446574656374696FA7
:1008C0006E4F6E5928293B2066616C73653F20008E
:1008D0006973546170446574656374696F6E4F6EBB
:1008E0005928293B20747275653F20006973546153
:1008F00070446574656374696F6E4F6E5828293B48
:100900002066616C73653F200069735461704465B3
:1009100074656374696F6E4F6E5828293B2074723A
:1009200075653F20006765745375707072657373E9
:1009300042697428293B2066616C73653F2000671B
:100940006574537570707265737342697428293BBE
:1009500020747275653F200069734163746976691C
:100960007479416328293A20006973496E61637480
:1009700069766974795A456E61626C656428293AB2
:1009800020006973496E61637469766974795945A9
:100990006E61626C656428293A20006973496E6152
:1009A0006374697669747958456E61626C65642810
:1009B000293A2000697341637469766974795A45EC
:1009C0006E61626C656428293A2000697341637422
:1009D000697669747959456E61626C656428293A53
:1009E00020006973416374697669747958456E6152
:1009F000626C656428293A200067657446726565F3
:100A000046616C6C4475726174696F6E28293A2076
:100A1000006765744672656546616C6C5468726502
:100A200073686F6C6428293A200067657454696D97
:100A300065496E616374697669747928293A200082
:100A4000676574496E616374697669747954687214
:100A50006573686F6C64282920006765744163744E
:100A600069766974795468726573686F6C64282953
:100A70002000676574446F75626C655461705769D6
:100A80006E646F7728292000676574446F75626C07
:100A9000655461704C6174656E637928293A200051
:100AA0006765745461704475726174696F6E28294A
:100AB0003A2000676574417869734F6666736574A0
:100AC0002826782C2026792C20267A293A2000679F
:100AD00065745461705468726573686F6C6428291A
:100AE0003A200058595A2047733A200058595A2042
:100AF000434F554E54533A20007365742067616923
:100B00006E735B5D3A006761696E735F6F726967F0
:100B10005B5D3A00005EBCE2613FDD83C29C7E20EB
:100B2000A3FD1F41009D23BE46DB65F88C11AF324B
:100B3000CA57E9744F6666206169722D636F6E64EF
:100B400021004974277320746F6F20636F6F6C21CD
:100B50000054656D702069732066696E65210049D7
:100B600073206169722D636F6E64206F6E3F004960
:100B700074277320717569746520686F742100494A
:100B8000742773207665727920686F742120004F76
:100B90006666206169722D636F6E64210049742757
:100BA0007320746F6F20636F6F6C210054656D70DC
:100BB0002069732066696E6521004973206169723E
:100BC0002D636F6E64206F6E3F0049742773207130
:100BD0007569746520686F742100497427732076E5
:100BE00065727920686F74210054656D70204875B6
:100BF0006D696469747900482D6669656C64005399
:100C0000656172636820446972656374696F6E0020
:100C100020202020202020202020202020202020D4
:100C200000202020202020202020202020202020E4
:100C30002000697465726174696F6E3D0073656E42
:100C4000736F72233D0043757272656E7420737406
:100C5000617475733A206379636C653D006E6379E6
:100C6000636C653D006E73656E736F72733D006DEE
:100C700061786E73656E736F72733D00656E61624D
:100C80006C65643D00234D756C746973656E736F9C
:100C90007273206D6561737572656D656E74207316
:100CA000657474696E67733A007365703D006976A8
:100CB000616C3D006E697465723D00230023616EB6
:100CC0006F7468657220495220696E7075743D00BA
:100CD00023456E64206F66204D756C746973656E74
:100CE000736F72204379636C652300236B65793DD4
:100CF000004E6F2053656E736F7221004E6F20445B
:100D00005320546865726D6F6D657465722100447F
:100D10005320546865726D2E0046696E64696E6773
:100D2000205769466920495000416E676C65732FF2
:100D3000003E6128782C792C7A292F673A004E6F73
:100D40002073656E736F72210049522054656D7077
:100D500065726174757265004D6561737572696E57
:100D6000672E2E004E6F2073656E736F723F0049C1
:100D7000522054656D7065726174757265004D65C1
:100D800061737572696E672E2E00232D2D2D2D2D0A
:100D90002D2D2D2D2D2D2D2D2D2D2D2D2D2D2D2D83
:100DA0002D2D2D2D2D2D2D2D2D2D2D2D2D2D2D00A0
:100DB000235265736F6C7574696F6E3A2020200042
:100DC000234D696E2056616C75653A202020200005
:100DD000234D61782056616C75653A2020202000F3
:100DE00023556E697175652049443A202020200002
:100DF00023447269766572205665723A202020007D
:100E00002353656E736F723A20202020202020002B
:100E1000232D2D2D2D204D61676E65746963205340
:100E2000656E736F72202D2D2D2D2D2D2D2D2D2DB9
:100E30002D2D2D2D2D2D2D2D2D2D00482D66696547
:100E40006C643A2028002020202020202020202010
:100E500020202020202000202020202020202020B2
:100E600020202020202020002020202020202020A2
:100E70002020202020202000202020202020202092
:100E80002020202020202000233A53686F772F480D
:100E9000696465204C4344002A3A546869732048C9
:100EA000656C700044433A436C656172204C434466
:100EB0000044423A5265736574204C6F67676572EF
:100EC0000044363A44532054656D700044353A5519
:100ED0005620496E74656E736974790044343A4FD4
:100EE0003220636F6E632E0044333A434F322063E7
:100EF0006F6E632E0044323A504D28313A322E350F
:100F00003A3130290044323A504D28313A322E35A8
:100F10003A3130292A0044313A5475726269646961
:100F200074790044303A566F6C7461676500393AE1
:100F30006F7220334420616363656C2E00393A4937
:100F40006E636C2E20616E672E00383A70482076F2
:100F5000616C756500373A49522054656D700037F1
:100F60003A49522054656D702A00363A4D61676ED9
:100F700065746963206669656C6400353A4761731E
:100F8000204C6576656C00343A495220466C616DA0
:100F90006500333A4C6967687420496E742E0032DC
:100FA0003A616E642048656967687400323A546536
:100FB0006D7020507265737375726500313A5465B7
:100FC0006D702048756D696469747900303A536FAB
:100FD000756E64204C6576656C00303A536F756EA3
:100FE00064204C6576656C2A0054696D65206C61DF
:100FF0007073653A00576946692049503A0000000D
:101000002100240027002A002D00300033000101B8
:101010000000040107010A01000022002500280049
:101020002B002E00310034000201000005010801F0
:101030000B01000020002300260029002C002F00B7
:101040003200000100000301060109010505050544
:10105000070508080808020202020A0A0808040430
:10106000040401010101010101010303030303035E
:101070000303040707070C0C0C0C0C0C0C0C0202ED
:10108000020206060606060606060B0B0B0B0B0BEA
:101090000B0B010210202008081020401020408077
:1010A000020102010804020101020408102040802C
:1010B00080402010080402018004020180402010BA
:1010C0000804020108040201010204081020408003
:1010D000010204081020408000000A0B02090C0DD8
:1010E0000E080703040100000000000000000000DB
:1010F00000000000000000000000000000000000F0
:1011000000000000121110000000000000000000AC
:101110000000000000000000000000000000969B9E
:10112000DF9D11241FBECFEFD1E2DEBFCDBF00E0B7
:101130000CBF1CE0A0E0B2E0EAE7F4E501E00BBF81
:1011400002C007900D92A238B107D9F724E1A2E8B6
:10115000BCE001C01D92A733B207E1F718E0C0E977
:10116000D8E000E006C021970109802FFE010E940F
:101170007FA7CF38D10780E00807A9F70E947E91AA
:101180000C942CAA0C9400002F923F924F925F92E5
:101190006F927F928F929F92AF92BF92CF92DF9287
:1011A000EF92FF920F931F93CF93DF93CDB7DEB7EC
:1011B000C654D1090FB6F894DEBF0FBECDBF109153
:1011C0002714112321F0109227140C949822809157
:1011D000E6129091E712019709F050C060E070E0CC
:1011E00082EE92E10E94654D082E000C990B0E9440
:1011F000C3A9892B09F442C06BE675E0CE01839642
:101200000E94DC4EBE016D5D7F4F82EE92E10E9436
:10121000F849811127C06EEB79E0CE0145960E9416
:10122000DC4EBE016B5E7F4F82EE92E10E94F84978
:10123000811114C064E47BE0CE0101960E94DC4E73
:10124000BE016F5F7F4F82EE92E10E94F84911E08C
:10125000811110E0CE0101960E94984ECE01459674
:101260000E94984ECE0183960E94984E112331F031
:1012700062EE72E186ED92E10E94494E8091E612A3
:101280009091E712049708F041C060E078E0CE0149
:1012900001960E94DC4EBE016F5F7F4F82EE92E1AD
:1012A0000E94F849182FCE0101960E94984E1123F2
:1012B00069F161E070E082EE92E10E94654D803359
:1012C0000CF484516AE270E0681B710987FD739524
:1012D000CE0101960E946F5EBE016F5F7F4F82EE6E
:1012E00092E10E945E4ECE0101960E94984E62EEFF
:1012F00072E186ED92E10E94494E82EE92E10E94F7
:10130000FA4CCB010E94B2220C9498226DE675E053
:10131000CE0145960E94DC4EBE016B5E7F4F82EE91
:1013200092E10E94F849811116C061E775E0CE0193
:1013300001960E94DC4EBE016F5F7F4F82EE92E10C
:101340000E94F84911E0811101C010E0CE01019620
:101350000E94984E01C011E0CE0145960E94984E21
:10136000112309F453C365E775E0CE0101960E948D
:10137000DC4ECE0101960E948754CE0101960E9458
:10138000984E61E875E0CE0101960E94DC4E6FEB4D
:1013900073E1CE0101960E94E94DBC01CE01459654
:1013A0000E94D44ECE0145960E948754CE014596A8
:1013B0000E94984ECE0101960E94984E60916B0457
:1013C00070916C0480916D0490916E040E94A1A2B2
:1013D00020E030E048EC52E40E94F1A4AB01BC01F3
:1013E00022E0CE0145960E949D4E67E975E0CE0150
:1013F00001960E94DC4EBE016B5E7F4FCE010196CE
:101400000E94E94D68EF76E00E94D24DBC01CE010A
:1014100083960E94D44ECE0183960E948754CE01BB
:1014200083960E94984ECE0101960E94984ECE015E
:1014300045960E94984E40916704509168046091CF
:10144000690470916A0424E0CE0145960E949D4E85
:101450006CEA75E0CE0101960E94DC4EBE016B5E27
:101460007F4FCE0101960E94E94DBC01CE018396CB
:101470000E94D44ECE0183960E948754CE0183965B
:101480000E94984ECE0101960E94984ECE0145963C
:101490000E94984E40915B0450915C0460915D0401
:1014A00070915E0422E0CE018F960E949D4E409185
:1014B000530450915404609155047091560423E0F4
:1014C000CE0189960E949D4E40915F045091600428
:1014D000609161047091620422E0CE0183960E94C3
:1014E0009D4E409157045091580460915904709159
:1014F0005A0423E0CE0145960E949D4E69EC75E0AA
:10150000CE0101960E94DC4EBE016B5E7F4FCE0184
:1015100001960E94E94D6EED75E00E94D24DBE012C
:101520006D5D7F4F0E94E94D61EE75E00E94D24DE6
:10153000BE01675D7F4F0E94E94D6EED75E00E9430
:10154000D24DBE01615D7F4F0E94E94D67EE75E0AF
:101550000E94D24DBC01CE01C5960E94D44ECE0150
:10156000C5960E948754CE01C5960E94984ECE0122
:1015700001960E94984ECE0145960E94984ECE014B
:1015800083960E94984ECE0189960E94984ECE0175
:101590008F960E94984E4091C2045091C30460916E
:1015A000C4047091C50423E0CE0183960E949D4E31
:1015B00020914F04309150044091510450915204B5
:1015C00060E070E080E291E40E949FA6AB01BC0164
:1015D00021E0CE0145960E949D4E6CEE75E0CE0155
:1015E00001960E94DC4EBE016B5E7F4FCE010196DC
:1015F0000E94E94D6FEF75E00E94D24DBE016D5D16
:101600007F4F0E94E94D65E076E00E94D24DBC011B
:10161000CE0189960E94D44ECE0189960E948754AD
:10162000CE0189960E94984ECE0101960E94984E56
:10163000CE0145960E94984ECE0183960E94984E08
:101640004091BE045091BF046091C0047091C104E8
:1016500023E0CE0183960E949D4E20914B04309151
:101660004C0440914D0450914E0460E070E080E2E3
:1016700091E40E949FA6AB01BC0121E0CE014596FA
:101680000E949D4E68E076E0CE0101960E94DC4EFD
:10169000BE016B5E7F4FCE0101960E94E94D6FEF58
:1016A00075E00E94D24DBE016D5D7F4F0E94E94DF5
:1016B00065E076E00E94D24DBC01CE0189960E9481
:1016C000D44ECE0189960E948754CE0189960E94FD
:1016D000984ECE0101960E94984ECE0145960E94EA
:1016E000984ECE0183960E94984E409147045091A7
:1016F00048046091490470914A0422E0CE01459665
:101700000E949D4E6BE176E0CE0101960E94DC4E78
:10171000BE016B5E7F4FCE0101960E94E94D61E3F1
:1017200076E00E94D24DBC01CE0183960E94D44E39
:10173000CE0183960E948754CE0183960E94984ED4
:10174000CE0101960E94984ECE0145960E94984E79
:1017500040914304509144046091450470914604C3
:1017600022E0CE0145960E949D4E68E376E0CE01D0
:1017700001960E94DC4EBE016B5E7F4FCE0101964A
:101780000E94E94D65E076E00E94D24DBC01CE0199
:1017900083960E94D44ECE0183960E948754CE0138
:1017A00083960E94984ECE0101960E94984ECE01DB
:1017B00045960E94984E51E3C52E54E0D52E01E087
:1017C00010E067E1E62E80912F049091300480179D
:1017D00091070CF44DC0D601AD90BD906D01B501DF
:1017E000CE0183960E946F5EB801CE0145960E949D
:1017F0006F5E6BE476E0CE0101960E94DC4EBE0186
:101800006B5E7F4FCE0101960E94E94D68E176E064
:101810000E94D24DBE016D5D7F4F0E94E94D63E590
:1018200076E00E94D24DEA9CB001EB9C700D112431
:10183000695E7D4F0E94D24DBC01CE0189960E9407
:10184000D44ECE0189960E948754CE0189960E947B
:10185000984ECE0101960E94984ECE0145960E9468
:10186000984ECE0183960E94984E0F5F1F4FABCFCC
:101870008091BF0D9091C00D892B71F469E576E0E0
:10188000CE0101960E94DC4ECE0101960E94875443
:10189000CE0101960E94984E8091BF0D9091C00D8F
:1018A000019771F468E676E0CE0101960E94DC4E65
:1018B000CE0101960E948754CE0101960E94984E57
:1018C0008091BF0D9091C00D029771F462E776E0B0
:1018D000CE0101960E94DC4ECE0101960E948754F3
:1018E000CE0101960E94984E60914104709142048D
:1018F000CE0145960E946F5E64E876E0CE010196C7
:101900000E94DC4EBE016B5E7F4FCE0101960E94AD
:10191000E94DBC01CE0183960E94D44ECE01839640
:101920000E948754CE0183960E94984ECE01019664
:101930000E94984ECE0145960E94984E4091130207
:1019400050911402609115027091160222E0CE01AE
:1019500045960E949D4E61EA76E0CE0101960E9476
:10196000DC4EBE016B5E7F4FCE0101960E94E94DB9
:1019700064E379E00E94D24DBC01CE0183960E94BF
:10198000D44ECE0183960E948754CE0183960E9446
:10199000984ECE0101960E94984ECE0145960E9427
:1019A000984E40918004509181046091820470911E
:1019B000830422E0CE0145960E949D4E61EB76E0C5
:1019C000CE0101960E94DC4EBE016B5E7F4FCE01C0
:1019D00001960E94E94D64E379E00E94D24DBC017A
:1019E000CE0183960E94D44ECE0183960E948754E6
:1019F000CE0183960E94984ECE0101960E94984E89
:101A0000CE0145960E94984E109212028091E612E5
:101A10009091E7128330910508F092C081309105D2
:101A200041F460E070E082EE92E10E94654DF82E94
:101A300062C0029709F05FC060E078E0CE010196D5
:101A40000E94DC4EBE016F5F7F4F82EE92E10E94EA
:101A5000F849182FCE0101960E94984E112309F4DF
:101A60004AC061E070E082EE92E10E94654D1A8208
:101A700019821C821B821E821D828D8B1E8ABE01D2
:101A80006B5E7F4FCE0101960E94344EBE016F5FA8
:101A90007F4F86ED92E10E945E4ECE0101960E943C
:101AA000984E60E070E082EE92E10E94654DF82E63
:101AB00080911F0D8823F9F061EC76E0CE0101964C
:101AC0000E94DC4E62EE72E1CE0101960E94E94D69
:101AD00066EE7BE00E94D24DBC0180E490E10E9462
:101AE0003A4FCE0101960E94984E66ED72E180E475
:101AF00090E10E94857A8F2D0F2C000C990B0E948B
:101B0000C3A9892BB1F00E94976B0E94927F66EE69
:101B10007BE0CE0101960E94DC4E4AE050E060E09E
:101B200070E0CE0101960E94FA60CE0101960E94FB
:101B3000984E8F2D0E949E540E94BE8D0C94882238
:101B400021E030E040E050E062EE72E1CE0101962B
:101B50000E94F04EBE016F5F7F4F84EC92E10E94C5
:101B60005E4ECE0101960E94984E64EF76E0CE0163
:101B700045960E94DC4EBE016B5E7F4F82EE92E185
:101B80000E94F849811116C06EEE7BE0CE010196ED
:101B90000E94DC4EBE016F5F7F4F82EE92E10E9499
:101BA000F84911E0811101C010E0CE0101960E94B8
:101BB000984E01C011E0CE0145960E94984E112327
:101BC00009F4BCC08091E6129091E712409710F0A2
:101BD0000C94982242E050E062EE72E1CE01019650
:101BE0000E945480BE016F5F7F4F84EC92E10E949F
:101BF0005E4ECE0101960E94984E64EC72E1CE01D9
:101C000001960E94D44ECE0101960E942960CE0119
:101C100001960E94984E0E943A8F20E030E048ECF6
:101C200052E40E9400A30E948AA5AB01BC0140932C
:101C30006B0450936C0460936D0470936E04CE013A
:101C400001960E943F7BCE0101960E942960CE0141
:101C500001960E94984E60916B0470916C04809183
:101C60006D0490916E048B019C0100591F45214029
:101C7000310901341C492105310588F067EC76E013
:101C8000CE0101960E94DC4E64EC72E1CE01019619
:101C90000E94E94D6AED76E00E94D24DBBC11A82E6
:101CA0001982FE01339626E0DF011D922A95E9F79D
:101CB0000E94A1A220E030E048EC52E40E94F1A48E
:101CC0008E010F5F1F4F22E047E00E940B9EBC0178
:101CD0008AEC92E10E94344E6AEE76E0CE0145969F
:101CE0000E94DC4E6AEC72E1CE0145960E94E94DFD
:101CF00067EF76E00E94D24DBC018AEC92E10E942F
:101D0000494ECE0145960E94984E1092DA0C1092E0
:101D1000D90C80916B0490916C04A0916D04B091EA
:101D20006E048093490D90934A0DA0934B0DB09390
:101D30004C0D80E090E00E94F27E75C16CEF76E081
:101D4000CE0145960E94DC4EBE016B5E7F4F82EE57
:101D500092E10E94F849811116C062E077E0CE015D
:101D600001960E94DC4EBE016F5F7F4F82EE92E1D2
:101D70000E94F84911E0811101C010E0CE010196E6
:101D80000E94984E01C011E0CE0145960E94984EE7
:101D9000112309F469C026E030E045E050E062EE2E
:101DA00072E1CE0101960E94F04EBE016F5F7F4F3F
:101DB00084EC92E10E945E4ECE0101960E94984E04
:101DC00084EC92E10E94FA4C6B017C016FE276E0B8
:101DD000CE0101960E94DC4EBE016F5F7F4F82EE06
:101DE00092E10E949549AC014F5F5F4F62EE72E154
:101DF000CE0145960E945480BE016B5E7F4F84ECFD
:101E000092E10E945E4ECE0145960E94984ECE0110
:101E100001960E94984E84EC92E10E94FA4C9B013C
:101E2000EFE2F4E041E050E0A0912F04B0913004E3
:101E3000A417B5075CF0A281B3812A173B0711F400
:101E4000138212824F5F5F4F3296EECF9601220FC0
:101E5000331FF901E15DFB4F7183608382E090E005
:101E60000E94F16C0C94E91868E077E0CE01459689
:101E70000E94DC4EBE016B5E7F4F82EE92E10E94BB
:101E8000F849811116C06EE077E0CE0101960E94FC
:101E9000DC4EBE016F5F7F4F82EE92E10E94F849F7
:101EA00011E0811101C010E0CE0101960E94984E10
:101EB00001C011E0CE0145960E94984E112339F1E0
:101EC000EFE2F4E081E090E020912F0430913004C3
:101ED0002817390774F0863091051CF493838283A8
:101EE00005C09C012E5F3F4F3383228301963296BB
:101EF000EBCF82E090E00E94F16C1092DA0C10922D
:101F0000D90C80E090E00E94F27E0C94742264E18F
:101F100077E0CE0145960E94DC4EBE016B5E7F4F9E
:101F200082EE92E10E94F849811116C06BE177E0E0
:101F3000CE0101960E94DC4EBE016F5F7F4F82EEA4
:101F400092E10E94F84911E0811101C010E0CE0138
:101F500001960E94984E01C011E0CE0145960E9464
:101F6000984E1123F9F08091470D9091480D892BDF
:101F7000A1F481E090E09093480D8093470D8EEDA1
:101F800093E09093DA0C8093D90C0E941B7F68EC4D
:101F900070E080E090E00E94868DE0E0F0E019952E
:101FA0000C94762262E277E0CE0145960E94DC4EE8
:101FB000BE016B5E7F4F82EE92E10E94F849811173
:101FC00016C06AE277E0CE0101960E94DC4EBE01A7
:101FD0006F5F7F4F82EE92E10E94F84911E081111C
:101FE00001C010E0CE0101960E94984E01C011E0A0
:101FF000CE0145960E94984E1123A1F162E377E04D
:10200000CE0101960E94DC4E69EB73E1CE01019690
:102010000E94E94DBC018AEC92E10E94494ECE013A
:1020200001960E94984E64E87BE0CE0101960E94E2
:10203000DC4E6AEC72E1CE0101960E94E94DBC01D2
:10204000CE0145960E94D44ECE0145960E948754FB
:10205000CE0145960E94984ECE0101960E94984E60
:102060000C9474226CE377E0CE0145960E94DC4E1E
:10207000BE016B5E7F4F82EE92E10E94F8498111B2
:1020800016C063E477E0CE0101960E94DC4EBE01EB
:102090006F5F7F4F82EE92E10E94F84911E081115B
:1020A00001C010E0CE0101960E94984E01C011E0DF
:1020B000CE0145960E94984E112349F069E875E0DB
:1020C000CE0101960E94DC4E6FEB73E19FCF6AE474
:1020D00077E0CE0145960E94DC4EBE016B5E7F4FDD
:1020E00082EE92E10E94F849811116C061E577E025
:1020F000CE0101960E94DC4EBE016F5F7F4F82EEE3
:1021000092E10E94F84911E0811101C010E0CE0176
:1021100001960E94984E01C011E0CE0145960E94A2
:10212000984E112309F48FC06FE276E0CE0101963C
:102130000E94DC4EBE016F5F7F4F82EE92E10E94F3
:102140009549AC014F5F5F4F62EE72E1CE0145965B
:102150000E945480BE016B5E7F4F84EC92E10E942E
:102160005E4ECE0145960E94984ECE0101960E9489
:10217000984E84EC92E10E94FA4C8B0161E574E088
:102180008AEC92E10E940E4E8091C411882331F0B6
:1021900065E474E08AEC92E10E940E4E011511058F
:1021A00011F40C946622CE0101960E948E69CE0134
:1021B00001960E948754CE0101960E94984E0230EB
:1021C000110514F40C94742264E576E0CE01459672
:1021D0000E94CC4EBE016B5E7F4FCE0101960E94E5
:1021E000D44ECE0101960E948754CE0101960E94E2
:1021F000984EE12CF12C8091C611082E000C990B01
:10220000E816F9068CF4B701CE0101960E947368B6
:10221000CE0101960E948754CE0101960E94984EED
:10222000FFEFEF1AFF0AE7CFCE0145960E94984EC6
:102230000230110511F40C9474228CE291E00E949A
:10224000687F0C94742268E577E0CE0145960E9481
:10225000DC4EBE016B5E7F4F82EE92E10E94F84938
:10226000811116C06FE577E0CE0101960E94DC4E29
:10227000BE016F5F7F4F82EE92E10E94F84911E04C
:10228000811101C010E0CE0101960E94984E01C05C
:1022900011E0CE0145960E94984E112309F48EC399
:1022A00062EE72E1CE018F5B9F4F0E94D44E6FE2CF
:1022B00076E0CE0101960E94DC4EBE016F5F7F4F3B
:1022C000CE018F5B9F4F0E949549AC014F5F5F4FDE
:1022D000BE016F5B7F4FCE01CB960E945480CE0132
:1022E00001960E94984EBE016F5B7F4FCE01019612
:1022F0000E94D44ECE0101960E942960CE01019623
:102300000E94984E6CE577E0CE0101960E94DC4E6B
:10231000BE016F5F7F4FCE01CB960E9459498C0161
:10232000CE0101960E94984E6AE37CE0CE01C596EC
:102330000E94DC4E6AE37CE0CE018F960E94DC4E68
:102340001016110694F5A8014F5F5F4F21968EADD0
:102350009FAD21974817590790F4BE01655C7F4FE8
:10236000CE0101960E945480BE016F5F7F4FCE0167
:10237000C5960E945E4ECE0101960E94984E98012D
:1023800040E050E0BE01655C7F4FCE0101960E94A7
:10239000F04EBE016F5F7F4FCE018F960E945E4E62
:1023A000CE0101960E94984E0DC06AE37CE0CE01FA
:1023B000C5960E94344EBE01655C7F4FCE018F965C
:1023C0000E94494E8BA99CA9892B09F4E7C2CE0132
:1023D0008F960E94FA4C8B010150110908311105AA
:1023E00014F007E110E017FF02C00FEF1FEFB80174
:1023F000CE0145960E946F5E6EE577E0CE010196B4
:102400000E94DC4EBE016B5E7F4FCE0101960E94A2
:10241000E94DBC01CE0183960E94D44ECE01839635
:102420000E942960CE0183960E94984ECE010196AB
:102430000E94984ECE0145960E94984EBE016B5C5C
:102440007F4FCE01CB960E94494E6CE577E0CE01DE
:1024500001960E94DC4EBE016F5F7F4FCE01CB968E
:102460000E9459497C01CE0101960E94984E6AE370
:102470007CE0CE01C5960E94344E6AE37CE0CE013A
:102480008F960E94344E1E141F040CF050C0A701FA
:102490004F5F5F4F21968EAD9FAD2197481759072B
:1024A00090F4BE01655C7F4FCE0101960E9454807E
:1024B000BE016F5F7F4FCE01C5960E945E4ECE017A
:1024C00001960E94984E970140E050E0BE01655C85
:1024D0007F4FCE0101960E94F04EBE016F5F7F4F8D
:1024E000CE018F960E945E4ECE0101960E94984EBC
:1024F000AE014F5F5F4F5A01E12CF12CA8014F5FF5
:102500005F4F8AE0849F9001859F300D1124B901AF
:102510006C537E4E6B01809F9001819F300D112482
:10252000C9018E529E4E3C019AE2592EC2C06AE306
:102530007CE0CE01C5960E94344EBE01655C7F4FA3
:10254000CE018F960E94494ED3CFCE018F96E114D3
:10255000F10409F0BBC00F3FAFEF1A0709F4B6C092
:102560000E94054DC114D10439F044E050E0B60199
:10257000CE018F960E947349B601CE0183960E94C8
:10258000DC4E63E677E0CE0145960E94DC4EBE014C
:102590006D5D7F4FCE0145960E94E94DBC01CE0195
:1025A00089960E94D44ECE0189960E942960CE0160
:1025B00089960E94984ECE0145960E94984ECE0173
:1025C00083960E94984E8BA99CA9029708F477C025
:1025D00061E070E0CE018F960E94654D082E000CE0
:1025E000990B803391050CF44497B52DB81BF3017A
:1025F000B083FFEFEF1AFF0ABE016B5C7F4FCE0185
:10260000CB960E94494E6CE577E0CE0145960E943C
:10261000DC4EBE016B5E7F4FCE01CB960E945949C6
:102620004C01CE0145960E94984E6AE37CE0CE01B3
:10263000C5960E94344E6AE37CE0CE018F960E94DC
:10264000344E181419040CF047C0A4014F5F5F4FBB
:1026500021968EAD9FAD21974817590790F4BE0182
:10266000655C7F4FCE0145960E945480BE016B5E33
:102670007F4FCE01C5960E945E4ECE0145960E94C8
:10268000984E940140E050E0BE01655C7F4FCE0162
:1026900045960E94F04EBE016B5E7F4FCE018F9635
:1026A0000E945E4ECE0145960E94984E92E0A90E81
:1026B000B11C8BA99CA9892B09F047CF1BC0CE0167
:1026C0008F960E94FA4CD3016C9393CF0E94FA4CE0
:1026D000F501718360838DCF6AE37CE0CE01C596FE
:1026E0000E94344EBE01655C7F4FCE018F960E94E2
:1026F000494EDCCF0F3F2FEF120709F07DC06CE58C
:1027000077E0CE0145960E94DC4EBE016B5E7F4FA6
:10271000CE01C5960E9459498C01CE0145960E9472
:10272000984E17FF3BC109811A811016110634F427
:10273000093111052CF008E110E002C001E010E0C1
:102740000093C611B801CE0183960E946F5E61E7C7
:1027500077E0CE0145960E94DC4EBE016D5D7F4F55
:10276000CE0145960E94E94DBC01CE0189960E949A
:10277000D44ECE0189960E942960CE0189960E948E
:10278000984ECE0145960E94984ECE0183960E94A7
:10279000984EE114F10459F18B819C8197FF02C09E
:1027A00080E090E09093C8118093C71141E0E41657
:1027B000F104E9F08D819E81181619062CF480171A
:1027C000910724F48C0102C001E010E00150009355
:1027D000CB1152E0E516F10451F08F81988518165F
:1027E000190614F081E090E081508093CC118CE2C6
:1027F00091E00E943F7FD2C08091C511082E000C4D
:10280000990B081719070CF083C0B701CE01839606
:102810000E946F5E6BE777E0CE0145960E94DC4E2A
:10282000BE016D5D7F4FCE0145960E94E94DBC0112
:10283000CE0189960E94D44ECE0189960E942960CD
:10284000CE0189960E94984ECE0145960E94984EE0
:10285000CE0183960E94984E8AE0809FF001819F6E
:10286000F00D1124EC53FE4E81E0878783E090E069
:10287000918B808B938B828BE114F10409F48EC0D1
:102880008B819C818038910514F08FE790E080382F
:102890006FEF960714F480E89FEF878771E0E716E3
:1028A000F10409F47BC08AE0809FF001819FF00D64
:1028B0001124EC53FE4E8D819E8197FF02C080E073
:1028C00090E0918B808B82E0E816F10409F466C0F9
:1028D0008AE0809FF001819FF00D1124EC53FE4EA1
:1028E0008F81988597FF02C080E090E0938B828B68
:1028F0008091C611082E000C990B081719071CF0BF
:102900000F5F0093C6118CE291E00E94687F46C081
:10291000BE016B5C7F4FCE0189960E94D44E6091C0
:10292000C511062E000C770BCE0183960E946F5EB8
:1029300063E877E0CE0145960E94DC4EBE01675DFC
:102940007F4FCE0145960E94E94D64E977E00E94F1
:10295000D24DBE016D5D7F4F0E94E94DBC01CE019D
:1029600089960E94494ECE0145960E94984ECE010E
:1029700083960E94984EBE01675D7F4FCE014596BB
:102980000E94D44ECE0145960E948754CE014596B2
:102990000E94984ECE0189960E94984ECE018F9645
:1029A0000E94984ECE01C5960E94984ECE01CB96BD
:1029B0000E94984ECE018F5B9F4F4EC268E977E030
:1029C000CE0145960E94DC4EBE016B5E7F4F82EECB
:1029D00092E10E94F849811116C06DE977E0CE01BD
:1029E00001960E94DC4EBE016F5F7F4F82EE92E146
:1029F0000E94F84911E0811101C010E0CE0101965A
:102A00000E94984E01C011E0CE0145960E94984E5A
:102A10001123D9F16FE276E0CE0101960E94DC4EDF
:102A2000BE016F5F7F4F82EE92E10E949549AC013B
:102A30004F5F5F4F62EE72E1CE0145960E94548077
:102A4000BE016B5E7F4F84EC92E10E945E4ECE0130
:102A500045960E94984ECE0101960E94984E84ECB5
:102A600092E10E94FA4C6115710521F481E0809396
:102A7000850407C06130710511F00C947422109226
:102A800085040E94A76B0C94742262EA77E0CE0161
:102A900045960E94DC4EBE016B5E7F4F82EE92E156
:102AA0000E94F849811116C066EA77E0CE010196CE
:102AB0000E94DC4EBE016F5F7F4F82EE92E10E946A
:102AC000F84911E0811101C010E0CE0101960E9489
:102AD000984E01C011E0CE0145960E94984E1123F8
:102AE00009F424C143E050E062EE72E1CE010196A8
:102AF0000E945480BE016F5F7F4F84EC92E10E9480
:102B00005E4ECE0101960E94984E64EC72E1CE01B9
:102B100001960E94D44ECE0101960E942960CE01FA
:102B200001960E94984E1092DA0C1092D90C64EC27
:102B300072E185EC93E10E94494E64EC72E18FEB07
:102B400093E10E94494E85E69DE0009739F048E008
:102B500050E0BC0185EC93E10E94734983EC9DE059
:102B6000009739F04CE050E0BC018FEB93E10E94FC
:102B700073498091D90C9091DA0C0E94F27E6AEA36
:102B800077E0CE0101960E94DC4E6FEB73E1CE013F
:102B900001960E94E94DBC01CE0183960E94D44E5D
:102BA000CE0101960E94984E8091BF0D9091C00D6C
:102BB000892B39F4BE016D5D7F4F89E69EE00E944E
:102BC0003A4F8091BF0D9091C00D029709F09BC0C4
:102BD0006FEB73E1CE0189960E94D44E62EB77E0F1
:102BE000CE0101960E94DC4ECE0101960E94129BFE
:102BF000CE0101960E94984E64EF71E080E090E073
:102C00000E94868D65EB77E0CE0101960E94DC4E36
:102C1000CE0101960E94129BCE0101960E94984E11
:102C200064EF71E080E090E00E94868D6EEB77E0CB
:102C3000CE0101960E94DC4ECE0101960E94129BAD
:102C4000CE0101960E94984E64EF71E080E090E022
:102C50000E94868D67EC77E0CE0101960E94DC4EE3
:102C6000CE0101960E94129BCE0101960E94984EC1
:102C700064EF71E080E090E00E94868D65ED77E082
:102C8000CE0101960E94DC4ECE0101960E94129B5D
:102C9000CE0101960E94984E64EF71E080E090E0D2
:102CA0000E94868D6AEA77E0CE0101960E94DC4E92
:102CB000BE01675D7F4FCE0101960E94E94DBC01C8
:102CC000CE0145960E94D44ECE0101960E94984EA8
:102CD000CE0145960E94054DBE016B5E7F4FCE0131
:102CE00001960E94D44ECE0101960E94129BCE0105
:102CF00001960E94984ECE0145960E94984ECE01B4
:102D000089960E94984E65E67DE0CE0101960E946C
:102D1000DC4ECE0101960E942960CE0101960E94F0
:102D2000984E10921202CE01839696C063EE77E021
:102D3000CE0145960E94DC4EBE016B5E7F4F82EE57
:102D400092E10E94F849811116C068EE77E0CE0149
:102D500001960E94DC4EBE016F5F7F4F82EE92E1D2
:102D60000E94F84911E0811101C010E0CE010196E6
:102D70000E94984E01C011E0CE0145960E94984EE7
:102D8000112309F46DC044E050E062EE72E1CE011F
:102D900001960E945480BE016F5F7F4F84EC92E1E8
:102DA0000E945E4ECE0101960E94984E6DEE77E035
:102DB000CE0145960E94DC4E64EC72E1CE01459650
:102DC0000E94E94DBC01CE0101960E94D44ECE0175
:102DD00045960E94984E8091BF0D9091C00D892B11
:102DE00039F4BE016F5F7F4F89E69EE00E943A4F43
:102DF00068EB7BE080E090E00E94868D8091BF0DC3
:102E00009091C00D029779F4BE016F5F7F4FCE01A4
:102E100045960E94D44ECE0145960E94129BCE014B
:102E200045960E94984E68EB7BE080E090E00E941F
:102E3000868DBE016F5F7F4FCE0145960E94D44EB6
:102E4000CE0145960E942960CE0145960E94984E7B
:102E500010921202CE0101960E94984E0C94762296
:102E600064EF77E0CE0145960E94DC4EBE016B5EBA
:102E70007F4F82EE92E10E94F849811116C068EFFF
:102E800077E0CE0101960E94DC4EBE016F5F7F4F5E
:102E900082EE92E10E94F84911E0811101C010E038
:102EA000CE0101960E94984E01C011E0CE014596D8
:102EB0000E94984E112309F463C062EE72E184EC23
:102EC00092E10E94494E81E08093120262EE72E12B
:102ED000CE0101960E94D44ECE0101960E94296037
:102EE000CE0101960E94984E8091BF0D9091C00D29
:102EF000029709F164EC72E189E69EE00E943A4F84
:102F000068EB7BE080E090E00E94868DCE01019628
:102F10000E94D159BE016F5F7F4F82EE92E10E9405
:102F20005E4ECE0101960E94984E60ED77E080E003
:102F300090E00E94868D8091BF0D9091C00D029708
:102F400071F464EC72E1CE0101960E94D44ECE0180
:102F500001960E94129BCE0101960E94984E80918C
:102F6000E6129091E712892B11F40C94742264E814
:102F70007BE0CE0101960E94DC4E62EE72E15BC8FE
:102F80006CEF77E0CE0145960E94DC4EBE016B5E91
:102F90007F4F82EE92E10E94F849811116C062E0F3
:102FA00078E0CE0101960E94DC4EBE016F5F7F4F3C
:102FB00082EE92E10E94F84911E0811101C010E017
:102FC000CE0101960E94984E01C011E0CE014596B7
:102FD0000E94984E112309F461C08091BF0D909119
:102FE000C00D019711F00C947422CE0101960E943D
:102FF000ED6E8D819E81009711F40C947022E98111
:10300000FA812081222311F40C947022079710F486
:103010000C9470226CE374E0CE0145960E94CC4E75
:1030200048EC50E06FEF7FEFCE0145960E94FA60CA
:10303000CE0145960E94984EBE016F5F7F4FCE0134
:1030400045960E94D44E40ED57E06FEF7FEFCE01E2
:1030500045960E94C07FCE0145960E94984E68E03A
:1030600078E0CE0145960E94DC4E62EE72E1CE0120
:1030700045960E94E94DBC01CE0183960E94D44E34
:10308000CE0183960E948754CE0183960E94984E6B
:10309000CE0145960E94984E0C94702266E178E02D
:1030A000CE0145960E94DC4EBE016B5E7F4F82EEE4
:1030B00092E10E94F849811116C06BE178E0CE01DF
:1030C00001960E94DC4EBE016F5F7F4F82EE92E15F
:1030D0000E94F84911E0811101C010E0CE01019673
:1030E0000E94984E01C011E0CE0145960E94984E74
:1030F0001123F1F025E030E044E050E062EE72E1AF
:10310000CE0101960E94F04EBE016F5F7F4F84ECAE
:1031100092E10E945E4ECE0101960E94984E84EC90
:1031200092E10E94FA4C7093C00D6093BF0D51C0A4
:1031300060E278E0CE0145960E94DC4EBE016B5EF7
:103140007F4F82EE92E10E94F849811117C065E23B
:1031500078E0CE0101960E94DC4EBE016F5F7F4F8A
:1031600082EE92E10E94F849FF24F394811101C09C
:10317000F12CCE0101960E94984E02C0FF24F394D8
:103180008E010B5E1F4FC8010E94984EFF2089F1EF
:1031900026E030E044E050E062EE72E1CE010196BC
:1031A0000E94F04EBE016F5F7F4F84EC92E10E945F
:1031B0005E4ECE0101960E94984E84EC92E10E94F0
:1031C000FA4C7093C20D6093C10D709342046093EA
:1031D000410462EE72E1CE0101960E94D44ECE010E
:1031E00001960E942960CE0101960E94984E0C948F
:1031F0007D0F6AE278E0C8010E94DC4EB80182EEE1
:1032000092E10E94F849811117C061E378E0CE0194
:1032100001960E94DC4EBE016F5F7F4F82EE92E10D
:103220000E94F849FF24F394811101C0F12CCE01D2
:1032300001960E94984E02C0FF24F394C8010E9498
:10324000984EFF2069F127E030E046E050E062EE62
:1032500072E1CE0101960E94F04EBE016F5F7F4F7A
:1032600084EC92E10E945E4ECE0101960E94984E3F
:1032700084EC92E10E94FA4C672B19F410921F0D16
:1032800003C081E080931F0D62EE72E1CE010196D2
:103290000E94D44ECE0101960E9429600C947022A7
:1032A00068E378E0CE0183960E94DC4EBE016D5D3E
:1032B0007F4F82EE92E10E94F849811129C06BE3B1
:1032C00078E0C8010E94DC4EB80182EE92E10E94D3
:1032D000F849811117C06EE378E0CE0101960E9493
:1032E000DC4EBE016F5F7F4F82EE92E10E94F84993
:1032F000FF24F394811101C0F12CCE0101960E94AC
:10330000984E02C0FF24F394C8010E94984E02C058
:10331000FF24F394CE0183960E94984EFF2009F477
:1033200024C1BAE0CB2ED12C412C512C3201AA243D
:10333000AA9483E0B82E6EE170E080E090E00E94F5
:10334000868D809110020E943C8DB5010E946CA771
:10335000072E000C880B990B0E94A1A220E030E000
:1033600040EA50E40E9400A39B01AC01C301B201FA
:103370000E942BA42B013C0191E0C91AD108D9F677
:1033800020E030E040E251E4C301B2010E94F1A428
:103390004B015C0161E478E0C8010E94DC4EB80199
:1033A00082EE92E10E94F849811117C065E478E04D
:1033B000CE0101960E94DC4EBE016F5F7F4F82EE10
:1033C00092E10E94F849EE24E394811101C0E12CBE
:1033D000CE0101960E94984E01C0EF2CC8010E94B8
:1033E000984EEE2009F43FC020E030E040E650E483
:1033F000C501B4010E9400A39B01AC0160E070E034
:1034000080E890E40E942AA4AB01BC0140930C0226
:1034100050930D0260930E0270930F0222E0CE01D2
:1034200001960E949D4EBE016F5F7F4F8AEC92E134
:103430000E945E4ECE0101960E94984E69E478E0AB
:10344000CE0101960E94DC4E6AEC72E1CE0101963B
:103450000E94E94DBC018AEC92E10E94494ECE01E6
:1034600001960E94984E68E578E0C8010E94DC4E03
:10347000B80182EE92E10E94F849811116C06DE513
:1034800078E0CE0101960E94DC4EBE016F5F7F4F57
:1034900082EE92E10E94F849FF24F394811101C069
:1034A000F12CCE0101960E94984EC8010E94984EC0
:1034B000FF2009F43FC020E030E040E650E4C501C1
:1034C000B4010E9400A39B01AC0160E070E080E2C7
:1034D00091E40E942AA4AB01BC01409308025093DE
:1034E000090260930A0270930B0222E0CE0101965A
:1034F0000E949D4EBE016F5F7F4F8AEC92E10E9459
:103500005E4ECE0101960E94984E62E678E0CE01B2
:1035100001960E94DC4E6AEC72E1CE0101960E9497
:10352000E94DBC018AEC92E10E94494ECE01019620
:103530000E94984E64E87BE0CE0101960E94DC4E2A
:103540006AEC72E1CE0101960E94E94DBC01C8010E
:103550000E94D44EC8010E948754C8010E94984E10
:10356000CE0101960E94984EC1C762E778E0CE0175
:1035700001960E94DC4EBE016F5F7F4F82EE92E1AA
:103580000E94F849F82ECE0101960E94984EFF2025
:1035900009F468C08091E6129091E712079708F449
:1035A000A5C746E050E062EE72E1CE0101960E94AE
:1035B0005480BE016F5F7F4F84EC92E10E945E4EAB
:1035C000CE0101960E94984E0E943A8FAB01BC0139
:1035D00040931302509314026093150270931602E5
:1035E00021E0C8010E949D4E61EA76E0CE0101967D
:1035F0000E94DC4EB801CE0101960E94E94D64E3C1
:1036000079E00E94D24DBC018AEC92E10E94494EC1
:10361000CE0101960E94984EC8010E94984E6AEC15
:1036200072E1CE0101960E94D44ECE0101960E9415
:103630008754CE0101960E94984E0E94BE8D28EEBE
:1036400033E040E050E00E94F9A3CA01B9010E94B2
:103650009FA26093820C7093830C8093840C909350
:10366000850C44C769E778E0CE0101960E94DC4EE4
:10367000BE016F5F7F4F82EE92E10E94F849F82E03
:10368000CE0101960E94984EFF20C1F18091E61272
:103690009091E712079708F429C746E050E062EEE0
:1036A00072E1CE0101960E945480BE016F5F7F4F90
:1036B00084EC92E10E945E4ECE0101960E94984EEB
:1036C0000E943A8FAB01BC01409380045093810467
:1036D000609382047093830421E0C8010E949D4E90
:1036E00061EB76E0CE0101960E94DC4EB801CE017E
:1036F00001960E94E94D64E379E083C360E878E0D5
:10370000C8010E94DC4EB80182EE92E10E94F849A5
:10371000811117C064E878E0CE0101960E94DC4E6A
:10372000BE016F5F7F4F82EE92E10E94F849FF2455
:10373000F394811101C0F12CCE0101960E94984EA4
:1037400002C0FF24F394C8010E94984EFF2009F4A0
:1037500055C080910602909107020E94C66E609348
:103760005704709358048093590490935A046093BB
:103770005D0D70935E0D80935F0D9093600D80E002
:1037800090E0A0E8BFE380935F0490936004A0936F
:103790006104B09362048093550D9093560DA093ED
:1037A000570DB093580D80911F0D882381F060E272
:1037B00074E080E490E10E94484F6091570470915A
:1037C00058048091590490915A040E94094510921E
:1037D000DA0C1092D90C80E090E00E94F27E4091C9
:1037E0005704509158046091590470915A0422E092
:1037F000C8010E949D4E68E878E053C661E978E010
:10380000C8010E94DC4EB80182EE92E10E94F849A4
:10381000811117C067E978E0CE0101960E94DC4E65
:10382000BE016F5F7F4F82EE92E10E94F849FF2454
:10383000F394811101C0F12CCE0101960E94984EA3
:1038400002C0FF24F394C8010E94984EFF2009F49F
:10385000B8C08091E6129091E7120797E8F046E031
:1038600050E062EE72E1CE0101960E945480BE01EA
:103870006F5F7F4F84EC92E10E945E4ECE01019615
:103880000E94984E0E943A8F6093470470934804B8
:103890008093490490934A04809104029091050218
:1038A00099270E94056EBC01990F880B990B0E9405
:1038B000A1A22DE038E643E55BE30E9400A36B0183
:1038C0007C012091A6043091A7044091A804509156
:1038D000A9040E949BA218164CF060918E0470916E
:1038E0008F0480919004909191041BC02091BA04A0
:1038F0003091BB044091BC045091BD04C701B60196
:103900000E94E0A587FF05C0C701B6010E94B07DF7
:1039100008C06091A2047091A3048091A4049091C6
:10392000A50420E030E048EC52E40E9400A36B01C3
:103930007C0120E030E0A9010E949BA2181634F01F
:10394000C12CD12CA8EAEA2EA1E4FA2EC092470499
:10395000D0924804E0924904F0924A04C0927D0D4E
:10396000D0927E0DE0927F0DF092800D80911F0D20
:10397000882381F06EE074E080E490E10E94484F7B
:1039800060914704709148048091490490914A04E1
:103990000E9409451092DA0C1092D90C80E090E058
:1039A0000E94F27E4091470450914804609149047E
:1039B00070914A0422E0C8010E949D4E6DE978E0B2
:1039C00070C567EA78E0C8010E94DC4EB80182EE5B
:1039D00092E10E94F849811117C06CEA78E0CE01AB
:1039E00001960E94DC4EBE016F5F7F4F82EE92E136
:1039F0000E94F849FF24F394811101C0F12CCE01FB
:103A000001960E94984E02C0FF24F394C8010E94C0
:103A1000984EFF2009F494C08091E6129091E7122D
:103A20000697F8F045E050E062EE72E1CE010196B3
:103A30000E945480BE016F5F7F4F84EC92E10E9430
:103A40005E4ECE0101960E94984E0E943A8F0E94CF
:103A500021A660934F047093500480935104909377
:103A600052048091C6049091C7040E94579B20E0A5
:103A700030E048E051E40E94F1A46093C2047093E6
:103A8000C3048093C4049093C50460936D0D709338
:103A90006E0D80936F0D9093700D80914F049091F7
:103AA0005004A0915104B09152048093750D9093ED
:103AB000760DA093770DB093780D80911F0D88231C
:103AC00041F16DEF73E080E490E10E94484F209156
:103AD0004F0430915004409151045091520460E0E1
:103AE00070E080E291E40E949FA641E050E00E94D5
:103AF0008A7C61EB78E080E490E10E941350609151
:103B0000C2047091C3048091C4049091C5040E94C2
:103B100009451092DA0C1092D90C80E090E00E94D6
:103B2000F27E4091C2045091C3046091C40470912C
:103B3000C50423E0C8010E949D4E68EB78E0BEC03A
:103B400063EC78E0C8010E94DC4EB80182EE92E19D
:103B50000E94F849811117C068EC78E0CE01019607
:103B60000E94DC4EBE016F5F7F4F82EE92E10E94A9
:103B7000F849FF24F394811101C0F12CCE01019684
:103B80000E94984E02C0FF24F394C8010E94984EF0
:103B9000FF2009F49FC08091E6129091E7120697EA
:103BA000F8F045E050E062EE72E1CE0101960E942D
:103BB0005480BE016F5F7F4F84EC92E10E945E4EA5
:103BC000CE0101960E94984E0E943A8F0E9421A633
:103BD00060934B0470934C0480934D0490934E0477
:103BE0008091C6049091C7040E94579B20E030E06A
:103BF00048E051E40E94F1A46093BE047093BF04B6
:103C00008093C0049093C1046093710D7093720D02
:103C10008093730D9093740D80914B0490914C049C
:103C2000A0914D04B0914E048093790D90937A0D3C
:103C3000A0937B0DB0937C0D80911F0D882341F1E3
:103C40006DEE73E080E490E10E94484F20914B04B8
:103C500030914C0440914D0450914E0460E070E06E
:103C600080E291E40E949FA641E050E00E948A7C9D
:103C700061EB78E080E490E10E9413506091BE0413
:103C80007091BF048091C0049091C1040E940945C5
:103C90001092DA0C1092D90C80E090E00E94F27E33
:103CA0004091BE045091BF046091C0047091C10462
:103CB00023E0C8010E949D4E6DEC78E0CE01019694
:103CC0000E94DC4EB801CE0101960E94E94D61ECE4
:103CD00078E097C066ED78E0C8010E94DC4EB8013C
:103CE00082EE92E10E94F849811117C06AED78E0F6
:103CF000CE0101960E94DC4EBE016F5F7F4F82EEC7
:103D000092E10E94F849FF24F394811101C0F12C43
:103D1000CE0101960E94984E02C0FF24F394C80180
:103D20000E94984EFF2009F46FC09090020260E05C
:103D3000892D0E94008DF9E1AF2EB12CC12CD12C20
:103D40007601892D0E943C8DBC01990F880B990B3F
:103D50000E94A1A29B01AC01C701B6010E942BA445
:103D60006B017C016AE070E080E090E00E94868D4B
:103D7000A1E0AA1AB10829F720E030E040EA50E4B7
:103D8000C701B6010E9400A320E030E040E85AE3FA
:103D90000E9400A320E030E048EC51E40E94F1A42E
:103DA00060934304709344048093450490934604C5
:103DB0006093930D7093940D8093950D9093960D51
:103DC0001092DA0C1092D90C80E090E00E94F27E02
:103DD000409143045091440460914504709146041D
:103DE00022E0C8010E949D4E68E376E0CE01019674
:103DF0000E94DC4EB801CE0101960E94E94D65E0BB
:103E000076E00E94D24D56C36EED78E0C8010E9464
:103E1000DC4EB80182EE92E10E94F849811117C090
:103E200062EE78E0CE0101960E94DC4EBE016F5F2B
:103E30007F4F82EE92E10E94F849FF24F3948111B2
:103E400001C0F12CCE0101960E94984E02C0FF24C1
:103E5000F394C8010E94984EFF2009F43FC126E068
:103E600030E044E050E062EE72E1CE0101960E9443
:103E7000F04EBE016F5F7F4F84EC92E10E945E4E78
:103E8000CE0101960E94984E84EC92E10E94FA4C79
:103E90004B015C016B016FE276E0CE0101960E945E
:103EA000DC4EBE016F5F7F4F82EE92E10E9495492A
:103EB000AC014F5F5F4F62EE72E1C8010E94548017
:103EC000B80184EC92E10E945E4EC8010E94984EB7
:103ED000CE0101960E94984EF09000020E943A8F07
:103EE0002B013C011401B1E02B1A310880911F0D08
:103EF0008823B9F065E773E080E490E10E94484FC1
:103F00004AE050E0B40180E490E10E94C94F66EEBF
:103F10007BE080E490E10E941350C301B2010E9453
:103F200009456F2DC8010E94938618870F831D8253
:103F30001E82198289E08A8381E08B838C831C8AAC
:103F40001B8ACE0101960E945D47CE0101960E9418
:103F5000ED46CE0101960E941246EE80F12CEBE078
:103F6000EE16F1041CF0EAE0EE2EF12CFBE58F16C4
:103F7000910408F44CC071EBA72E7CE0B72E4501EC
:103F8000412C512C3201C12CD12CCE14DF04BCF4B5
:103F90006C2DCE0101960E94A2459B01AC01D4017B
:103FA0006D937D938D939D934D01C301B2010E944A
:103FB0002BA42B013C01BFEFCB1ADB0AE6CFB701E4
:103FC0000F2C000C880B990B0E94A1A29B01AC0145
:103FD000C301B2010E94F1A42B013C01C12CD12CE0
:103FE000CE14DF040CF058C0F501208131814281EC
:103FF0005381C301B2010E942AA4D5016D937D9320
:104000008D939D935D01BFEFCB1ADB0AE9CF1C14A2
:104010001D0414F5EC14FD0424F41701E1E02E1A3C
:104020003108622DCE0101960E94A2459B01AC0190
:10403000C101880F991F880F991FBC016F54734FDE
:104040001B01C301B2010E942AA4D1016D937D938B
:104050008D939C93139720C0CD28F1F481EBA82E6B
:104060008CE0B82EC12CD12CCE14DF04ACF46C2D16
:10407000CE0101960E94A2459B01AC01C301B20191
:104080000E942AA4F50161937193819391935F013A
:10409000FFEFCF1ADF0AE8CFE1EBFCE0A7E9BDE0D4
:1040A00041915191619171914D935D936D937D9388
:1040B0002CE0E93DF207A1F71092DA0C1092D90C2E
:1040C00080E090E00E94F27E44E050E062EE72E117
:1040D000C8010E94548066EE78E0E3C167E079E0B1
:1040E000C8010E94DC4EB80182EE92E10E94F849BC
:1040F000811117C06BE079E0CE0101960E94DC4E81
:10410000BE016F5F7F4F82EE92E10E94F849FF246B
:10411000F394811101C0F12CCE0101960E94984EBA
:1041200002C0FF24F394C8010E94984EFF2009F4B6
:1041300055C080910602909107020E94C66E60935E
:1041400053047093540480935504909356046093E1
:10415000610D7093620D8093630D9093640D80E008
:1041600090E5A3ECB7E480935B0490935C04A09388
:104170005D04B0935E048093590D90935A0DA09303
:104180005B0DB0935C0D80911F0D882381F06FEC67
:1041900073E080E490E10E94484F60915304709175
:1041A000540480915504909156040E940945109240
:1041B000DA0C1092D90C80E090E00E94F27E4091DF
:1041C000530450915404609155047091560422E0B8
:1041D000C8010E949D4E6FE079E063C16AE179E019
:1041E000C8010E94DC4EB80182EE92E10E94F849BB
:1041F000811117C06EE179E0CE0101960E94DC4E7C
:10420000BE016F5F7F4F82EE92E10E94F849FF246A
:10421000F394811101C0F12CCE0101960E94984EB9
:1042200002C0FF24F394C8010E94984EFF2009F4B5
:1042300084C08091E6129091E7120497E8F044E080
:1042400050E062EE72E1CE0101960E945480BE0100
:104250006F5F7F4F84EC92E10E945E4ECE0101962B
:104260000E94984E0E943A8F60935F04709360049E
:10427000809361049093620480915F049091600444
:10428000A0916104B09162048093550D9093560DF6
:10429000A093570DB093580D80911F0D882391F076
:1042A00066EB73E080E490E10E94484F60915F0408
:1042B00070916004809161049091620442E050E04A
:1042C0000E948A7C80910602909107020E94C66E2D
:1042D00060935704709358048093590490935A0440
:1042E00060935D0D70935E0D80935F0D9093600DF4
:1042F00080911F0D882381F06CEA73E080E490E1E7
:104300000E94484F6091570470915804809159045D
:1043100090915A040E9409451092DA0C1092D90C1F
:1043200080E090E00E94F27E409157045091580442
:104330006091590470915A04AEC06AE279E0C801F4
:104340000E94DC4EB80182EE92E10E94F849811190
:1043500017C06EE279E0CE0101960E94DC4EBE01EC
:104360006F5F7F4F82EE92E10E94F849FF24F39441
:10437000811101C0F12CCE0101960E94984E02C01D
:10438000FF24F394C8010E94984EFF2009F4AEC0A8
:104390008091E6129091E7120497E8F044E050E033
:1043A00062EE72E1CE0101960E945480BE016F5F01
:1043B0007F4F84EC92E10E945E4ECE0101960E94F6
:1043C000984E0E943A8F60935B0470935C048093D4
:1043D0005D0490935E0480915B0490915C04A091D5
:1043E0005D04B0915E048093590D90935A0DA09393
:1043F0005B0DB0935C0D80911F0D882391F063E9F4
:1044000073E080E490E10E94484F60915B047091FA
:104410005C0480915D0490915E0442E050E00E9453
:104420008A7C80910602909107020E94C66E60937A
:1044300053047093540480935504909356046093EE
:10444000610D7093620D8093630D9093640D809164
:104450001F0D882381F069E873E080E490E10E94F9
:10446000484F609153047091540480915504909189
:1044700056040E9409451092DA0C1092D90C80E083
:1044800090E00E94F27E4091530450915404609158
:1044900055047091560422E0C8010E949D4E62E2CC
:1044A00079E0CE0101960E94DC4EB801CE01019662
:1044B0000E94E94DBC018AEC92E10E94494ECE0176
:1044C00001960E94984EC8010E94984E6AEC72E1D3
:1044D000CE0101960E94D44ECE0101960E948754CF
:1044E000CE0101960E94984E109212028091120203
:1044F000882371F062EE72E1CE0101960E94D44EE3
:10450000CE0101960E942960CE0101960E94984E2C
:104510000E94BE8D6093860C7093870C8093880CEC
:104520009093890C6AE37CE082EE92E10E94344E23
:10453000CA5BDF4F0FB6F894DEBF0FBECDBFDF9171
:10454000CF911F910F91FF90EF90DF90CF90BF9090
:10455000AF909F908F907F906F905F904F903F9023
:104560002F9008952F923F924F925F926F927F9279
:104570008F929F92AF92BF92CF92DF92EF92FF9273
:104580000F931F93CF93DF93CDB7DEB7CA54D109F2
:104590000FB6F894DEBF0FBECDBF26969FAF8EAF8D
:1045A0002697E090A90CF090AA0C80911F0D88230B
:1045B00061F06AE476E080E490E10E94484F26963C
:1045C0008EAD9FAD26970E94E75F26960EAD1FAD7C
:1045D00026970B5F1F4F0530110540F18091A90C04
:1045E0009091AA0C26962EAD3FAD26972817390735
:1045F00039F10E94927F0E94976B26964EAD5FAD77
:1046000026975093AA0C4093A90CBA01CE010196AB
:104610000E946F5EBE016F5F7F4F86ED92E10E9448
:104620005E4ECE0101960E94984E0AC026968EAD2F
:104630009FAD2697029621F40E94A76B0C94133726
:104640006AE37CE08AEC92E10E94344E0530110569
:1046500090F066EE7BE0CE0101960E94DC4E4AE0CF
:1046600050E06FEF7FEFCE0101960E94FA60CE011D
:1046700001960E94984E2696EEADFFAD26977A964B
:10468000E633F10510F00C9421368827EE58FF4FE1
:104690008F4F0C947FA78091220D882309F426C1A7
:1046A00086E09FE00E94C85A61E080912A040E943F
:1046B000008D60E0809128040E94008D0E94DE5DE4
:1046C0000E94386B0E94556BAB01BC0123E0CE0108
:1046D00080960E949D4EBE01605E7F4FCE01019686
:1046E0000E94D44E65E779E0CE0101960E94D24D3A
:1046F000BC0184EC92E10E94494ECE0101960E94D9
:10470000984ECE0180960E94984E6FE679E0CE01D9
:1047100001960E94DC4E64EC72E1CE0101960E948B
:10472000E94DBC018AEC92E10E94494ECE0101960E
:104730000E94984E0E94556B6B017C010E94618D16
:104740004B015C016EE170E080E090E00E94868D9C
:104750000E94556B2B013C010E94618D9B01AC01B5
:10476000281939094A095B0949015A0131ED8316B3
:1047700037E09306A104B1040CF441C0A7019601EF
:10478000C301B2010E942AA46B017C0120E030E049
:10479000A9010E94E0A518165CF426EA3BE944EC66
:1047A0005BE3C701B6010E949BA287FF0BC027C035
:1047B00026EA3BE944EC5BEBC701B6010E94E0A5A9
:1047C0001816ECF0C501B40128EE33E040E050E0EB
:1047D0000E94CDA3CA01B9010E94A1A24B015C01B4
:1047E00020E030E04AE754E4C701B6010E9400A38C
:1047F000A50194010E94F1A4AB01BC0103C040E0FB
:1048000050E0BA0122E0CE0180960E949D4EBE018A
:10481000605E7F4FCE0101960E94D44E62E379E044
:10482000CE0101960E94D24DBC018EEB92E10E9416
:10483000494ECE0101960E94984ECE0180960E946C
:10484000984E66E379E0CE0101960E94DC4E6EEB55
:1048500072E1CE0101960E94E94DBC018AEC92E121
:104860000E94084ECE0101960E94984E66EE7BE0B3
:10487000CE0101960E94DC4E6EEB72E1CE010196F4
:104880000E94E94DBC0184EC92E10E94084ECE01E9
:1048900001960E94984E6EE574E0CE0101960E944A
:1048A000CC4E4AE050E060E070E0CE0101960E94FC
:1048B0005560CE0101960E94984E64EC72E1CE01E3
:1048C00001960E94D44E45E050E06FEF7FEFCE019D
:1048D00001960E94C07FCE0101960E94984E6AE325
:1048E00079E08AEC92E10E94FA4DE3C1C090800425
:1048F000D0908104E0908204F09083040E94BE8DE9
:104900006CAF7DAF8EAF9FAF86E09FE00E94C85A2C
:1049100061E080912A040E94008D60E0809128046B
:104920000E94008D0E94DE5D0E94386B0E94556BD4
:1049300024966CAF7DAF8EAF9FAF24970E94618DA0
:104940004B015C016AE070E080E090E00E94868D9F
:104950006DE479E08AEC92E10E94344E20E030E090
:104960004AE754E4C701B6010E9400A32A966CAF3F
:104970007DAF8EAF9FAF2A97412C512C3201C12CB5
:10498000D12C7601C701B6010E94A1A22A962CADB6
:104990003DAD4EAD5FAD2A970E949BA287FF89C1B6
:1049A0000E94BE8D2CAD3DAD4EAD5FAD621B730B55
:1049B000840B950B0E949FA220E030E04AE754E46C
:1049C0000E94F1A4AB01BC0123E0CE0101960E943C
:1049D0009D4EBE016F5F7F4F84EC92E10E945E4E60
:1049E000CE0101960E94984E0E94556B6B017C018E
:1049F0000E94618D9B01AC01281939094A095B09A4
:104A000049015A0131ED831637E09306A104B10440
:104A10000CF443C020E030E0A901C701B6010E94B8
:104A2000E0A518165CF426EA3BE944EC5BE3C70119
:104A3000B6010E949BA287FF0BC02FC026EA3BE96C
:104A400044EC5BEBC701B6010E94E0A518162CF1FF
:104A5000C501B40128EE33E040E050E00E94CDA350
:104A6000CA01B9010E94A1A24B015C0124962CADA0
:104A70003DAD4EAD5FAD2497C701B6010E942AA49B
:104A800020E030E04AE754E40E9400A3A50194012D
:104A90000E94F1A44B015C0103C0812C912C5401B4
:104AA00064EC72E1CE0101960E94D44E64E379E099
:104AB000CE0101960E94D24DBC0184EC92E10E948D
:104AC000494ECE0101960E94984E23E0B701A601FF
:104AD000CE0180960E949D4EBE01605E7F4FCE014A
:104AE00001960E94D44E6BE679E0CE0101960E94B9
:104AF000D24DBC018EEB92E10E94494ECE0101964F
:104B00000E94984ECE0180960E94984E22E0B501F8
:104B1000A401CE0101960E949D4E62EF7BE0CE0182
:104B200080960E94DC4E64EC72E1CE0180960E9479
:104B3000E94D6EE679E00E94D24D6EEB72E10E9483
:104B4000E94D67E379E00E94D24DBE016F5F7F4F70
:104B50000E94E94D62E379E00E94D24DBC018AECEB
:104B600092E10E94084ECE0180960E94984ECE019E
:104B700001960E94984E20E030E0A901C501B401E1
:104B80000E94E0A587FD06C066EE7BE08EEB92E119
:104B90000E94FA4D22E0B501A401CE0180960E9448
:104BA0009D4EBE01605E7F4FCE0101960E94D44EA5
:104BB00062E379E0CE0101960E94D24DBC018EEBFA
:104BC00092E10E94084ECE0101960E94984ECE01BD
:104BD00080960E94984E6AEC72E1CE0101960E9486
:104BE000D44ECE0101960E948754CE0101960E94B8
:104BF000984EC301B20125E030E040E050E00E9451
:104C0000CDA3672B682B692B21F565E674E0CE01F7
:104C100001960E94CC4E45E050E060E070E0CE018D
:104C200001960E945560CE0101960E94984E6EEB4F
:104C300072E1CE0101960E94D44E45E050E06FEF44
:104C40007FEFCE0101960E94C07FCE0101960E94A7
:104C5000984E6AE37CE08AEC92E10E94344E65E073
:104C600070E080E090E00E94868D0E94BE8D6B0116
:104C70007C012CAD3DAD4EAD5FADC21AD30AE40A46
:104C8000F50A0E94556B24966CAF7DAF8EAF9FAF37
:104C900024970E94618D4B015C016AE070E080E026
:104CA00090E00E94868D3FEF431A530A630A730A0D
:104CB00069CE60E080912A040E94008D0C944F36EA
:104CC00080910002909101020E9473700C944F3603
:104CD000409102022B964FAF2B9760E0842F0E94E9
:104CE000008D8091220D811109C08091BF11811129
:104CF0000EC08FE090E0A0E0B0E00DC023E030E017
:104D000040E050E02CAF3DAF4EAF5FAF08C083E056
:104D100090E0A0E0B0E08CAF9DAFAEAFBFAF64E776
:104D200074E08AEC92E10E940E4E6AEC72E1CE01D0
:104D300001960E94D44E4AE050E06FEF7FEFCE0123
:104D400001960E945560CE0101960E94984E2196D0
:104D50001FAE219727961FAE2797212C312CC12CEF
:104D6000D12C760102E310E0812C912C54012B967A
:104D70008FAD2B970E943C8D092E000CAA0BBB0B0C
:104D8000880E991EAA1EBB1E65E070E080E090E0D0
:104D90000E94868D0150110951F7409043045090B4
:104DA00044046090450470904604C501B4010E941B
:104DB000A1A220E030E040EA50E40E9400A320E0FD
:104DC00030E040E85AE30E9400A320E030E048E4ED
:104DD00052E40E94F1A4A30192010E942AA420E0BF
:104DE00030E040E751E40E9400A34B015C01A301C5
:104DF00092016AE979E989E390E40E942AA49B017F
:104E0000AC01C501B4010E94F1A420E030E0A90189
:104E10000E942BA420E030E040E251E40E9400A375
:104E20005B018C0121962FAD219727963FAD2797E7
:104E3000A1010E94E0A518163CF42196AFAE21977F
:104E40002796BFAE2797180120E030E0A901B501F1
:104E5000C8010E949BA287FF04C0A12CB12C00E0D6
:104E600010E022E0A501B801CE0180960E949D4E7F
:104E7000BE01605E7F4FCE0101960E94D44E62E774
:104E800079E0CE0101960E94D24DBC0184EC92E102
:104E90000E94494ECE0101960E94984ECE01809606
:104EA0000E94984E64EC72E1CE0101960E94D44EAD
:104EB0004AE050E060E070E0CE0101960E94C07FC1
:104EC000CE0101960E94984E0E94BE8D80908A0C61
:104ED00090908B0CA0908C0CB0908D0C950184015F
:104EE0000C591F4F2F4F3F4F061717072807390739
:104EF00010F40C9474360E94BE8D0E949FA22B0168
:104F00003C01C501B4010E94A1A220E030E048ECC0
:104F100051E40E942BA49B01AC01C301B2010E9489
:104F20009BA287FF02C00C9474366CE370E080E0B3
:104F300090E00E94868D9FEFC91AD90AE90AF90A02
:104F40002CAD3DAD4EAD5FAD2C153D054E055F055D
:104F50000CF008CF64E670E080E090E00E94868D5F
:104F60000E94927F64E670E080E090E00E94868D6F
:104F70006CE674E084EC92E10E940E4E64EC72E107
:104F8000CE0101960E94D44E44E150E060E070E012
:104F9000CE0101960E945560CE0101960E94984E66
:104FA00022E021964FAD219727965FAD2797B1015B
:104FB000CE0180960E949D4EBE01605E7F4FCE0165
:104FC00001960E94D44E62E779E0CE0101960E94DC
:104FD000D24DBC0184EC92E10E94494ECE01019673
:104FE0000E94984ECE0180960E94984E64EC72E129
:104FF000CE0101960E94D44E42E350E06FEF7FEF66
:10500000CE0101960E94C07FCE0101960E94984E6B
:1050100064E170E080E090E00E94868D0E94B37FA2
:105020006EE170E080E090E00E94868D6EE170E0BD
:1050300080E090E00E94868D67E779E0CE010196DE
:105040000E94DC4E64EC72E1CE0101960E94E94DB3
:105050006BE779E00E94D24D6AEC72E10E94E94D63
:10506000BC018AEC92E10E94494E0C94603580911B
:1050700004029091050299270E94056EBC01990FC8
:10508000880B990B0E94A1A22DE038E643E55BE373
:105090000E9400A36B017C012091A6043091A7041B
:1050A0004091A8045091A9040E949BA218164CF0AC
:1050B00060918E0470918F0480919004909191047E
:1050C0001BC02091BA043091BB044091BC045091A4
:1050D000BD04C701B6010E94E0A587FF05C0C70156
:1050E000B6010E94B07D08C06091A2047091A30433
:1050F0008091A4049091A50420E030E048EC52E4B3
:105100000E9400A320E030E048EA51E40E9400A39E
:1051100020914704309148044091490450914A0439
:105120000E94F1A46B017C0161E874E084EC92E1DF
:105130000E940E4E64EC72E1CE0101960E94D44EA4
:1051400042E350E060E070E0CE0101960E945560BD
:10515000CE0101960E94984E22E0B701A601CE0131
:1051600001960E949D4E65E879E0CE0180960E94EE
:10517000DC4EBE016F5F7F4FCE0180960E94E94DED
:105180006FE779E00E94D24DBC018AEC92E10E9467
:10519000494ECE0180960E94984ECE0101960E9403
:1051A000984E6AEC72E1CE0101960E94D44E42E321
:1051B00050E06FEF7FEFCE0101960E94C07FCE01DD
:1051C00001960E94984E8091220D882311F40C9430
:1051D0004F3660E273E080E090E0CCC20E94927FA4
:1051E00065EB74E08AEC92E10E940E4E6AEC72E18B
:1051F000CE0101960E94D44E4AE050E060E070E09B
:10520000CE0101960E945560CE0101960E94984EF3
:105210006CEA74E084EC92E10E940E4E64EC72E160
:10522000CE0101960E94D44E44E150E06FEF7FEF33
:10523000CE0101960E94C07FCE0101960E94984E39
:1052400080918E0C90918F0C8230910549F40E94D0
:10525000148E81111AC010928F0C10928E0C15C0F2
:10526000892BC9F40E94148E882339F082E090E0E3
:1052700090938F0C80938E0C08C00E94148E811125
:10528000F5CF0E94148E8111F1CF80918E0C9091F8
:105290008F0C029741F160EA74E08AEC92E10E947F
:1052A0000E4E6AEC72E1CE0101960E94D44E4AE0A5
:1052B00050E060E070E0CE0101960E945560CE01A2
:1052C00001960E94984E6AEC72E1CE0101960E940E
:1052D000D44E66EE7BE0CE0101960E94D24D64EC86
:1052E00072E10C942A338AE090E00E94D36B6B0148
:1052F0007C0120E030E0A9010E949BA2181634F046
:105300008AE090E00E94D36B6B017C010BE010E01F
:1053100020E030E042ED53E4C701B6010E949BA2B9
:10532000181684F00150110969F068EC70E080E013
:1053300090E00E94868D83E090E00E94D36B6B0129
:105340007C01E6CF20E030E0A901C701B6010E9450
:105350009BA218163CF062E974E08AEC92E10E948C
:105360000E4E31C020E030E048EC52E4C701B601F7
:105370000E949BA287FF02C021E001C020E0B7018C
:10538000A601CE0101960E949D4E64E879E0CE010F
:1053900080960E94DC4EBE016F5F7F4FCE018096EB
:1053A0000E94E94D69E879E00E94D24DBC018AEC87
:1053B00092E10E94494ECE0180960E94984ECE0105
:1053C00001960E94984E6AEC72E1CE0101960E940D
:1053D000D44E42E350E06FEF7FEFCE0101960E9482
:1053E000C07FCE0101960E94984E69E874E084EC7B
:1053F00092E10E940E4E64EC72E1CE0101960E9491
:10540000D44E42E350E060E070E0CE0101960E948D
:105410005560D5CE0E94BE8D2B013C0186E09FE0F9
:105420000E94C85A64E670E080E090E00E94868D99
:1054300040E855E260E070E086E09FE00E948F7EE9
:1054400064E670E080E090E00E94868D6EEE74E08D
:1054500084EC92E10E940E4E64EC72E1CE01019662
:105460000E94D44E42E350E06FEF7FEFCE010196F1
:105470000E945560CE0101960E94984E63EE74E042
:1054800084EC92E10E940E4E64EC72E1CE01019632
:105490000E94D44E42E350E06FEF7FEFCE010196C1
:1054A0000E94C07FCE0101960E94984E8091AF0C61
:1054B0009091B00C8D7F1CAEC12CD12CE12CF12C25
:1054C00000E010E0019709F47AC0BCED8B2EB5E046
:1054D0009B2EA12CB12CAE01405E5F4F59AF48AF5F
:1054E000CE014E969BAF8AAF0E94BE8DDC01CB01F0
:1054F00084199509A609B709883B9B40A105B10508
:1055000008F05DC086E09FE00E946F4A892B09F495
:105510004FC080920A0F90920B0FA0920C0FB09286
:105520000D0F0E945B7E97FD06C082349105C9F77E
:1055300080E090E002C08FEF9FEF892BC9F59E01BC
:105540002F5F3F4F22963FAF2EAF229719010E9447
:105550005B7E97FF06C089818D3451F520E030E0F5
:1055600009C0D1018D931D01E8ADF9ADEA17FB0724
:1055700071F7F1CF2296AEADBFAD22978D912296F5
:10558000BFAFAEAF2297280F311DEAADFBADAE170E
:10559000BF0781F72E5B3F4F8E8D90E0982F8827B5
:1055A0004F8D840F911D2817390711F40C9478360C
:1055B00062E370E080E090E00E94868D95CF0E94CB
:1055C000BE8DDC01CB0184199509A609B709883B7A
:1055D0009B40A105B10518F42CAD2111BDC00E945E
:1055E000927F64EC72E1CE0180960E94D44E42E339
:1055F00050E066E070E0CE0180960E945560CE01DA
:1056000080960E94984E4CAD442311F40C94913630
:1056100082E090E09093B00C8093AF0CB601CE0185
:1056200080960E946F5EB701CE0186960E946F5EE3
:10563000B801CE01C2960E946F5EBE016E5C7F4FC4
:10564000CE018C960E94D44E60E778E0CE018C9615
:105650000E94D24DBE016A5D7F4F0E94E94D60E716
:1056600078E00E94D24DBE01605E7F4F0E94E94DFE
:10567000BC018AEC92E10E94494ECE018C960E94B8
:10568000984ECE01C2960E94984ECE0186960E94F8
:10569000984ECE0180960E94984E6AEC72E1CE013F
:1056A00080960E94D44E4AE050E06FEF7FEFCE012B
:1056B00080960E94C07FCE0180960E94984E6DED2C
:1056C00074E08BEC93E10E94484FB601CE018096C6
:1056D0000E946F5EB701CE0186960E946F5EB80190
:1056E000CE018C960E946F5E6DE879E0CE01C29685
:1056F0000E94DC4EBE01645D7F4FCE01C2960E94C7
:10570000E94D66EE7BE00E94D24DBE016A5D7F4F9F
:105710000E94E94D66EE7BE00E94D24DBE01605EC4
:105720007F4F0E94E94D6DE979E00E94D24DBC01A6
:105730008AEC92E10E94494ECE01C2960E94984E98
:10574000CE018C960E94984ECE0186960E94984E6D
:10575000CE0180960E94984E62E370E080E090E077
:105760000E94868D86E09FE00E94C85A62E370E046
:1057700080E090E00E94868D0C944F3600910602E6
:105780001091070263EA79E084EC92E10E94344EC2
:105790000E94927F64EC72E1CE0101960E94D44E89
:1057A0004AE050E06FEF7FEFCE0101960E94556016
:1057B000CE0101960E94984EC8010E94C66E2496A2
:1057C0006CAF7DAF8EAF9FAF2497809057049090C1
:1057D0005804A0905904B0905A04A5019401609116
:1057E00053047091540480915504909156040E9482
:1057F0002AA42B013C0120E030E0A9010E949BA2D9
:10580000882309F453C0C0905F04D0906004E090F6
:105810006104F090620420E030E0A901C701B60104
:105820000E949BA218160CF041C080915B049091DD
:105830005C04A0915D04B0915E048CAF9DAFAEAFEF
:10584000BFAF9C01AD01C701B6010E949BA2882396
:1058500069F1A70196016CAD7DAD8EAD9FAD0E9443
:10586000F1A40E942CA66CAF7DAF8EAF9FAFA501B7
:10587000940124966CAD7DAD8EAD9FAD24970E94B2
:105880002AA4A30192010E94F1A42CAD3DAD4EAD1E
:105890005FAD0E9400A30E945EA59B01AC01C70101
:1058A000B6010E9400A36B017C0103C0C12CD12C66
:1058B000760164EC72E1CE0101960E94D44E4AE07A
:1058C00050E060E070E0CE0101960E945560CE018C
:1058D00001960E94984E20E030E64AEE56E4C70159
:1058E000B6010E94E0A518163CF46AEF74E08AEC59
:1058F00092E10E940E4E25C021E0B701A601CE0123
:1059000080960E949D4E6DEA79E0CE0101960E943C
:10591000DC4EBE01605E7F4FCE0101960E94E94DD4
:1059200061EB79E00E94D24DBC018AEC92E10E94C9
:10593000494ECE0101960E94984ECE0180960E945B
:10594000984E6AEC72E1CE0101960E94D44E4AE074
:1059500050E06FEF7FEFCE0101960E94C07FCE0135
:1059600001960E94984E64E670E080E090E00E940C
:10597000868D29CC00918C0410918D040E94927F19
:10598000C8010E94056E8C0162E370E080E090E047
:105990000E94868DB801110F880B990B0E94A1A25D
:1059A00020E030E040EA50E40E9400A320E030EC28
:1059B0004FE754E40E94F1A4AB01BC0123E0CE0107
:1059C00001960E949D4E68E779E0CE0180960E9484
:1059D000DC4EBE016F5F7F4FCE0180960E94E94D85
:1059E00065E076E00E94D24DBC018AEC92E10E9413
:1059F000494ECE0180960E94984ECE0101960E949B
:105A0000984E65EB79E084EC92E10E94344E64ECB0
:105A100072E1CE0101960E94D44E4AE050E068E067
:105A200070E0CE0101960E945560CE0101960E9461
:105A3000984E6AEC72E1CE0101960E94D44E4AE083
:105A400050E06FEF7FEFCE0101960E94C07FCE0144
:105A500001960E94984E64EC72E18AEC92E10E94F9
:105A6000084EB1CB9091A80C81E089278093A80CB7
:105A70008091220D882331F06AEC72E189E69EE084
:105A80000E94857A68EC70E080E090E073CE10921E
:105A9000220D0C944F3681E08093220D8093CD111E
:105AA0008091C411882349F16FEF77E086ED92E190
:105AB0000E94344E86EE9FEF9093AA0C8093A90C1F
:105AC0002091C7113091C8118091C9119091CA11CC
:105AD0008217930724F01092CA111092C9111092E4
:105AE000BB111092BC111092BD111092BE116CE24C
:105AF00071E080E090E00E94868D66ED72E18CEDB1
:105B000092E10E94494E8091A90C9091AA0C909329
:105B1000210D8093200D0C944F36809127148823FB
:105B200021F0109227140C944F360E9442890C9455
:105B30004F3683EA9FE00E94C85A40E052EC61E091
:105B400070E083EA9FE00E948F7E8CED95E0A0E0FC
:105B5000B0E08093A70F9093A80FA093A90FB093E4
:105B6000AA0F64E670E080E090E00E94868D80914C
:105B70008E0C90918F0C019759F483E090E00E9475
:105B8000296E811140C010928F0C10928E0C1AC099
:105B900081E090E00E94296E882339F081E090E056
:105BA00090938F0C80938E0C0DC083E090E00E9448
:105BB000296E8111F3CF83E090E00E94296E81115C
:105BC000EDCF06C080918E0C90918F0C0197D9F08B
:105BD00069E375E084EC92E10E940E4E64EC72E1A0
:105BE000CE0101960E94D44E44E150E06FEF7FEF6A
:105BF000CE0101960E94C07FCE0101960E94984E70
:105C00006DE275E0CFC061E275E08AEC92E10E943E
:105C10000E4E6AEC72E1CE0101960E94D44ECE0186
:105C200001960E942960CE0101960E94984E62E37F
:105C300070E080E090E00E94868D6AEC72E1CE0117
:105C400001960E94D44E42E350E06FEF7FEFCE0109
:105C500001960E945560CE0101960E94984E65E122
:105C600075E084EC92E10E940E4E64EC72E1CE018C
:105C700001960E94D44E44E150E06FEF7FEFCE01D9
:105C800001960E94C07FCE0101960E94984E8BEB38
:105C900088A38AEA89A381E08AA3E12CF12CC12C94
:105CA000D12C412C512C3201FAE02F2E312CC7017E
:105CB000B1010E946CA7892B49F443E050E0BE017A
:105CC000605E7F4F83EA9FE00E94144A65E070E0C7
:105CD00080E090E00E94868DBFEFEB1AFB0A00E0A7
:105CE00010E0812C912C540183EA9FE00E946F4ABE
:105CF000892B81F4E4E08E169104A104B10454F0E0
:105D000094E0C916D10464F4A0E9EA16A1E0FA0609
:105D100071F606C00630110514F40C94BD36F0CFB0
:105D2000C301B2010E94A1A220E030E040E251E4B0
:105D30000E94F1A420E030E040E85EE30E9400A36E
:105D40006B017C0120E030E040EA51E40E94E0A5D4
:105D5000181634F521E0B701A601CE0101960E9484
:105D60009D4E69E577E0CE0180960E94DC4EBE0133
:105D70006F5F7F4FCE0180960E94E94D6DEB79E019
:105D80000E94D24DBC018AEC92E10E94494ECE01A4
:105D900080960E94984ECE0101960E94984E06C0B1
:105DA00069E075E08AEC92E10E940E4E6AEC72E1C5
:105DB000CE0101960E94D44E4AE050E060E070E0CF
:105DC000CE0101960E945560CE0101960E94984E28
:105DD0006AEC72E1CE0101960E94D44E66EE7BE041
:105DE000CE0101960E94D24D64EC72E10E94E94D11
:105DF000BC018AEC92E10E94494ECE0101960E94BC
:105E0000984E83EA9FE00E94C85ADDC964ED75E0B0
:105E1000CE0101960E94CC4E4AE050E06FEF7FEF3A
:105E2000CE0101960E94C07FCE0101960E94984E3D
:105E300060918A0470918B04809141049091420496
:105E40000E94515274E1872E912CA12CB12CE12C8F
:105E5000F12C5FEFE51AF50AC501B4010E94868DA9
:105E600060918A0470918B04809141049091420466
:105E70000E9451528C0183E0E816F10434F03EE1B7
:105E8000E316F10444F4012B51F044E1840E911C1B
:105E9000A11CB11CDECF0115110509F00CC18091C8
:105EA0004104909142048B309105C9F480912813EC
:105EB00090912913A0912A13B0912B138093EC0C8D
:105EC0009093ED0CA093EE0CB093EF0C8091241303
:105ED00090912513A0912613B09127131DC08631F0
:105EE000910521F30C9701F58091DF0C9091E00C66
:105EF000A091E10CB091E20C8093EC0C9093ED0C2E
:105F0000A093EE0CB093EF0C8091DB0C9091DC0C25
:105F1000A091DD0CB091DE0C8093E80C9093E90C1D
:105F2000A093EA0CB093EB0C4091EC0C5091ED0C6B
:105F30006091EE0C7091EF0C21E0CE0101960E9471
:105F40009D4E66EB7BE0CE0180960E94DC4EBE014A
:105F50006F5F7F4FCE0180960E94E94DBC018AECB5
:105F600092E10E94494ECE0180960E94984ECE0149
:105F700001960E94984E4091E80C5091E90C609176
:105F8000EA0C7091EB0C21E0CE0101960E949D4E2F
:105F900060EC79E0CE0180960E94DC4EBE016F5F1E
:105FA0007F4FCE0180960E94E94DBC018AEC92E1C0
:105FB0000E94084ECE0180960E94984ECE01019616
:105FC0000E94984E62E879E08AEC92E10E94FA4DD4
:105FD0006AE37CE0CE0101960E94DC4E44E150E091
:105FE00060E070E0CE0101960E945560CE010196FE
:105FF0000E94984EC090EC0CD090ED0CE090EE0C0E
:10600000F090EF0C20E030E0A901C701B6010E943A
:10601000E0A520E030E040E05FE387FD05C0C70178
:10602000B6010E942BA404C0C701B6010E942AA495
:106030000E948AA5AB01BC01CE0101960E943F7B64
:10604000BE016F5F7F4F84EC92E10E945E4ECE01F5
:1060500001960E94984E60E087E00E94147B64ECF9
:1060600072E18BEC93E10E943A4F6FED8BEC93E180
:106070000E94334F66EC79E08BEC93E10E94135061
:106080006091E80C7091E90C8091EA0C9091EB0C16
:106090000E948AA54AE050E08BEC93E10E94C94F30
:1060A00062E879E08BEC93E10E94135064E670E0C3
:1060B00080E090E05FCB0F3F9FEF1907ACF066ECFC
:1060C00075E0CE0101960E94CC4E4AE050E060E0BF
:1060D00070E0CE0101960E945560CE0101960E94AB
:1060E000984E63EA75E047C00E3FAFEF1A0779F1AB
:1060F00065E975E0CE0101960E94CC4E4AE050E081
:1061000060E070E0CE0101960E945560CE010196DC
:106110000E94984E66E875E08AEC92E10E940E4E6D
:10612000B801CE0101960E946F5EBE016F5F7F4F86
:106130008AEC92E10E94084ECE0101960E94984E90
:1061400060E775E08AEC92E10E94764DA8C565E6AD
:1061500075E0CE0101960E94CC4E4AE050E060E02E
:1061600070E0CE0101960E945560CE0101960E941A
:10617000984E65E475E08AEC92E10E940E4E8FC560
:1061800080912C04882309F48AC56AE37CE0CE015F
:1061900001960E94DC4E4AE050E061E070E0CE01E2
:1061A00001960E945560CE0101960E94984E0E9471
:1061B000BB8F75C58091220D81110AC08091BF11DE
:1061C000811106C06EE1462E512C612C712C05C048
:1061D00053E0452E512C612C712C62EE75E08AEC57
:1061E00092E10E940E4E6AEC72E1CE0101960E948D
:1061F000D44E4AE050E06FEF7FEFCE0101960E944F
:10620000C07FCE0101960E94984E812C912C5401A2
:106210001CAE1DAE1EAE1FAE83E20E94F97A87E06F
:1062200090E00E94F47A0E94F27A66E970E080E0E1
:1062300090E00E94868D83E20E94F97A80E290E0ED
:106240000E94F47A0E94F27A66E970E080E090E0C1
:106250000E94868D62E070E083E290E00E94A65B7F
:10626000C12CD12C76018091F90C90E02091FA0C90
:10627000821B9109181619066CF48DED90E10E94AD
:106280009085FE2CED2CDC2CCC24C80ED11CE11CFE
:10629000F11CE9CFC701B6010E94A1A22AE939E9A0
:1062A00049E95FE30E94F1A40E948AA5AB01BC0109
:1062B00084169506A606B70614F44A015B01CE01C2
:1062C00080960E943F7BBE01605E7F4FCE010196AB
:1062D0000E94D44E69EC79E0CE0101960E94D24D25
:1062E000BC0184EC92E10E94494ECE0101960E94CD
:1062F000984ECE0180960E94984E64EC72E1CE01D9
:1063000001960E94D44E4EE150E060E070E0CE0174
:1063100001960E94FA60CE0101960E94984E2CAD23
:106320003DAD4EAD5FAD2F5F3F4F4F4F5F4F2CAF39
:106330003DAF4EAF5FAF42165306640675060CF0D4
:106340006BCFB501A401CE0180960E943F7BBE01B8
:10635000605E7F4FCE0101960E94D44E69EC79E0D9
:10636000CE0101960E94D24DBC0184EC92E10E94C4
:10637000494ECE0101960E94984ECE0180960E9411
:10638000984E64EC72E1CE0101960E94D44E4AE030
:1063900050E060E070E0CE0101960E945560CE01B1
:1063A00001960E94984EB501A401CE0101960E946B
:1063B0003F7B6DEC79E0CE0180960E94DC4EBE0101
:1063C0006F5F7F4FCE0180960E94E94D60ED79E0CE
:1063D0000E94D24D6AEC72E10E94E94DBC018AEC48
:1063E00092E10E94494ECE0180960E94984ECE01C5
:1063F00001960E94984EBAC90091880410918904B0
:1064000081E08093E00464E670E080E090E00E9428
:10641000868D0E94927FC8010E94056E60E074E044
:10642000681B790BCE0101960E946F5E65ED79E0E5
:10643000CE0180960E94DC4EBE016F5F7F4FCE0181
:1064400080960E94E94DBC018AEC92E10E94494E7F
:10645000CE0180960E94984ECE0101960E94984EE1
:1064600060E087E00E94147B62EF75E0CE01019648
:106470000E94CC4E42E350E068E070E0CE0101960D
:106480000E945560CE0101960E94984E6AEC72E11E
:10649000CE0101960E94D44E42E350E06FEF7FEFB1
:1064A000CE0101960E94C07FCE0101960E94984EB7
:1064B0006CED79E0C7C080918604909187040E94BA
:1064C000056E8C019093910C8093900C62E370E0C8
:1064D00080E090E00E94868DB801CE0101960E9476
:1064E0006F5EBE016F5F7F4F8AEC92E10E945E4E4D
:1064F000CE0101960E94984E809122139091231311
:10650000892B09F45EC06EE173E1CE0180960E9492
:10651000D44EBE01605E7F4FCE0101960E94D44EE4
:1065200044E150E060E070E0CE0101960E945560C9
:10653000CE0101960E94984E66EE79E0CE0101965A
:106540000E94DC4E6AEC72E1CE0101960E94E94D98
:10655000BC0184EC92E10E94494ECE0101960E945A
:10656000984E64EC72E1CE0101960E94D44E44E153
:1065700050E06FEF7FEFCE0101960E94C07FCE0109
:1065800001960E94984EBE01605E7F4FCE0101963B
:106590000E94D44E66EE7BE0CE0101960E94D24D61
:1065A00064EC72E10E94E94DBC018AEC92E10E9428
:1065B000494ECE0101960E94984ECE0180960C94D1
:1065C000E12861EF79E084EC92E10E94344E64ECC2
:1065D00072E1CE0101960E94D44E44E150E060E0A9
:1065E00070E0CE0101960E945560CE0101960E9496
:1065F000984E65ED79E0CE0101960E94DC4E6AEC82
:1066000072E1CE0101960E94E94DBC0184EC92E159
:106610000E94494ECE0101960E94984E64EC72E1B0
:10662000CE0101960E94D44E44E150E06FEF7FEF1F
:10663000CE0101960E94C07FCE0101960E94984E25
:1066400066EE79E0CE0101960E94DC4E6AEC72E1C2
:10665000CE0101960E94E94DBC018AEC92E10E94B4
:10666000494ECE0101960E94984E0C94E3288091E9
:106670002C04882309F413C38091220D811104C0D6
:106680008091BF11882329F082E090E00E94608011
:1066900006C30E94A45E03C30E94087389E69EE0BD
:1066A0000E940D4BFCC26AE076E084EC92E10E940D
:1066B0000E4E64EC72E1CE0101960E94D44E4AE087
:1066C00050E060E070E0CE0101960E945560CE017E
:1066D00001960E94984E309010028091A00C81117A
:1066E00005C00E94BE8D81E08093A00C8091980C23
:1066F000811105C00E94BE8D81E08093980C10929C
:10670000970C1092960C0091960C1091970C0832F1
:1067100011050CF07BC0832D0E943C8DF801EE0F1B
:10672000FF1FE153F24F918380830E948B7C20E016
:1067300030E040EA50E40E9400A320E030E040E86E
:106740005AE30E9400A32B013C0180900C02909020
:106750000D02A0900E02B0900F02A501940160916D
:1067600008027091090280910A0290910B020E9426
:106770002AA49B01AC0160E070E080EC90E40E94F0
:106780002AA46B017C0120E030E0A9010E949BA2B9
:1067900020E030E040E650E4811105C0C301B201C1
:1067A0000E9400A31EC0C301B2010E9400A3A50164
:1067B00094010E942BA420E030E040E850E40E94C5
:1067C0002AA4A70196010E94F1A420E030E040EC49
:1067D00050E40E9400A320E030E040E850E40E9432
:1067E0002BA46093920C7093930C8093940C9093D1
:1067F000950C64E170E080E090E00E94868D0F5F70
:106800001F4F1093970C0093960C7DCFC090920C65
:10681000D090930CE090940CF090950C20E030E038
:10682000A901C701B6010E94E0A587FD1EC022E0B4
:10683000B701A601CE0101960E949D4E65EF79E059
:10684000CE0180960E94DC4EBE016F5F7F4FCE016D
:1068500080960E94E94DBC018AEC92E10E94494E6B
:10686000CE0180960E94984E04C26BEF75E08AECD0
:1068700092E10E940E4E01C280912C04882309F4FB
:106880000EC28091220D81112BC08091BF11811108
:1068900027C0C0908004D0908104E0908204F090E2
:1068A000830420E030E04AE754E4C701B6010E94C7
:1068B00000A30E948AA54B015C0120E030E040EA81
:1068C00050E4C701B6010E9400A320E030E040EA96
:1068D00050E40E942BA40E948AA5A501940108C03F
:1068E00021E030E040E050E06AE070E080E090E0DD
:1068F0000E945D76D4C18091BF0D9091C00D00972C
:10690000F1F581E090E09093C00D8093BF0D69EFA9
:1069100079E0CE0101960E94DC4ECE0101960E94E4
:106920002960CE0101960E94984E62E07AE0CE0185
:1069300001960E94DC4E6FEB73E1CE0101960E943E
:10694000E94DBC01CE0180960E94D44E48EC50E047
:106950006FEF7FEFCE0180960E945560CE0180964A
:106960000E94984ECE0101960E94984E89E69EE0C4
:106970000E94C85A40E052EC61E070E078C0029793
:1069800099F51092C00D1092BF0D68E07AE0CE012B
:1069900001960E94DC4ECE0101960E942960CE0134
:1069A00001960E94984E66E17AE0CE0101960E941F
:1069B000DC4E6FEB73E1CE0101960E94E94DBC0104
:1069C000CE0180960E94D44E48EC50E06FEF7FEFEE
:1069D000CE0180960E945560CE0180960E94984E0E
:1069E000CE0101960E94984E8091BF0D9091C00DEE
:1069F0000197A9F582E090E09093C00D8093BF0DC0
:106A00006AE17AE0CE0101960E94DC4ECE01019649
:106A10000E942960CE0101960E94984E6BE27AE0B6
:106A2000CE0101960E94DC4E6FEB73E1CE01019620
:106A30000E94E94DBC01CE0180960E94D44E48ECE4
:106A400050E06FEF7FEFCE0180960E945560CE013F
:106A500080960E94984ECE0101960E94984E89E63B
:106A60009EE00E94C85A40E855E260E070E089E686
:106A70009EE00E948F7E1092DA0C1092D90C80E07A
:106A800090E00E94F27E60E37AE0CE0101960E94DF
:106A9000DC4E69EB73E1CE0101960E94E94DBC0129
:106AA000CE0180960E94D44E40ED57E06FEF7FEF0D
:106AB000CE0180960E94C07FCE0180960E94984EA3
:106AC000CE0101960E94984EEAC08091470D9091A8
:106AD000480D892BA1F481E090E09093480D8093BC
:106AE000470D8EED93E09093DA0C8093D90C0E94C1
:106AF0001B7F68EC70E080E090E00E94868DE0E013
:106B0000F0E01995CCC00E94D28E0E94927F0E9424
:106B1000976BC5C09091C41181E089278093C411FF
:106B2000882369F163E476E08AEC92E10E940E4EDC
:106B30000E94BE8D6093BB117093BC118093BD11F8
:106B40009093BE118091C7119091C8111816190623
:106B50005CF42091C9113091CA112817390724F02B
:106B60001092CA111092C9119091CB118091C61147
:106B700098175CF01092CB111092CC1106C06BE309
:106B800076E08AEC92E10E940E4E8091C4118093CF
:106B9000BF116AEC72E1CE0101960E94D44E4AE028
:106BA00050E068E070E0CE0101960E945560CE0191
:106BB00001960E94984E6EE276E0CE0101960E9408
:106BC000CC4E4AE050E06FEF7FEFCE0101960E947D
:106BD000C07FCE0101960E94984E60E276E08AEC7A
:106BE00092E10E94764D64E87BE0CE0101960E941E
:106BF000DC4E6AEC72E1CE0101960E94E94DBC01C7
:106C00008AEC92E10E94494ECE0101960E94984E74
:106C10008091220D8093CD118CE291E00E943F7F04
:106C20008091220D8823D9F16FEF77E086ED92E114
:106C30000E94344E86EE9FEF9093AA0C8093A90C8D
:106C40002EC0F092AA0CE092A90C63E176E08AECE7
:106C500092E10E940E4E6AE37CE0CE0101960E9412
:106C6000DC4E4AE050E060E070E0CE0101960E9408
:106C70005560CE0101960E94984E6AEC72E1CE01F9
:106C800001960E94D44E4AE050E06FEF7FEFCE01B4
:106C900001960E94C07FCE0101960E94984E80917D
:106CA000CE129091CF120097C1F0419740F42696F2
:106CB0002EAD3FAD2697223031050CF0A1C06AEC15
:106CC00072E1CE0101960E94D44ECE0101960E943F
:106CD0008754CE0101960E94984E64E670E080E0F1
:106CE00090E00E94868D9FC00E94B37F0C949527F0
:106CF0000C8110E0102F00278D81080F111DEE80F0
:106D0000F12CFE2CEE248F81E80EF11CC884D12CCE
:106D1000DC2CCC248985C80ED11C31E03CAF0C940E
:106D2000D82A62ED74E08AEC92E10E940E4E6AEC81
:106D300072E1CE0180960E94D44E4AE050E060E0BD
:106D400070E0CE0180960E94C07FCE0180960E94A6
:106D5000984E6FEB74E08AEC92E10E940E4E8091A7
:106D6000AF0C9091B00C029711F00C94AC2B1092D8
:106D7000B00C1092AF0C0C94AC2B83EA9FE00E94F5
:106D80006F4A892B69F083EA9FE00E944D4AE1E057
:106D9000F0E0EC0FFD1FE00FF11F80830F5F1F4F2E
:106DA00065E070E080E090E00E94868D063011057D
:106DB00001F5998188A198131CC09A8189A1981323
:106DC00018C09B818AA1981314C08D8190E0A0E027
:106DD000B0E0BA2FA92F982F88272C81820F911D00
:106DE000A11DB11D480E591E6A1E7B1EFFEFCF1A52
:106DF000DF0A2FEF821A920AA20AB20A0C94742EAA
:106E00006AEC72E1CE0101960E94D44E4AE050E055
:106E10006FEF7FEFCE0101960E94C07FCE010196F9
:106E20000E94984E4CCFC65BDF4F0FB6F894DEBF82
:106E30000FBECDBFDF91CF911F910F91FF90EF90CB
:106E4000DF90CF90BF90AF909F908F907F906F908A
:106E50005F904F903F902F9008952F923F924F92C6
:106E60005F926F927F928F929F92AF92BF92CF92DA
:106E7000DF92EF92FF920F931F93CF93DF93CDB7E3
:106E8000DEB728970FB6F894DEBF0FBECDBFFC016A
:106E90008FEE90E1938782878091EC1090E0958748
:106EA00084878091B91190E0978786878091E91057
:106EB000853009F063C68091F1109091F2108858E6
:106EC00091098D35910588F48091EC10843041F45E
:106ED0008091F3109091F4108097479708F47DC04B
:106EE0008091EC10843408F05EC08091EC108A31FF
:106EF00008F4D5C08091EF109091F010843F91403C
:106F000050F4118610868FEF9FEFDC018483958308
:106F1000A683B7833CC08091F1109091F2108597C1
:106F20004B9708F0BCC005EFE02E00E1F02E82E0A8
:106F300090E040E050E0BA018C010F5F1F4F2091BC
:106F4000EC1030E0021713076CF49701225031095E
:106F5000D9012D913C91275031092730310508F492
:106F60007FC0C801019795958795918780870C9779
:106F70001CF41186108693C04483558366837783FF
:106F800084E090E00DC044835583668377838BE073
:106F900090E006C044835583668377838CE090E05D
:106FA000918380831EC58091F3109091F4108254D8
:106FB00091098E9708F099CF20E030E0C12CD12CB8
:106FC0007601A9014B505F4EDA014D915C91495019
:106FD00051094930510598F088CF8091F510909172
:106FE000F6100997099708F07BCF118610868FEF6E
:106FF0009FEFDC0184839583A683B783C2C5B90163
:1070000069507F4EDB014D915C91475151094231EE
:107010005105C0F4D701C601880F991FAA1FBB1FD5
:107020006C017D016894C0F82C5F3F4F203831051A
:1070300041F620E230E031872087C482D582E682A3
:10704000F7829FC5DB014D915C9146505109473055
:10705000510508F04ACFCC0CDD1CEE1CFF1CE4CF20
:10706000D7012D913C91235131092F30310550F436
:10707000440F551F661F771F41600296B4E0EB0E68
:10708000F11C5ACFD7012D913C912A50310929305A
:10709000310528F4440F551F661F771FEECF8091EE
:1070A000EC108A3108F460C08091EF109091F010DC
:1070B0008032934008F425CF8091F1109091F21026
:1070C000C697869708F050C08091F3109091F41005
:1070D000C697869708F048C0B7EFEB2EB0E1FB2EBD
:1070E00083E090E040E050E0BA018C010F5F1F4F59
:1070F0002091EC1030E00217130764F4970122503E
:107100003109D9012D913C912C5031092B30310599
:1071100060F0C801019795958795918780870C97B6
:107120000CF031CF118610861FC0D7012D913C91F4
:10713000255231092B31310550F4440F551F661F7C
:10714000771F41600296B4E0EB0EF11CCECFD70161
:107150002D913C912C5031092A30310528F4440FEF
:10716000551F661F771FEECF8091EC10823208F416
:1071700052C08091F1109091F2100697079708F095
:107180004AC045EFC42E40E1D42E82E090E040E0BA
:1071900050E0BA018C010F5F1F4F2091EC1030E0DE
:1071A00002171307F4F4D6011297ED90FC90119793
:1071B0009D01BEE1EB1AF108A7E1EA16F104E0F443
:1071C000440F551F661F771F4160D6012D913C91DA
:1071D000B4E0CB0ED11C2350310925303105C8F065
:1071E000C8010197959587959187808740970CF006
:1071F000D1CE118610860FC0D9012D913C912C5013
:1072000031092B30310538F4440F551F661F771FA5
:10721000DCCF0296BFCF7F011C821B8281E090E011
:107220009A8389838091EC108D3070F41C821B82CC
:1072300081E090E09A838983F7018485958518160B
:1072400019060CF474C0D1C029E733E0AE014D5FDC
:107250005F4FBE016F5F7F4FC7010E94468F892B32
:1072600029F729E733E0AE014D5F5F4FBE016F5F45
:107270007F4FC7010E94468F0197C1F629E733E08F
:10728000AE014D5F5F4FBE016F5F7F4FC7010E9430
:10729000468F892B59F6812C912C540100E010E087
:1072A0008091EC1090E029813A812817390794F5F4
:1072B00029E733E0AE014D5F5F4FBE016F5F7F4F47
:1072C000C7010E94468F6C0129E733E0AE014D5F94
:1072D0005F4FBE016F5F7F4FC7010E94468FF1E095
:1072E000CF16D10451F4892B09F0A0CF880C991C3A
:1072F000AA1CBB1C689480F80AC0CD2809F096CF60
:10730000019709F093CF880C991CAA1CBB1C0F5F36
:107310001F4FC6CFD70119961C930E931897F701EC
:1073200084829582A682B78281E090E039CE028481
:10733000F385E02D82E090E09A83898382819381B6
:1073400089974E9708F051C083E090E09A83898333
:10735000848195810B970A9708F047C02CEB31E0A8
:10736000AE014D5F5F4FBE016F5F7F4FC7010E944F
:10737000468F892BD1F52CEB31E0AE014D5F5F4F8D
:10738000BE016F5F7F4FC7010E94468F019769F56D
:10739000412C512C320100E010E0F70124853585A5
:1073A00089819A81821793070CF02FC12CEB31E071
:1073B000AE014D5F5F4FBE016F5F7F4FC7010E94FF
:1073C000468F5C010330110509F0E5C02CEB31E07C
:1073D000AE014D5F5F4FBE016F5F7F4FC7010E94DF
:1073E000468FA816B90609F4D6C0D7011A96ED91B2
:1073F000FC911B9782819381C6978697E0F48481E4
:1074000095814B974597B8F4DF0116966F0126ECEE
:10741000C20ED11C20E030E040E050E060E070E0BF
:1074200080E090E00D911C911197095011090830EE
:10743000110508F4F4C08091EC10893370F1828159
:107440009381895791098335910508F41BC125C0A3
:10745000D90112966D917C91139766517109613132
:10746000710508F037C1D501C401880F991FAA1F03
:10747000BB1F4C015D01689480F84E5F5F4F2C5F2D
:107480003F4F4B33510509F40CC1D9016D917C91EB
:107490006A50710969307105D8F28091EC1082321E
:1074A00031F4828193810A97099708F423C182817C
:1074B00093818957910983359105D0F48091EC101F
:1074C0008132B0F084819581CA97899788F49F01B1
:1074D0002A5F3F4F812C912C540143E050E0D901A9
:1074E0006D917C916A5071096930710508F41EC173
:1074F000828193818C549109C59778F48091EC1026
:10750000843031F4848195818097479708F46CC169
:107510008091EC10843408F04EC18091EC108634D8
:1075200060F1828193810C970B9708F4A9C125C063
:10753000D90112966D917C9113976E517109673143
:10754000710508F0D1C1D501C401880F991FAA1F88
:10755000BB1F4C015D01689480F84E5F5F4F2C5F4C
:107560003F4F4534510509F4A6C1D9016D917C9175
:107570006C5071096B307105D8F28091EC10883530
:1075800008F4E4C182819381855891098B35910576
:1075900008F4BAC1DBC12CEB31E0AE014D5F5F4FA7
:1075A000BE016F5F7F4FC7010E94468F6C010330A1
:1075B000110579F42CEB31E0AE014D5F5F4FBE0158
:1075C0006F5F7F4FC7010E94468FC816D90609F02A
:1075D0000CCFA114B10459F4CA94CD2809F005CFF9
:1075E000440C551C661C771C689440F80BC0AA9488
:1075F000AB2809F0FACECD2809F0F7CE440C551C83
:10760000661C771C0F5F1F4FC8CE11870087F701DC
:10761000448255826682778282E090E0C1CC1296E5
:107620000D911C911397015111090D301105E0F4D2
:1076300001E00E9487A721601496AC15BD0509F0F2
:10764000F1CEF701248335834683578300E20E94FD
:10765000A2A72283338385E090E09183808380E337
:1076600090E091878087BDC112960D911C91139770
:10767000045011090530110508F0DDCE01E00E942B
:1076800087A7DACF84819581CA97899708F005CFBB
:107690009F012A5F3F4F812C912C540143E050E021
:1076A000F4CE9F012A583F4FD9012D913C912A5089
:1076B00031092930310508F0F0CE2CE130E0F70136
:1076C00031872087D70184829582A682B7828AE09B
:1076D00090E085C1D90112966D917C911397665007
:1076E00071096730710508F0D8CE880C991CAA1C66
:1076F000BB1CC3CE2091EC10CF01820F911D820FD5
:10770000911DDC0112978D919C910A97099708F0C1
:10771000CECEF701118610868FEF9FEFDC018483B8
:107720009583A683B78386E090E03ACCD901129680
:107730006D917C911397665171096131710558F50E
:10774000D501C401880F991FAA1FBB1F4C015D0101
:10775000689480F84E5F5F4F2C5F3F4F4332510576
:1077600009F0BDCE9F012A5B3F4FD9012D913C917D
:107770002A5031092930310508F0BACE20E130E035
:10778000F70131872087D70184829582A682B7824C
:1077900086E090E024C1D90112966D917C911397F7
:1077A000665071096730710508F0A2CE880C991CEB
:1077B000AA1CBB1CCFCF8481958189549109C397A2
:1077C00008F0ABCE9F012A5F3F4FAF014A575F4F92
:1077D000812C912C5401D9016D917C9169507109D2
:1077E00069307105B8F099CE86819781099709971C
:1077F00008F08ECED70119961C921E9218978FEF23
:107800009FEFDC01F70184839583A683B78387E02C
:1078100090E0C6CBD90112966D917C911397665179
:10782000710961317105E0F4D501C401880F991F18
:10783000AA1FBB1F4C015D01689480F82C5F3F4F6D
:107840002417350741F620E230E0F7013187208721
:10785000D70184829582A682B78287E090E0BFC07C
:10786000D90112966D917C9113976650710967301A
:10787000710508F052CE880C991CAA1CBB1CDECFE7
:10788000848195810997099708F077CE8681978141
:107890008C974F9708F071CE8085918589974D9789
:1078A00008F06BCE9F01265F3F4F812C912C540135
:1078B00045E050E05ACE9F0126573F4FD9012D9108
:1078C0003C912C5031092B30310508F056CE20E286
:1078D00030E0F70131872087D70184829582A68224
:1078E000B78288E090E07BC0D90112966D917C91BF
:1078F0001397695071096930710508F03ECE880C04
:10790000991CAA1CBB1C29CE8481958182549109A3
:107910008E97E0F48F01045C1F4F8DE190E040E012
:1079200050E02091EC1030E0245031098217930789
:107930000CF063C0980122503109D9012D913C917E
:10794000295031092830310508F46EC08091EC10BF
:10795000803209F07EC0828193810697069708F0F5
:1079600078C0848195810997099708F072C09F01BA
:107970002A5F3F4FAF01425C5F4F812C912C540135
:10798000D9016D917C91665071096630710508F0DE
:1079900060C0D90112966D917C911397695171095C
:1079A0006331710508F0D5C0D501C401880F991F56
:1079B000AA1FBB1F4C015D01689480F82C5F3F4FEC
:1079C00024173507E9F62EE030E0F70131872087EC
:1079D000D70184829582A682B7828FE090E08D9352
:1079E0009C9381E090E0D0C0D8012D913C9128512A
:1079F00031092231310550F1CB01019795958795D9
:107A0000D70119969C938E9318978A970CF49ECF62
:107A1000052E000C660B770BF701448355836683B4
:107A2000778389E090E0BCCABC016F5F7F4FD801CB
:107A30002D913C912750310927303105A8F6440F8C
:107A4000551F416002960C5F1F4F6BCF440F551FAF
:107A5000F9CFD7011C962D903C901D97B6E02B16C0
:107A600031040CF486C08F010E5F1F4F75EC872E1A
:107A70007DE9972E7CE1A72E71E8B72EE3E0CE2EAC
:107A8000D12CF801648175816080718080E090E084
:107A90000E949FA26D837E838F839887B30180E0CD
:107AA00090E00E949FA22B013C012DEC3CEC4CE4A9
:107AB0005FE30E9400A39B01AC016D817E818F81F9
:107AC00098850E949BA287FD19C02DEC3CEC4CE4EC
:107AD0005FE36D817E818F8198850E9400A39B0169
:107AE000AC01C301B2010E949BA2E82F880FFF0BDB
:107AF000EE27FF0FEE1FFF27319602C0E0E0F0E017
:107B0000A501940163E971E080E091E00E9449A73A
:107B10004F01FF0FAA08BB0886269726A826B9267C
:107B2000FFEFCF1ADF0A0E5F1F4F2C143D0409F040
:107B3000A8CFD70114968D929D92AD92BC921797C3
:107B400080E290E019969C938E9318978FEF9FEFA9
:107B500046CFD90112966D917C91139769507109A6
:107B60006930710508F075CF880C991CAA1CBB1CE4
:107B700025CF82E08093E9101092EC1080E090E035
:107B800003C083E090E00CCA28960FB6F894DEBFDD
:107B90000FBECDBFDF91CF911F910F91FF90EF905E
:107BA000DF90CF90BF90AF909F908F907F906F901D
:107BB0005F904F903F902F9008954F925F926F92F9
:107BC0007F929F92AF92BF92CF92DF92EF92FF92FD
:107BD0000F931F93CF93DF93CDB7DEB7A9970FB65F
:107BE000F894DEBF0FBECDBF982E882351F0809150
:107BF0001F0D882331F06AE37CE080E490E10E946D
:107C00006C7B0E943D5E60E08DE20E94146060E14A
:107C10008DE20E94146068E08DE20E941460409042
:107C20003413509035136090361370903713498E8B
:107C30005A8E6B8E7C8EC0903813D0903913E090A2
:107C40003A13F0903B13CD8EDE8EEF8EF8A280912A
:107C50003C1390913D13A0913E13B0913F138EA31E
:107C60009FA3A8A7B9A789A39AA3ABA3BCA3992054
:107C7000D1F180911F0D8823B1F166E07BE0CE0148
:107C800001960E94CC4ECE0101960E942960CE0141
:107C900001960E94984E8E01075E1F4F5E0195E28D
:107CA000A90EB11CD8016D917D918D919D918D0191
:107CB00046E050E00E948A7C66EE7BE080E490E142
:107CC0000E941350A016B10669F76AE37CE0CE016A
:107CD00001960E94DC4ECE0101960E942960CE01E1
:107CE00001960E94984E23E938E144E85FE3C3011E
:107CF000B2010E9400A32B013C016D877E878F8714
:107D0000988B22E430E645E85FE3C701B6010E94A4
:107D100000A36B017C01698B7A8B8B8B9C8B25E894
:107D20003BEE41E95FE36EA17FA188A599A50E9482
:107D300000A36D8B7E8B8F8B988F40923413509263
:107D400035136092361370923713C0923813D09265
:107D50003913E0923A13F0923B1360933C13709303
:107D60003D1380933E1390933F13992009F4A1C0D3
:107D700080911F0D882309F49CC069EF7AE0CE0141
:107D800001960E94CC4ECE0101960E942960CE0140
:107D900001960E94984E8E01035F1F4F6E01B9E15C
:107DA000CB0ED11C7801F801619171918191919173
:107DB0008F0142E050E00E948A7C66EE7BE080E426
:107DC00090E10E9413500C151D0569F76AE37CE0F1
:107DD000CE0101960E94DC4ECE0101960E942960E0
:107DE000CE0101960E94984E40E453E166E070E0B7
:107DF00082E30E94AD5FA0904013B0904113C09009
:107E00004213D090431300914413109145136CEE2C
:107E10007AE080E490E10E94484F4AE050E0B501EA
:107E200080E490E10E94C94F66EE7BE080E490E13F
:107E30000E9413504AE050E0B60180E490E10E94B5
:107E4000C94F66EE7BE080E490E10E9413504AE067
:107E500050E0B80180E490E10E94C94F6AE37CE001
:107E600080E490E10E946C7BCE010196E1D563EE47
:107E70007AE080E490E10E94484F8E010F5F1F4F2F
:107E8000D8016D917D918D919D918D014AE050E0D9
:107E90000E948A7C66EE7BE080E490E10E941350B1
:107EA0000E151F0569F76AE37CE080E490E10E940B
:107EB0006C7B61E08DE10E9414609920B1F08091AB
:107EC0001F0D882391F06FEC7AE080E490E10E942E
:107ED000484FAE014B5D5F4F61E070E08DE10E9465
:107EE000AD5F8DA190E00E94E75F62E08EE10E94AD
:107EF000146063E08FE10E94146064E080E20E94FD
:107F00001460992009F450C080911F0D882309F452
:107F10004BC063EB7AE080E490E10E94484FAE01F1
:107F20004B5D5F4F61E070E08EE10E94AD5FCDA0E0
:107F3000D12CAE014B5D5F4F61E070E08FE10E949C
:107F4000AD5FEDA0F12CAE014B5D5F4F61E070E0E5
:107F500080E20E94AD5F0DA110E04AE050E0B60162
:107F600080E490E10E94C94F66EE7BE080E490E1FE
:107F70000E9413504AE050E0B70180E490E10E9473
:107F8000C94F66EE7BE080E490E10E9413504AE026
:107F900050E0B80180E490E10E94C94F6AE37CE0C0
:107FA00080E490E10E946C7B65E081E20E941460B5
:107FB0009920B1F080911F0D882391F060EA7AE05A
:107FC00080E490E10E94484FAE014B5D5F4F61E05D
:107FD00070E081E20E94AD5F8DA190E00E94E75FBA
:107FE00066E082E20E9414609920B1F080911F0D3A
:107FF000882391F068E87AE080E490E10E94484F9D
:10800000AE014B5D5F4F61E070E082E20E94AD5FC8
:108010008DA190E00E94E75F67E083E20E94146018
:108020009920B1F080911F0D882391F062E77AE0EA
:1080300080E490E10E94484FAE014B5D5F4F61E0EC
:1080400070E083E20E94AD5F8DA190E00E94E75F47
:1080500068E084E20E9414609920B1F080911F0DC5
:10806000882391F06AE57AE080E490E10E94484F2D
:10807000AE014B5D5F4F61E070E084E20E94AD5F56
:108080008DA190E00E94E75F69E085E20E941460A4
:108090009920B1F080911F0D882391F060E47AE07F
:1080A00080E490E10E94484FAE014B5D5F4F61E07C
:1080B00070E085E20E94AD5F8DA190E00E94E75FD5
:1080C0006AE086E20E9414609920B1F080911F0D51
:1080D000882391F06AE27AE080E490E10E94484FC0
:1080E000AE014B5D5F4F61E070E086E20E94AD5FE4
:1080F0008DA190E00E94E75F6BE088E20E9414602F
:108100009920B1F080911F0D882391F061E17AE010
:1081100080E490E10E94484FAE014B5D5F4F61E00B
:1081200070E088E20E94AD5F8DA190E00E94E75F61
:108130006CE089E20E941460992009F479C0809172
:108140001F0D882309F474C069EF79E080E490E1A1
:108150000E94484FAE014B5D5F4F61E070E089E2E5
:108160000E94AD5F8DA190E00E94E75F62EE79E032
:1081700080E490E10E94484F66E070E087E20E9450
:10818000FA5F90E00E94E75F6BEC79E080E490E1B9
:108190000E94484F65E070E087E20E94FA5F90E03D
:1081A0000E94E75F64EB79E080E490E10E94484F31
:1081B00064E070E087E20E94FA5F90E00E94E75F6F
:1081C0006BE979E080E490E10E94484F62E070E062
:1081D00087E20E94FA5F90E00E94E75F62E879E040
:1081E00080E490E10E94484F61E070E087E20E94E5
:1081F000FA5F90E00E94E75F69E679E080E490E151
:108200000E94484F60E070E087E20E94FA5F90E0D1
:108210000E94E75F68E579E080E490E10E94484FC2
:1082200063E070E087E20E94FA5F90E00E94E75FFF
:1082300041E067E070E087E29FD341E063E070E0F7
:1082400087E29AD341E063E070E08AE295D3992017
:1082500091F080911F0D882371F06FE379E080E445
:1082600090E10E94484F63E070E08AE20E94FA5F6A
:1082700090E00E94E75F40E063E070E08AE27CD338
:10828000992091F080911F0D882371F065E279E0CB
:1082900080E490E10E94484F63E070E08AE20E942F
:1082A000FA5F90E00E94E75F41E062E070E08AE2FE
:1082B00063D3992091F080911F0D882371F069E0BC
:1082C00079E080E490E10E94484F62E070E08AE249
:1082D0000E94FA5F90E00E94E75F40E062E070E099
:1082E0008AE24AD3992091F080911F0D882371F082
:1082F0006CEE78E080E490E10E94484F62E070E02C
:108300008AE20E94FA5F90E00E94E75F41E061E04C
:1083100070E08AE231D3992091F080911F0D88237B
:1083200071F060ED78E080E490E10E94484F61E0F8
:1083300070E08AE20E94FA5F90E00E94E75F40E00E
:1083400061E070E08AE218D3992091F080911F0DCE
:10835000882371F063EB78E080E490E10E94484F5D
:1083600061E070E08AE20E94FA5F90E00E94E75FBD
:1083700041E060E070E08AE2FFD2992091F08091C4
:108380001F0D882371F067E978E080E490E10E9496
:10839000484F60E070E08AE20E94FA5F90E00E943D
:1083A000E75F40E060E070E08AE2E6D2992091F079
:1083B00080911F0D882371F06AE778E080E490E1F6
:1083C0000E94484F60E070E08AE20E94FA5F90E00D
:1083D0000E94E75F41E066E070E087E2CDD241E0D5
:1083E00065E070E087E2C8D241E064E070E087E2D7
:1083F000C3D240E062E070E087E2BED240E061E0DC
:1084000070E087E2B9D240E060E070E087E2B4D289
:10841000992009F475C080911F0D882309F470C05C
:1084200062E678E080E490E10E94484F66E070E008
:108430008BE20E94FA5F90E00E94E75F64E478E0DC
:1084400080E490E10E94484F65E070E08BE20E947A
:10845000FA5F90E00E94E75F66E278E080E490E1F6
:108460000E94484F64E070E08BE20E94FA5F90E067
:108470000E94E75F6DE078E080E490E10E94484F61
:1084800062E070E08BE20E94FA5F90E00E94E75F9A
:1084900064EF77E080E490E10E94484F61E070E093
:1084A0008BE20E94FA5F90E00E94E75F6BED77E05D
:1084B00080E490E10E94484F60E070E08BE20E940F
:1084C000FA5F90E00E94E75F68EC77E080E490E17B
:1084D0000E94484F63E070E08BE20E94FA5F90E0F8
:1084E0000E94E75F63EB77E080E490E10E94484FF1
:1084F00064E070E08CE20E94FA5F90E00E94E75F27
:1085000040E064E070E08CE237D2AE014B5D5F4F3B
:1085100061E070E08CE20E94AD5F6DA1607F6660FB
:108520008CE20E941460992009F45DC080911F0DB7
:10853000882309F458C06FE977E080E490E10E9455
:10854000484FAE014B5D5F4F61E070E08CE20E94EE
:10855000AD5F6DA16F7070E066507109072E000C61
:10856000880B990B0E94A1A29B01AC0160E070E016
:1085700080E090E40E949FA620E030E048EC50E4C8
:108580000E9400A346D268E877E080E490E10E9470
:10859000484FAE014B5D5F4F61E070E080E30E94A9
:1085A000AD5F6DA14AE050E080E490E117D260E752
:1085B00077E080E490E10E94484F61E070E080E362
:1085C0000E94FA5F90E00E94E75F67E577E080E451
:1085D00090E10E94484F61E070E08FE20E94FA5FF4
:1085E00090E00E94E75F41E061E070E08FE2C4D17B
:1085F000992091F080911F0D882371F06FE377E04F
:1086000080E490E10E94484F61E070E08EE20E94B9
:10861000FA5F90E00E94E75F41E061E070E08EE287
:10862000ABD140E067E070E081E3A6D1992009F486
:1086300055C080911F0D882309F450C06CE277E08B
:1086400080E490E10E94484F67E070E081E30E947F
:10865000FA5F90E00E94E75F6EE17BE080E490E1EA
:108660000E941350AE014B5D5F4F61E070E080E00F
:108670000E94AD5F8DA10E94EA876AE37CE080E4FE
:1086800090E10E946C7B0DE110E06AE57AE080E405
:1086900090E10E94135040E150E0B80180E490E185
:1086A0000E94C94F65EB78E080E490E10E9413508E
:1086B000AE014B5D5F4F61E070E0802F0E94AD5FC7
:1086C0008DA10E94EA876AE37CE080E490E10E9449
:1086D0006C7B0F5F1F4F0A331105B9F6A9960FB6D1
:1086E000F894DEBF0FBECDBFDF91CF911F910F91E8
:1086F000FF90EF90DF90CF90BF90AF909F907F90D2
:108700006F905F904F90089596E0899FD00111245B
:10871000AA5BBC4E90967C936E935F9791E0919686
:108720009C9391979091B213E091B313F091B4138D
:10873000992339F0309751F0811108C0809162136C
:1087400004C0309719F05C968C9119940895BF92EB
:10875000CF92DF92EF92FF920F931F93CF93DF930D
:10876000EC016B018D85811105C0CE010E945C86F4
:10877000811105C01B861D861C8680E060C040E01C
:1087800060EFCE010E94785101E0E12CB12C11E0A4
:10879000CE010E940986F82ECE010E94098691E042
:1087A000F91203C08130B1F434C02E2D30E0F8123C
:1087B0001BC08B85181738F4FE01E20FF31F83816D
:1087C000802341F402C0811729F0F12C193058F4AC
:1087D0001C8709C0FE01EE0DF11D8381802B838370
:1087E000FF24F39409C0B12EFE01E20FF31F938121
:1087F000802F8095892383836F2DCE010E942D8643
:108800001F5F000F11F4E39401E087E08E1508F07C
:10881000BFCF113408F4AECFBB86B11002C081E0E7
:108820008D878B81882309F4A5CFDE011396F6018D
:108830002B968D918193CA17DB07D9F781E0DF91E1
:10884000CF911F910F91FF90EF90DF90CF90BF904D
:108850000895DF92EF92FF920F931F93CF93DF93D0
:108860007C018B01D42EDC011696ED91FC911797BB
:10887000138615861486DF011B9633961E92EA171F
:10888000FB07E1F7C0E0B801F701868197815FDF60
:10889000D82F882371F0DC1209C067E0C8010E945C
:1088A0006051D80117969C91891721F0CF5FDC1693
:1088B00050F7D0E08D2FDF91CF911F910F91FF9056
:1088C000EF90DF9008950F931F93CF93DF93C82FFE
:1088D000D62F86E0C89FF0011124EA5BFC4E11A25E
:1088E000878D90A181309105D1F040F082309105C3
:1088F000A1F10397E1F560E070E033C06623B9F1C0
:1089000061E070E08C2F00DF0E94BE8D60939E13AB
:1089100070939F138093A0139093A11328C00E947B
:10892000BE8D00919E1310919F132091A013309142
:10893000A113AB01BC01401B510B620B730B809167
:10894000B0139091B113A0E0B0E084179507A6078B
:10895000B70718F462E070E004C0D11108C063E00A
:1089600070E08C2FDF91CF911F910F91CDCEDF91D1
:10897000CF911F910F910895FF920F931F93CF9363
:10898000DF931F92CDB7DEB7182F062FF42EAE015E
:108990004F5F5F4F61E070E00E94AD5F4981FF2053
:1089A00049F021E030E001C0220F0A95EAF7242BBC
:1089B000298309C081E090E001C0880F0A95EAF799
:1089C0008095842389836981812F0E9414600F9090
:1089D000DF91CF911F910F91FF9008950F931F93F7
:1089E000CF93DF93EC019A01452B11F4CAD506C051
:1089F000462F50E060E070E00E94814F8C01CE0174
:108A00000E94817A800F911FDF91CF911F910F916A
:108A10000895CF93DF9342E00E94B07BEC0180E4A5
:108A200090E10E94817A8C0F9D1FDF91CF91089574
:108A30008F929F92AF92BF92CF92DF92EF92FF926E
:108A40000F931F93CF93DF9300D000D0CDB7DEB745
:108A50005C0140E453E166E070E082E30E94AD5FB8
:108A600080914013909141139A838983809142139E
:108A7000909143139C838B83809144139091451371
:108A80009E838D83CE0101966C0184E3E82E83E101
:108A9000F82E8501F601619171916F01F7018190C6
:108AA0009190A190B1907F01072E000C880B990B3B
:108AB0000E94A1A2A50194010E9400A3F801619364
:108AC0007193819391938F01F0E4EF16F3E1FF0628
:108AD00009F726960FB6F894DEBF0FBECDBFDF9123
:108AE000CF911F910F91FF90EF90DF90CF90BF90AB
:108AF000AF909F908F900895CF93DF93C82F809170
:108B0000B8130E94F97A6C2F8DED90E10E94D88500
:108B100080E00E94967A63E08091B8130E949B5E89
:108B20008DED90E10E949085EC018DED90E10E9429
:108B3000908520E030E0382FC9018C2B9D2BDF91F0
:108B4000CF9108950F931F93CF93DF93CDB7DEB7E7
:108B500061970FB6F894DEBF0FBECDBF8C01462FD4
:108B6000BE01665F7F4F75DE811105C060E070E079
:108B70008EEF92EC4CC0AE014F5F5F4FBE01665F5F
:108B80007F4FC8010E94C951882361F12A8130E0DA
:108B9000C901982F8827990F990F990F698128E0AB
:108BA000629FB00111249C01262B372B8A858031CE
:108BB000E1F4688570E08F81AB01481B5109CA015F
:108BC0009695982F8827979587950E946CA7605156
:108BD0007109207F53E0220F331F5A95E1F7620F8E
:108BE000731F04C060E874EE01C0B901613854EE2F
:108BF00075070CF4BBCF072E000C880B990B0E9455
:108C0000A1A220E030E040E05CE30E9400A3619676
:108C10000FB6F894DEBF0FBECDBFDF91CF911F918D
:108C20000F9108959F92AF92BF92CF92DF92EF92F1
:108C3000FF920F931F93CF93DF93CDB7DEB761976A
:108C40000FB6F894DEBF0FBECDBF8C018CE0F801EB
:108C50008183C12CD12C2FE5E22E3FE7B32E4FE1CB
:108C6000A42E5FE3952EF801848190E0C816D90602
:108C70000CF0A1C04C2DBE01665F7F4FC801E9DD3D
:108C8000F8018181893038F0F82EFCE0F81728F4DB
:108C90009CE0F92E02C089E0F82E8A85803139F0F7
:108CA000BE01665F7F4FC8010E94245201C08CE064
:108CB000F81609F47CC0AE014F5F5F4FBE01665FDE
:108CC0007F4FC8010E94C951882309F470C08A856A
:108CD000803109F46CC08BE0F81651F0ECE0FE1620
:108CE00029F0FAE0FF1206C09D8205C0BD8203C0D4
:108CF000ED8201C0AD82F801868197810E945C8679
:108D0000BE01665F7F4FF801868197810E94AC515A
:108D100040E06EE4F801868197810E94785140E03E
:108D20006B81F801868197810E94785140E06C81C7
:108D3000F801868197810E9478518A85803139F0C7
:108D400040E06D81F801868197810E947851F80199
:108D5000868197810E945C86BE01665F7F4FF80125
:108D6000868197810E94AC51F801408168E4868138
:108D700097810E94785164E170E080E090E00E9469
:108D8000868DF8018081882331F06AE070E080E010
:108D900090E00E94868DF801868197810E945C8612
:108DA000F80181818F1508F48F2DF8018183FFEF81
:108DB000CF1ADF0A58CF61960FB6F894DEBF0FBE08
:108DC000CDBFDF91CF911F910F91FF90EF90DF907A
:108DD000CF90BF90AF909F9008958F929F92AF9247
:108DE000BF92CF92DF92EF92FF920F931F93CF9398
:108DF000DF93EC018E819F810E945C8640E06CECE9
:108E00008E819F810E947851488164E48E819F8188
:108E10000E9478518A81882309F442C0E981E9508F
:108E2000E33040F4F0E0EE0FFF1FE951FB4F00810B
:108E3000118102C00EEE12E08B818823F9F0888147
:108E400081111CC00E94BE8D4B015C016801110F95
:108E5000EE08FF088E819F810E940986813001F112
:108E60000E94BE8DDC01CB018C199D09AE09BF09A2
:108E700088159905AA05BB0568F312C0B801110F42
:108E8000880B990BDF91CF911F910F91FF90EF907D
:108E9000DF90CF90BF90AF909F908F900C94868D75
:108EA000DF91CF911F910F91FF90EF90DF90CF90C6
:108EB000BF90AF909F908F900895EF92FF920F9385
:108EC0001F93CF93DF93CDB7DEB728970FB6F894F3
:108ED000DEBF0FBECDBF8C01DC011696ED91FC917B
:108EE0001797138615861486DF011B9633961E92FC
:108EF000EA17FB07E1F7F80114821582EE24E394E8
:108F0000BE016F5F7F4FD80116968D919C91179788
:108F10001EDC882309F475C067E0CE0101960E942B
:108F2000605198858913ECCFF8018081811124C0AC
:108F3000868197810E945C86BE016F5F7F4FD8015A
:108F400016968D919C9117970E94AC5140E064EB6E
:108F5000F801868197810E947851D80116968D91EB
:108F60009C9117970E940986F82EF80186819781B7
:108F70000E945C86FF20B1F1D8011196FC90898196
:108F80008031D9F1BE016F5F7F4FC8010E9424522A
:108F90008F1518F4F80181810BC08981803111F49B
:108FA0008CE006C0BE016F5F7F4FC8010E94245253
:108FB000D80111968C93119714968C9114978F5F0A
:108FC00014968C938981883281F030F4803169F075
:108FD000823209F095CF09C08B3339F0823409F021
:108FE0008FCF03C0F801E082C7CFD80115968C91CE
:108FF00015978F5F15968C9383CFBCE0BF1550F209
:10900000CFCF28960FB6F894DEBF0FBECDBFDF914D
:10901000CF911F910F91FF90EF9008956F927F92E3
:109020008F929F92AF92BF92CF92DF92EF92FF9278
:109030000F931F93CF93DF9381E08093B2130E942D
:10904000BE8D0091A2131091A3132091A41330910F
:10905000A513AB01BC01401B510B620B730B80913C
:10906000AE139091AF13A0E0B0E084179507A60768
:10907000B70708F0E6C0C0E08091AC13C81730F025
:10908000712C812C912C5401839440C0E091A81341
:10909000F091A913EC0FF11D62E080810E94008D18
:1090A000CF5FEACFC62DD0E0E091A813F091A913CD
:1090B000EC0FFD1F80810E94AA8C2496CC0FDD1F2F
:1090C000CA5BDC4E892B09F04BC0888199818C29C1
:1090D0009D299983888363948091AC13681610F35B
:1090E000E091AA13F091AB13E00FF11F61E08081D2
:1090F0000E94D28C8091AA139091AB13FC01E00FD7
:10910000F11F60E080810E94008D73948091AD1307
:10911000781658F5072D10E0E091AA13F091AB13E3
:10912000E00FF11F61E080810E94008DE091AA13A1
:10913000F091AB13E00FF11F60E080810E94D28CB0
:10914000D501C401072C04C0880F991FAA1FBB1F9B
:109150000A94D2F76C017C01E094F094612CBCCFAE
:10916000888199818E219F21B4CF26E4E22E23E1CC
:10917000F22EF7018FEF9FEF278D30A1232B21F4E3
:10918000148E968F858F11A2369623E1E238F2076E
:1091900099F7C0E096E0D92E8091AC13C81758F526
:1091A000D0E00C2F10E0000F111F025B1C4E20912D
:1091B000AD13D217F0F4F801408151810D2E02C099
:1091C000569547950A94E2F7642F6170C29F90010B
:1091D00011242D0F311DE6E4F3E180E0A58DB68D5D
:1091E0002A173B0709F44DC08F5F36968A30B1F7D6
:1091F0002CC0CF5FD1CFC0E0F70181A18111C1E0C8
:10920000F6E0EF0EF11C22E8E21623E1F206A1F7E8
:109210000E94BE8D6093A2137093A3138093A41336
:109220009093A513CC2369F080916713882349F0AC
:109230008091651390916613019719F480916213E0
:1092400029C01092B21380E025C040FF1BC0E6E4A5
:10925000F3E180E090E0448D411116C0E091A61347
:10926000F091A713E20FF31F4081D89EF001D99E21
:10927000F00D1124EA5BFC4E448F368F258F10A22F
:10928000178E21DBDF5F93CF019636968A309105EA
:1092900011F7F8CFDF91CF911F910F91FF90EF90D1
:1092A000DF90CF90BF90AF909F908F907F906F9006
:1092B0000895CF93DF93FC0124813581232B71F036
:1092C000FB01DC01CD91DC9160817181CE010E94B6
:1092D00012AA009719F08C1B9D0B02C08FEF9FEF15
:1092E000DF91CF9108950F931F93CF93DF93FC01EC
:1092F000C481D581209719F4FB01108211C041501F
:1093000051094C175D0708F4EA018B01FC016081EB
:109310007181AE01C8010E9403AAC00FD11F18823B
:10932000DF91CF911F910F910895AF92BF92CF928D
:10933000DF92EF92FF920F931F93CF93DF93FC0185
:1093400024813581FB01448155818901041B150B62
:109350004115510551F12115310539F12417350712
:1093600020F10217130718F08901015011097B0140
:10937000FC01A080B180C501DFEFCFEF6501C00E19
:10938000D11EC816D906A0F0F701608171810E9434
:1093900012AA009769F09C012A193B0902171307CA
:1093A00010F0D22FC32F0196ECCF8FEF9FEF02C0AA
:1093B0008D2F9C2FDF91CF911F910F91FF90EF90F8
:1093C000DF90CF90BF90AF900895CF93DF931F921F
:1093D0001F92CDB7DEB769831A8241E050E0BE012B
:1093E0006F5F7F4FB2D30F900F90DF91CF910895B1
:1093F000FB0144815581FC01248135812417350707
:1094000078F080819181009759F0FB016081718132
:109410006115710529F00E94F5A921E0892B09F059
:1094200020E0822F08950895CF92DF92EF92FF926D
:109430000F931F93CF93DF936C017A018B01C0E0F0
:10944000D0E0CE15DF0581F0D8016D918D01D601F8
:10945000ED91FC910190F081E02DC6011995892BC9
:1094600011F02196EECF7E01C701DF91CF911F91C0
:109470000F91FF90EF90DF90CF900895FC01538DF6
:10948000448D252F30E0842F90E0821B930B5417DE
:1094900010F0CF96089501970895FC01918D828D6B
:1094A000981761F0828DDF01A80FB11D5D968C9138
:1094B000928D9F5F9F73928F90E008958FEF9FEF43
:1094C0000895FC01918D828D981731F0828DE80FFF
:1094D000F11D858D90E008958FEF9FEF0895FC01B9
:1094E000918D228D892F90E0805C9F4F821B910986
:1094F0008F739927089589E69EE0F1DF21E0892B9B
:1095000009F420E0822F089586E09FE0E8DF21E063
:10951000892B09F420E0822F089583EA9FE0DFDFA2
:1095200021E0892B09F420E0822F089580E490E166
:10953000D6DF21E0892B09F420E0822F0895FC0179
:10954000848DDF01A80FB11DA35ABF4F2C91848DCC
:1095500090E001968F739927848FA689B7892C9301
:10956000A089B1898C91837080648C93938D848D54
:10957000981306C00288F389E02D80818F7D808357
:109580000895EF92FF920F931F93CF93DF93EC0117
:1095900081E0888F9B8D8C8D981305C0E889F989AF
:1095A000808185FD25C0F62E0B8D10E00F5F1F4FCB
:1095B0000F731127E02E8C8DE8120BC00FB607FC3D
:1095C000FACFE889F989808185FFF5CFCE01B7DF31
:1095D000F2CF8B8DFE01E80FF11DE35AFF4FF082B1
:1095E0009FB7F8940B8FEA89FB89808180620AC05B
:1095F0009FB7F894EE89FF896083E889F9898081B3
:109600008370806480839FBF81E090E0DF91CF9181
:109610001F910F91FF90EF900895CF93DF93EC018E
:10962000888D8823C1F0EA89FB89808185FD05C08A
:10963000A889B9898C9186FD0EC00FB607FCF5CFBD
:10964000808185FFF2CFA889B9898C9185FFEDCF04
:10965000CE0175DFE8CFDF91CF91089580E090E0F3
:10966000892B19F063DF811116C080E090E0892B0F
:1096700019F053DF811112C080E090E0892B19F0BE
:1096800043DF81110EC080E090E0892B79F033DF59
:1096900081110AC008950E940000E7CF0E940000D7
:1096A000EBCF0E940000EFCF0C94000008950E94C1
:1096B000BFA9CF93DF93EC0188819981009711F0C6
:1096C0000E9456A8198218821D821C821B821A824F
:1096D000DF91CF9108950F931F93CF93DF93EC0108
:1096E00088819981009729F02A813B8126173707C5
:1096F00088F48B016F5F7F4F0E94DFA8009761F0B5
:10970000998388831B830A832C813D81232B11F449
:10971000FC01108281E001C080E0DF91CF911F91B8
:109720000F910895EF92FF920F931F93CF93DF93C2
:10973000EC017B018A01BA01CEDF811103C0CE01A9
:10974000B8DF07C01D830C83B701888199810E940F
:10975000EEA9CE01DF91CF911F910F91FF90EF9075
:1097600008950F931F93CF93DF938C01EB0188E251
:10977000FB0111928A95E9F74BE050E065E27BE04E
:10978000CE010E9403AA1B8681E090E0A0E0B0E039
:109790008C879D87AE87BF87F80185899689A789C1
:1097A000B08D888B998BAA8BBB8B82E090E0A0E078
:1097B000B0E08C8B9D8BAE8BBF8B1CA21DA21EA21A
:1097C0001FA280E090E0A8E4B4E4888F998FAA8F6C
:1097D000BB8F80E090E0A8E4B4EC8C8F9D8FAE8FBF
:1097E000BF8F8DEC9CECACE4BEE388A399A3AAA345
:1097F000BBA3DF91CF911F910F9108954F925F927C
:109800006F927F928F929F92AF92BF92CF92DF9290
:10981000EF92FF920F931F93CF93DF938C01EB0195
:1098200084E2FB0111928A95E9F78EE10E94F97AB0
:1098300083E090E00E94F47A0E94F27A66E08EE182
:109840000E949B5E8091F90C90E02091FA0C821BA3
:10985000910986309105ECF38DED90E10E949085A1
:10986000882E8DED90E10E949085982E8DED90E1EF
:109870000E949085682E8DED90E10E949085782E53
:109880008DED90E10E949085482E8DED90E10E9433
:109890009085582EB82CA12CB5016929072E000CF3
:1098A000880B990B0E94A1A24B015C01F801658312
:1098B000768387839087D42CC12CB6016529072E27
:1098C000000C880B990B0E94A1A2F8016187728796
:1098D00083879487F62CE12CB7016729072E000CAB
:1098E000880B990B0E94A1A2F8016587768787876C
:1098F000908B118A128A138A148A84E290E0A0E085
:10990000B0E088839983AA83BB8385899689A789D8
:10991000B08D8C839D83AE83BF8382E090E0A0E016
:10992000B0E088879987AA87BB87188A198A1A8A1C
:109930001B8AC0907C04D0907D04E0907E04F0905F
:109940007F04A7019601C501B4010E94F1A420E0A3
:1099500030E048EC52E40E9400A36C8B7D8B8E8B30
:109960009F8BA7019601F801618572858385948597
:109970000E94F1A420E030E048EC52E40E9400A3F1
:10998000688F798F8A8F9B8F20917804309179042A
:1099900040917A0450917B04F8016585768587852E
:1099A00090890E94F1A420E030E048EC52E40E944B
:1099B00000A36C8F7D8F8E8F9F8F81E0DF91CF9181
:1099C0001F910F91FF90EF90DF90CF90BF90AF90DD
:1099D0009F908F907F906F905F904F900895862F0B
:1099E0000C94AA8C862F642F0C94D28C862F642F13
:1099F0000C94008DFC0180819181009711F00C94F2
:109A00002D9E60E070E0CB010895AF92BF92CF929F
:109A1000DF92EF92FF920F931F93CF93DF93DC01BE
:109A2000CD90DC901197C114D10409F443C0149671
:109A3000CD91DC9115972097E9F18C0176015701C2
:109A4000BFEFAB1ABB0AF7018081082E000C990BFF
:109A50000E946BA2892B11F07501F1CF2197CC0DDB
:109A6000DD1D8881082E000C990B0E946BA2892BAA
:109A700029F0CE15DF0510F02197F3CFAE014F5F2F
:109A80005F4F4E195F09D80115965C934E9314975A
:109A9000CE14DF0420F4B701C6010E94DCA9D8016E
:109AA000ED91FC91119714968D919C911597E80F6B
:109AB000F91F1082DF91CF911F910F91FF90EF90CE
:109AC000DF90CF90BF90AF900895FC012481358145
:109AD0006217730748F480819181009729F0FC0197
:109AE000E60FF71F8081089580E00895EF92FF92BE
:109AF0000F931F93CF93DF936115710511F480E0ED
:109B00001DC08B01EC01CB010E945A9E0097A9F069
:109B10002C813D817C01E20EF31EB701CE01DBDD1D
:109B2000882369F3288139818C819D81B801820F56
:109B3000931F0E94539EFD82EC8281E0DF91CF91C2
:109B40001F910F91FF90EF900895EF92FF920F9366
:109B50001F93CF93DF936115710511F480E01BC053
:109B600041155105B9F07B01EC018C819D818A0181
:109B7000080F191FB801CE01AEDD882379F32881C3
:109B800039818C819D81B701820F931F0E94EEA9BC
:109B90001D830C8381E0DF91CF911F910F91FF9086
:109BA000EF900895CF93DF93EC016115710559F0A3
:109BB000FB0101900020E9F73197AF01461B570BDD
:109BC000C4DF811102C0CE0174DDCE01DF91CF91DF
:109BD0000895CF93DF93EC01FB01448155816081AF
:109BE0007181B3DF811102C0CE0163DDCE01DF914F
:109BF000CF9108956115710549F0FB010190002096
:109C0000E9F73197AF01461B570B9FCF80E00895CE
:109C1000FB01448155816081718197CFEF92FF9262
:109C20000F931F93CF93DF93EC018B0161157105A7
:109C300049F0CB010E945A9E7C01BC01CE014BDD54
:109C4000811103C0CE0135DD07C0FD82EC82B80171
:109C5000888199810E94539ECE01DF91CF911F91FF
:109C60000F91FF90EF900895CF93DF93EC01611572
:109C7000710551F0FB0101900020E9F73197AF0128
:109C8000461B570B4FDD01C014DDCE01DF91CF9194
:109C90000895CF93DF93EC01FB018617970751F0EE
:109CA000608171816115710521F0448155813ADD32
:109CB00001C0FFDCCE01DF91CF9108950F931F9378
:109CC000CF93DF938C01EB01FC01808191810097A0
:109CD00039F06881798161157105A1F40E9456A857
:109CE00088819981F801918380838A819B81938304
:109CF00082838C819D8195838483198218821B8243
:109D00001A820FC0F801428153812C813D81421794
:109D1000530720F30E94EEA98C819D81F801958361
:109D200084831D821C82DF91CF911F910F91089532
:109D3000FC01808191810C9456A8EF92FF920F93C1
:109D40001F93CF93DF93CDB7DEB7A1970FB6F894EB
:109D5000DEBF0FBECDBF7C01CB01BA01F70111827E
:109D60001082138212821582148242E0420F8E0109
:109D70000F5F1F4F0E940B9EBC01C70175DFA196AC
:109D80000FB6F894DEBF0FBECDBFDF91CF911F910C
:109D90000F91FF90EF900895FC01118210821382C1
:109DA0001282158214823ACFFC0111821082138232
:109DB0001282158214826DCFFC01118210821382EF
:109DC0001282158214826115710549F0FB01019020
:109DD0000020E9F73197AF01461B570BA3CC08953C
:109DE000BF92CF92DF92EF92FF920F931F93CF9388
:109DF000DF937C016B018A01E9012417350720F408
:109E0000812F8901C42FD82F6AE37CE0C701D4DFFA
:109E1000D60114968D919C91159708171907C0F4D7
:109E20008C179D0708F4EC01D601ED91FC91119778
:109E3000EC0FFD1FB08010826D917C91600F711F3F
:109E4000C70112DFD601ED91FC91EC0FFD1FB0822E
:109E5000C701DF91CF911F910F91FF90EF90DF909D
:109E6000CF90BF900895DC01ED91FC910190F081BD
:109E7000E02D1994DB0114964D915C9115976D912D
:109E80007C91DC01ED91FC910280F381E02D19942D
:109E9000EF92FF920F931F93CF93DF938C017B017F
:109EA000C0E0D0E0F701EC0FFD1F6491662361F084
:109EB000D801ED91FC910190F081E02DC801199538
:109EC000892B11F02196EECFCE01DF91CF911F911A
:109ED0000F91FF90EF9008956115710579F0FB01E6
:109EE00001900020E9F73197AF01461B570BDC01C9
:109EF000ED91FC910280F381E02D199480E090E0D7
:109F000008958F929F92AF92BF92EF92FF920F931C
:109F10001F93CF93DF93CDB7DEB7A1970FB6F89419
:109F2000DEBF0FBECDBF7C01FA01CB0119A22230EA
:109F300008F42AE08E010F5D1F4F822E912CA12C78
:109F4000B12CBF01A50194010E94F9A3F901CA0136
:109F5000015011096A3014F4605D01C0695CD801D8
:109F60006C93232B242B252B61F7B801C701B4DF99
:109F7000A1960FB6F894DEBF0FBECDBFDF91CF9193
:109F80001F910F91FF90EF90BF90AF909F908F9097
:109F90000895CF92DF92EF92FF920F931F93CF938A
:109FA000DF934115510579F4DC01ED91FC910190AD
:109FB000F081E02DDF91CF911F910F91FF90EF90F5
:109FC000DF90CF9019946B01770FEE08FF084A30AD
:109FD0005105E9F4F7FE19C0EC016DE244DF8C0194
:109FE00044275527BA014C195D096E097F092AE0FB
:109FF000CE0187DF800F911FDF91CF911F910F91CD
:10A00000FF90EF90DF90CF9008952AE001C0242FB9
:10A01000B701A601DF91CF911F910F91FF90EF90B3
:10A02000DF90CF906ECF58CF1F920F920FB60F9246
:10A0300011240BB60F922F933F934F935F936F931F
:10A040007F938F939F93AF93BF93EF93FF9389E693
:10A050009EE075DAFF91EF91BF91AF919F918F9143
:10A060007F916F915F914F913F912F910F900BBE18
:10A070000F900FBE0F901F9018951F920F920FB662
:10A080000F9211240BB60F922F933F934F935F9330
:10A090006F937F938F939F93AF93BF93EF93FF93B0
:10A0A00089E69EE00E94918CFF91EF91BF91AF9164
:10A0B0009F918F917F916F915F914F913F912F91E0
:10A0C0000F900BBE0F900FBE0F901F9018951F9210
:10A0D0000F920FB60F9211240BB60F922F933F934E
:10A0E0004F935F936F937F938F939F93AF93BF93A0
:10A0F000EF93FF9386E09FE022DAFF91EF91BF910B
:10A10000AF919F918F917F916F915F914F913F910F
:10A110002F910F900BBE0F900FBE0F901F901895B0
:10A120001F920F920FB60F9211240BB60F922F931E
:10A130003F934F935F936F937F938F939F93AF93CF
:10A14000BF93EF93FF9386E09FE00E94918CFF9175
:10A15000EF91BF91AF919F918F917F916F915F919F
:10A160004F913F912F910F900BBE0F900FBE0F900C
:10A170001F9018951F920F920FB60F9211240BB6D5
:10A180000F922F933F934F935F936F937F938F9390
:10A190009F93AF93BF93EF93FF9383EA9FE0CFD951
:10A1A000FF91EF91BF91AF919F918F917F916F91AF
:10A1B0005F914F913F912F910F900BBE0F900FBE6B
:10A1C0000F901F9018951F920F920FB60F921124A7
:10A1D0000BB60F922F933F934F935F936F937F93A1
:10A1E0008F939F93AF93BF93EF93FF9383EA9FE087
:10A1F0000E94918CFF91EF91BF91AF919F918F91B0
:10A200007F916F915F914F913F912F910F900BBE76
:10A210000F900FBE0F901F9018951F920F920FB6C0
:10A220000F9211240BB60F922F933F934F935F938E
:10A230006F937F938F939F93AF93BF93EF93FF930E
:10A2400080E490E17CD9FF91EF91BF91AF919F9114
:10A250008F917F916F915F914F913F912F910F90CF
:10A260000BBE0F900FBE0F901F9018951F920F926C
:10A270000FB60F9211240BB60F922F933F934F936B
:10A280005F936F937F938F939F93AF93BF93EF935E
:10A29000FF9380E490E10E94918CFF91EF91BF9138
:10A2A000AF919F918F917F916F915F914F913F916E
:10A2B0002F910F900BBE0F900FBE0F901F9018950F
:10A2C000DC0180E0615098F02D91982F9227E92FC2
:10A2D000EF70F0E0EC5EF44F249192959F70E92FBF
:10A2E000F0E0EC5DF44FE491822F8E27EBCF0895E0
:10A2F000DF92EF92FF920F931F93CF93DF93EC01C6
:10A30000D62EE42E08E010E0FF24F39461E08D2DBA
:10A310008F2109F460E0CE010E942D86FF0C0150D0
:10A320001109A1F7E11010C0F894E981FA81918137
:10A330008881809589238183E981FA81928188814E
:10A340008095892382837894DF91CF911F910F911B
:10A35000FF90EF90DF900895EF92FF920F931F937D
:10A36000CF93DF938C017B0140E065E5C1DFE7011E
:10A3700088E0E80EF11C699140E0C801B9DFCE1514
:10A38000DF05C9F7DF91CF911F910F91FF90EF90FB
:10A3900008956F927F928F929F92AF92BF92CF92C9
:10A3A000DF92EF92FF920F931F93CF93DF93EC0115
:10A3B0007B018A018E819F810E945C86882399F1AE
:10A3C000B7018E819F81C8DF40E06EEB8E819F8157
:10A3D0008FDF7801680189E0C80ED11CAE80BF8094
:10A3E00088E0882E912C712C66246394C5010E940C
:10A3F000098681117628660CE1E08E1A9108B1F782
:10A40000F70171927F01EC15FD0541F78E819F8167
:10A410000E945C86813039F468E0C80151DF91E028
:10A42000F8012085281390E0892FDF91CF911F91AB
:10A430000F91FF90EF90DF90CF90BF90AF909F90E3
:10A440008F907F906F900895CF93DF93CDB7DEB755
:10A4500029970FB6F894DEBF0FBECDBFAE014F5F98
:10A460005F4F97DF882389F08D818F3361F020F46F
:10A470008F3159F489E00CC08F3519F08F3739F0DE
:10A4800004C08BE005C08AE003C080E001C08CE01E
:10A4900029960FB6F894DEBF0FBECDBFDF91CF91E6
:10A4A00008958F929F92AF92BF92CF92DF92EF92D8
:10A4B000FF920F931F93CF93DF938C01862F0B3066
:10A4C000110509F06FC090913113992309F0F894A8
:10A4D00062E10E941E5F20913113222309F07894DB
:10A4E000009709F072C0E0902C13F0902D136F2D9F
:10A4F00070E080E090E00E94A1A22DEC3CEC4CECDE
:10A500005DE30E9400A34B015C016E2D70E080E0D2
:10A5100090E00E94A1A29B01AC01C501B4010E9480
:10A520002BA4609324137093251380932613909388
:10A530002713C0912E13D0912F136C2F6F7770E0DB
:10A5400080E090E00E94A1A24B015C016D2F70E0C1
:10A5500080E090E00E94A1A22DEC3CEC4CEC5DE38D
:10A560000E9400A39B01AC01C501B4010E942BA471
:10A57000C7FD09C0609328137093291380932A1391
:10A5800090932B130BC0DC01CB01B05880932813A0
:10A5900090932913A0932A13B0932B13FE0CCF0D85
:10A5A000CD0F71C00631110509F0B4C0909131137F
:10A5B000992309F0F89461E00E941E5F2091311305
:10A5C000222309F078940097A9F040E050EC69E765
:10A5D00074EC4093241350932513609326137093C7
:10A5E0002713409328135093291360932A137093D1
:10A5F0002B1395C0F0902D13D0912C1360912C1338
:10A6000070912D1376276727762780E090E00E94CF
:10A610009FA22DEC3CEC4CEC5DE30E9400A3609308
:10A620002413709325138093261390932713E0909F
:10A630002F13C0912E138C2F8F776E2D70E0782BF7
:10A6400080E090E00E949FA22DEC3CEC4CEC5DE39E
:10A650000E9400A3C7FD09C06093281370932913BB
:10A6600080932A1390932B130BC0DC01CB01B058BD
:10A670008093281390932913A0932A13B0932B133C
:10A68000DF0DED0ECE0D80913013C81346C0C09083
:10A690002413D0902513E0902613F090271320E088
:10A6A00030E048EC52E4C701B6010E94E0A518165C
:10A6B0001CF0C0E0D0E002C0CBEFDFEF20E030E0E4
:10A6C000A901C701B6010E949BA287FF02C0CAEF81
:10A6D000DFEFC0902813D0902913E0902A13F09058
:10A6E0002B1320E030E048EC52ECC701B6010E9489
:10A6F0009BA287FF02C0C9EFDFEF20E030E040EF10
:10A7000052E4C701B6010E94E0A51816ACF4C8EFE8
:10A71000DFEF12C0CFEFDFEF0FC08FEF9FEF8F3F64
:10A72000FFEF9F0709F4D6C0009709F4B0CF029657
:10A7300009F4DCC0CCEFDFEF0C30110509F0D9C013
:10A740008CE50E94F97A80E090E00E94F47A0E9401
:10A75000F27A65E08CE50E949B5EC82FD0E02097DE
:10A76000A1F0C530D105A4F00BED1CE08DED90E11A
:10A770000E949085F80180870F5F1F4FC8018B5D95
:10A780009C408C179D0794F306C0CEEFDFEFB1C05D
:10A79000CDEFDFEFAEC0C091E30C0091E40C602F71
:10A7A00070E080E090E00E94A1A22DEC3CEC4CEC2B
:10A7B0005DE30E9400A36B017C016C2F70E080E0E0
:10A7C00090E00E94A1A29B01AC01C701B6010E94CA
:10A7D0002BA46093DB0C7093DC0C8093DD0C9093C6
:10A7E000DE0CD091E50C1091E60C6D2F6F7770E0C8
:10A7F00080E090E00E94A1A26B017C01612F70E0DB
:10A8000080E090E00E94A1A22DEC3CEC4CEC5DE3DA
:10A810000E9400A39B01AC01C701B6010E942BA4BA
:10A82000D7FF5BC0DC01CB01B0588093DF0C909365
:10A83000E00CA093E10CB093E20C8C2F800FC82F9A
:10A84000CD0FC10F8091E70CC81344C0C090DB0C42
:10A85000D090DC0CE090DD0CF090DE0C20E030E0DD
:10A8600048EC52E4C701B6010E94E0A518161CF09E
:10A87000C0E0D0E002C0CBEFDFEF20E030E040EA04
:10A8800050E4C701B6010E949BA287FF02C0CAEF35
:10A89000DFEFC090DF0CD090E00CE090E10CF09086
:10A8A000E20C20E030E040EF51ECC701B6010E941D
:10A8B0009BA287FF02C0C9EFDFEF20E030E040EF4E
:10A8C00052E4C701B6010E94E0A5181694F4C8EF3F
:10A8D000DFEF0FC0CFEFDFEF0CC06093DF0C7093A2
:10A8E000E00C8093E10C9093E20CA7CFCEEFDFEF6A
:10A8F00023CFCE01DF91CF911F910F91FF90EF9069
:10A90000DF90CF90BF90AF909F908F900895CF939E
:10A91000DF93FC0124813581232B69F0EC01BC011C
:10A9200080E490E10E94857ABE0189E69EE0DF9195
:10A93000CF910C94857ADF91CF910895CF92DF92D9
:10A94000EF92FF920F931F93CF93DF93CDB7DEB7B4
:10A9500028970FB6F894DEBF0FBECDBF823409F43E
:10A960003EC0C4F4803309F457C074F4833209F450
:10A970004BC08A3209F06CC060E47BE082EE92E169
:10A9800073D98FEF9FEF61C0813309F452C08134D6
:10A99000E1F05EC08136C9F02CF4833451F1843487
:10A9A00039F056C0833629F1D4F0843609F050C00E
:10A9B0008091DA129091DB12892B09F4DDC086EDCB
:10A9C00092E118D897FF75C0D7C064E37BE082EEB0
:10A9D00092E14AD98091A90C9091AA0C36C067E304
:10A9E0007BE082EE92E140D91092220D8CEF9FEF36
:10A9F0002CC06AE37BE082EE92E136D981E080935D
:10AA0000220D8DEF9FEF21C06DE37BE082EE92E19E
:10AA10002BD98EEF9FEF19C065EA7BE086ED92E1BE
:10AA200023D965EA7BE082EE92E11ED980E090E0D6
:10AA30000CC061E47BE086ED92E116D961E47BE035
:10AA400082EE92E111D981E090E00E94B2229AC098
:10AA50001A8219821C821B821E821D828F83188695
:10AA6000BE01695F7F4FCE010196FED8BE016F5FC8
:10AA70007F4F86ED92E122D9CE01019659D960E04F
:10AA800070E086ED92E121D8082E000C990B0E940F
:10AA9000C3A9892B39F086ED92E10E94FA4CCB01D3
:10AAA0000E94B22264E670E080E090E00E94868D11
:10AAB00069C080911F0D882359F06DE27BE080E42E
:10AAC00090E1B1DA66ED72E180E490E10E94857A6E
:10AAD00086ED92E10E94FA4C0AEF1FEF2FEF3FEF55
:10AAE00068017901C61AD70AE80AF90AB701A6016E
:10AAF000CE0101960E943F7B30C08FEFE81AF80A22
:10AB000085E6E816F10459F06EE170E080E090E02F
:10AB10000E94868D0E940E48182F112371F3809198
:10AB20001F0D882369F06DE27BE080E490E17BDA21
:10AB3000612F80E490E197D980E490E10E94817ACE
:10AB400010330CF414516AE270E0611B710917FDB7
:10AB50007395CE0101960E946F5EBE016F5F7F4FBD
:10AB600086ED92E1ABD8CE010196E2D886ED92E176
:10AB70000E94FA4CCB0169CF0E940E48182FE12C9D
:10AB8000F12CCBCF28960FB6F894DEBF0FBECDBF09
:10AB9000DF91CF911F910F91FF90EF90DF90CF90B9
:10ABA00008958F929F92AF92BF92CF92DF92EF92D1
:10ABB000FF92CF93DF93CDB7DEB72C970FB6F89403
:10ABC000DEBF0FBECDBF69EE7BE0CE010196E4D8BB
:10ABD0004CE251E06FEF7FEFCE0101960E94C07F03
:10ABE000CE010196A5D860918A0470918B04809162
:10ABF00041049091420455DC84E1882E912CA12CD3
:10AC0000B12CE12CF12C2FEFE21AF20AC501B401AC
:10AC10000E94868D60918A0470918B04809141041A
:10AC2000909142043EDC23E0E216F10434F02AE085
:10AC3000E216F10444F4892B49F084E1880E911C5A
:10AC4000A11CB11CE0CF892B09F07FC18091410488
:10AC5000909142048B309105C9F480912813909112
:10AC60002913A0912A13B0912B138093EC0C90938D
:10AC7000ED0CA093EE0CB093EF0C80912413909107
:10AC80002513A0912613B09127131DC0863191057D
:10AC900021F30C9701F58091DF0C9091E00CA091CD
:10ACA000E10CB091E20C8093EC0C9093ED0CA0932E
:10ACB000EE0CB093EF0C8091DB0C9091DC0CA0912A
:10ACC000DD0CB091DE0C8093E80C9093E90CA0931E
:10ACD000EA0CB093EB0C4091EC0C5091ED0C6091B0
:10ACE000EE0C7091EF0C21E0CE01079626D866EBB2
:10ACF0007BE0CE01019660D8BE01695F7F4FCE0137
:10AD000001960E94E94DBC018AEC92E10E94494EF5
:10AD1000CE0101960DD8CE0107960AD84091E80CD5
:10AD20005091E90C6091EA0C7091EB0C21E0CE019E
:10AD3000079603D860EC79E0CE0101963DD8BE01BC
:10AD4000695F7F4FCE0101960E94E94DBC018AECFC
:10AD500092E10E94084ECE0101960E94984ECE01CB
:10AD600007960E94984E62E879E08AEC92E10E9490
:10AD7000FA4D6AE37CE0CE0101961ED844E150E032
:10AD800060E070E0CE0101960E945560CE01019610
:10AD90000E94984EC090EC0CD090ED0CE090EE0C20
:10ADA000F090EF0C20E030E0A901C701B6010E944D
:10ADB000E0A520E030E040E05FE387FD05C0C7018B
:10ADC000B6010E942BA404C0C701B6010E942AA4A8
:10ADD0000E948AA5AB01BC01CE0101960E943F7B77
:10ADE000BE016F5F7F4F84EC92E10E945E4ECE0108
:10ADF00001960E94984E60E087E00E94147B64EC0C
:10AE000072E18BEC93E136D86FED8BEC93E12BD8AC
:10AE100066EC79E08BEC93E106D96091E80C7091D7
:10AE2000E90C8091EA0C9091EB0C0E948AA54AE013
:10AE300050E08BEC93E1ADD862E879E08BEC93E1E4
:10AE4000F2D864E670E080E090E00E94868DC090C9
:10AE5000EC0CD090ED0CE090EE0CF090EF0C20E0BC
:10AE600030E040EF51E4C701B6010E94E0A587FD44
:10AE700003C06AED7BE054C020E030E040ED51E4D7
:10AE8000C701B6010E94E0A587FD1FC06AEC7BE008
:10AE9000CE0101960E94CC4E4AE050E06FEF7FEF6A
:10AEA000CE0101960E94C07FCE0101960E94984E6D
:10AEB00080916F04882331F06CED75E080E090E0C4
:10AEC0000E94868D6AEB7BE02BC020E030E040EBF7
:10AED00051E4C701B6010E94E0A587FD03C06CEAFA
:10AEE0007BE01EC06DE97BE0CE0101960E94CC4E56
:10AEF0004AE050E06FEF7FEFCE0101960E94C07FE5
:10AF0000CE0101960E94984E80916F04882331F003
:10AF10006CED75E080E090E00E94868D6FE87BE04C
:10AF2000CE0101960E94CC4E4AE050E06FEF7FEFD9
:10AF3000CE0101960E94C07FCE0101960E94984EDC
:10AF400062E370E080E090E0DAC00E94927F6EE100
:10AF500070E080E090E00E94868D30D66B017C012D
:10AF600064E670E080E090E00E94868D66EB7BE016
:10AF70008AEC92E10E94344E21E0B701A601CE0195
:10AF800001960E949D4EBE016F5F7F4F8AEC92E159
:10AF90000E94084ECE0101960E94984E6AEC72E122
:10AFA000CE0101960E94D44E4AE050E060E070E08D
:10AFB000CE0101960E945560CE0101960E94984EE6
:10AFC00080918504882371F080918404882351F056
:10AFD0006FED8BEC93E10E94334F64E47BE08BECEC
:10AFE00093E121D863E47BE08AEC92E10E94FA4D80
:10AFF000C092EC0CD092ED0CE092EE0CF092EF0CC3
:10B0000020E030E040EF51E4C701B6010E94E0A526
:10B0100087FD03C06FE77BE054C020E030E040EDE7
:10B0200051E4C701B6010E94E0A587FD1FC06FE68D
:10B030007BE0CE0101960E94CC4E4AE050E06FEFDB
:10B040007FEFCE0101960E94C07FCE0101960E9443
:10B05000984E80916F04882331F06CED75E080E0AC
:10B0600090E00E94868D6FE57BE02BC020E030E011
:10B0700040EB51E4C701B6010E94E0A587FD03C083
:10B0800061E57BE01EC062E47BE0CE0101960E9498
:10B09000CC4E4AE050E06FEF7FEFCE0101960E9468
:10B0A000C07FCE0101960E94984E80916F04882344
:10B0B00031F06CED75E080E090E00E94868D64E3F5
:10B0C0007BE0CE0101960E94CC4E4AE050E06FEF4B
:10B0D0007FEFCE0101960E94C07FCE0101960E94B3
:10B0E000984E6CE271E080E090E00E94868D809145
:10B0F0006F04882331F068EE73E080E090E00E94F6
:10B10000868D2C960FB6F894DEBF0FBECDBFDF91B3
:10B11000CF91FF90EF90DF90CF90BF90AF909F9036
:10B120008F900895DF92EF92FF920F931F93CF932A
:10B13000DF93CDB7DEB762970FB6F894DEBF0FBED0
:10B14000CDBF8C011092F00C6AE37CE0CE010D962D
:10B150000E94DC4EFF24F39480E490E10E946F4A49
:10B160002091F00C18161906D4F5211138C080E48E
:10B1700090E10E944D4A8A3041F08D3031F0682FC5
:10B18000CE010D960E94E54923C089899A89892BB1
:10B19000F9F0F092F00C66E47BE0CE0101960E949B
:10B1A000DC4EBE01635F7F4FCE0101960E94E94DE8
:10B1B000BC01CE0107960E94D44ECE01079649D716
:10B1C000CE0107960E94984ECE0101960E94984E9D
:10B1D0006AE070E080E090E00E94868DBDCF211192
:10B1E00075C0E12CF12CDD24D39489E69EE00E9409
:10B1F0006F4A1816190614F589E69EE00E944D4A1A
:10B200008A3079F08D3069F09091F00C911109C07D
:10B21000682FCE010D960E94E5498FEFE81AF80AD3
:10B2200006C089899A89892B11F0D092F00C65E0CB
:10B2300070E080E090E00E94868DD7CF64E170E0FE
:10B2400080E090E00E94868DEF2851F189899A89EB
:10B25000892B31F180911F0D8823C1F06FE47BE0D1
:10B2600080E490E10E941350BE01635F7F4FCE01E6
:10B2700001960E94D44EBE016F5F7F4F80E490E143
:10B280000E94857ACE0101960E94984E89E69EE042
:10B290000E940D4B64E170E080E090E00E94868D9A
:10B2A0008091F00C811112C089899A89892B71F4DF
:10B2B00064E670E080E090E00E94868D0E94BE8D82
:10B2C0006AE37CE0C8010E94DC4E58C089899A89F3
:10B2D000019709F046C064E379E0CE0107960E9429
:10B2E000DC4EBE01695F7F4FCE010D960E94F8498A
:10B2F000811116C066E577E0CE0101960E94DC4E12
:10B30000BE016F5F7F4FCE010D960E94F849FF246A
:10B31000F3948111F12CCE0101960E94984E01C048
:10B32000F12CCE0107960E94984EFF20A1F040E03C
:10B3300050E0BE01635F7F4FCE0101960E945480B2
:10B34000BE016F5F7F4F86ED92E10E945E4ECE019F
:10B3500001960E94984E64E170E080E090E00E94C7
:10B36000868DF80111821082138212821582148256
:10B37000BE01635F7F4FC8010E945E4ECE010D96F5
:10B380000E94984EC80162960FB6F894DEBF0FBEB9
:10B39000CDBFDF91CF911F910F91FF90EF90DF9084
:10B3A0000895DF92EF92FF920F931F93CF93DF9355
:10B3B000CDB7DEB72C970FB6F894DEBF0FBECDBF6A
:10B3C0008C011092F00C6AE37CE0CE0107960E949B
:10B3D000DC4EE12CF12CDD24D39489E69EE00E9422
:10B3E0006F4A1816190614F58091F00C81111EC0D1
:10B3F00089E69EE00E944D4A8A3059F08D3049F02E
:10B40000682FCE0107960E94E5498FEFE81AF80AE7
:10B4100006C08B859C85892B11F0D092F00C6FE0D3
:10B4200070E080E090E00E94868DD7CF62E370E00C
:10B4300080E090E00E94868DEF2851F089E69EE042
:10B440000E940D4B64E670E080E090E00E94868DE3
:10B450008091F00C81110AC08B859C85892B31F479
:10B460006AE37CE0C8010E94DC4E1FC080911F0D82
:10B47000882371F0BE01695F7F4FCE0101960E9463
:10B48000D44ECE01019643DACE0101960E94984E29
:10B49000F801118210821382128215821482BE0179
:10B4A000695F7F4FC8010E945E4ECE0107960E94E1
:10B4B000984EC8012C960FB6F894DEBF0FBECDBFD4
:10B4C000DF91CF911F910F91FF90EF90DF90089542
:10B4D0009091450E9111FCCF91E09093450E909381
:10B4E000440E2FEF2093430E1092420E260F20930E
:10B4F000410E9093200E9091200E880F892B8093FF
:10B50000200E80911F0E813061F410921F0E8091E9
:10B51000200E8093BB008091BC0083FDF8CF85ECAA
:10B5200001C085EE8093BC008091450E8130E1F32F
:10B530008091420E861710F46091420EA1E2BEE0A7
:10B54000EBEFFCE080E0861721F09D9191938F5FF7
:10B55000FACF0895CF93DF93209185042223A9F099
:10B5600020918404222389F0EC016FED8BEC93E1B0
:10B570000E94334F8C819D81892B39F0BE018BEC69
:10B5800093E1DF91CF910C943A4FDF91CF910895E1
:10B59000CF93DF93EC010E940D4BEA89FB898081F8
:10B5A0008F7E8083EA89FB898081877F8083EA8917
:10B5B000FB8980818F778083EA89FB8980818F7DF9
:10B5C00080838A8D898FDF91CF9108953F924F922A
:10B5D0005F926F927F928F929F92AF92BF92CF9223
:10B5E000DF92EF92FF920F931F93CF93DF9300D0E0
:10B5F0001F921F92CDB7DEB7982E0E94BE8D2B01F1
:10B600003C0120ED420E27E0521E611C711C60E0DF
:10B610008091B5130E94D28C45E0842ECE01019614
:10B620006C01AA24A394B12CF601282D11922A951D
:10B63000E9F7860135E0332E27E0E22EF12C8091E8
:10B64000B6130E94AA8C019739F40E94BE8D64152E
:10B6500075058605970598F38091B6130E94AA8C0C
:10B66000892B39F40E94BE8D6415750586059705F2
:10B6700098F38091B7130E94AA8C892B51F0F8019E
:10B680002081C5010E2C01C0880F0A94EAF7822B95
:10B690008083F1E0EF1AF10890F63A940F5F1F4FA4
:10B6A0003110CACF0E94BE8D6415750586059705B9
:10B6B00050F061E08091B5130E94D28C60E070E0A0
:10B6C00080EC9FE72CC089818911AECF9A818B8154
:10B6D000890F890D9C818913A7CF8D818D3009F049
:10B6E000A3CF61E08091B5130E94D28C6A818B81D7
:10B6F00070E0762F6627680F711D072E000C880BEF
:10B70000990B0E94A1A220E030E040E85DE30E9496
:10B7100000A323E333E948E853E40E942AA40F90EE
:10B720000F900F900F900F90DF91CF911F910F917D
:10B73000FF90EF90DF90CF90BF90AF909F908F9051
:10B740007F906F905F904F903F900895613208F026
:10B7500060E2BEDE1092FA0C8093F90C0895CF934C
:10B76000C82F87E70E94F97A6C2F8DED90E10E9437
:10B77000D8850E94F27A87E70E94F97A61E070E04A
:10B7800087E790E0E3DF8DED90E10E949085C82F80
:10B790000E94F27A8C2FCF910895CF93DF93C82F18
:10B7A00087E70E94F97A6C2F8DED90E10E94D88591
:10B7B0000E94F27A87E70E94F97A62E070E087E7F8
:10B7C00090E0C4DF8DED90E10E949085D82F80E05D
:10B7D000C82F8DED90E10E949085C82BD92B0E9437
:10B7E000F27ACE01DF91CF91089587E70E94F97A2E
:10B7F00064EF8DED90E10E94D8856EE28DED90E1D1
:10B800000E94D8850E94F27A65E070E080E090E0C6
:10B810000E94868D86EFC1CF4F925F926F927F928A
:10B820008F929F92AF92BF92CF92DF92EF92FF9250
:10B830000F931F93CF93DF9300D01F921F92CDB72A
:10B84000DEB7D3DF4C01A12CB12C2091E812229558
:10B85000220F220F207C2C5C298387E70E94F97A33
:10B8600064EF8DED90E10E94D88569818DED90E1C6
:10B870000E94D8850E94F27A8091E812811105C059
:10B8800065E070E080E090E012C0813029F468E06B
:10B8900070E080E090E00BC0823029F46EE070E050
:10B8A00080E090E004C06AE170E080E090E00E94F7
:10B8B000868D86EF72DF6C01E12CF12CFE2CED2CD5
:10B8C000DC2CCC2488EF4BDFC82A3091E8123D8372
:10B8D0008091FD129091FE12A5019401281B390B55
:10B8E00041095109A091FB12B091FC120E94E9A3F9
:10B8F0002B013C01AFE07594679457944794AA9547
:10B90000D1F76091F5127091F612CB01770FAA0B67
:10B91000BB0BBC01CD01BBE0660F771F881F991FD1
:10B92000BA95D1F72091F7123091F8128901330FAF
:10B93000220B330BA9019801240D351D461D571DFF
:10B940000E94CDA3420E531E641E751E40EA441A87
:10B950004FE0540A61087108A3019201C301B201CA
:10B960000E9449A79B01AC011CE05595479537956E
:10B9700027951A95D1F729833A834B835C83E0910D
:10B98000E912F091EA12A091ED12B091EE12A3012A
:10B9900092010E94F3A34B015C010DE0B594A794C2
:10B9A000979487940A95D1F7A091EF12B091F01275
:10B9B00029813A814B815C810E94F3A3BB2797FDCB
:10B9C000B095AB2F880D991DAA1DBB1D0296A11D18
:10B9D000B11D32E0B595A795979587953A95D1F722
:10B9E0009C01AD0130584F4F5F4FA091F912B091BB
:10B9F000FA120E94E9A34B015C014FE0B694A794B0
:10BA0000979487944A95D1F788E090E03D81831B15
:10BA1000910904C0F694E794D794C7948A95D2F715
:10BA2000A091F112B091F21229813A814B815C818F
:10BA30000E94F3A39B01AC016BE0559547953795A8
:10BA400027956A95D1F729833A834B835C83A0912C
:10BA5000EB12B091EC12A30192010E94F3A3DC015E
:10BA6000CB017BE0B595A795979587957A95D1F70A
:10BA700049815A816B817C81480F591F6A1F7B1F46
:10BA8000CF01FF0FAA0BBB0BE2E0880F991FAA1F83
:10BA9000BB1FEA95D1F7840F951FA61FB71F0D8016
:10BAA00004C0880F991FAA1FBB1F0A94D2F7BC01BC
:10BAB000CD016E5F7F4F8F4F9F4F24E030E040E01D
:10BAC00050E00E94CDA3D701C601821B930BA40BAB
:10BAD000B50B9C01AD0180E593ECA0E0B0E0BC01AA
:10BAE000CD010D8004C096958795779567950A944A
:10BAF000D2F70E9449A797FD0BC0660F771F881FDA
:10BB0000991FA50194010E94F9A349015A010AC095
:10BB1000A50194010E94F9A349015A01880C991CBE
:10BB2000AA1CBB1C9927B7FC9A958B2D7A2D692DE1
:10BB30009B01AC010E9449A79B01AC01AEEDBBE0AB
:10BB40000E94E9A36B017C01A3E4B3EEA50194017B
:10BB50000E94F5A3BB2797FDB095AB2F6701FF248B
:10BB6000D7FCF094EF2C8C0D9D1DAE1DBF1D815395
:10BB7000914FAF4FBF4F44E0B595A79597958795E7
:10BB80004A95D1F7BC01CD01680D791D8A1D9B1D19
:10BB90000F900F900F900F900F90DF91CF911F910A
:10BBA0000F91FF90EF90DF90CF90BF90AF909F905C
:10BBB0008F907F906F905F904F900895CF92DF921B
:10BBC000EF92FF920F931F9310DEAC0160E070E0E4
:10BBD000E8EEF2E1858996899A01AB01281B390BC1
:10BBE00041095109A389B4890E94E9A36B017C0131
:10BBF0008FE0F594E794D794C7948A95D1F765853B
:10BC00007685CB01770FAA0BBB0BBC01CD012BE0D6
:10BC1000660F771F881F991F2A95D1F727853089CE
:10BC20008901330F220B330BA90198012C0D3D1D07
:10BC30004E1D5F1D0E94CDA3DA01C9018C0D9D1D13
:10BC4000AE1DBF1D0896A11DB11DBC01CD0134E084
:10BC500095958795779567953A95D1F70E94A1A21A
:10BC600020E030E040E251E40E94F1A41F910F91E6
:10BC7000FF90EF90DF90CF9008951092FA0C109201
:10BC8000F90C1092470E1092680E1092450E81E04A
:10BC90008093440E10921F0E61E084E10E94D28CCA
:10BCA00061E085E10E94D28CE9EBF0E080818E7F3B
:10BCB000808380818D7F808388E48093B80085E4D1
:10BCC0008093BC008EE795E89093F80C8093F70C76
:10BCD0008FE795E89093F60C8093F50C08950F93F9
:10BCE0001F93CF93DF93CDB7DEB762970FB6F8946B
:10BCF000DEBF0FBECDBF8C01CB01F80111821082D7
:10BD000013821282158214824AE0BE016F5F7F4F58
:10BD10000E94639EBE016F5F7F4FC8010E94344E38
:10BD200062960FB6F894DEBF0FBECDBFDF91CF9104
:10BD30001F910F910895613208F060E2C9DB109203
:10BD4000FA0C8093F90C0895CF92DF92EF92FF9254
:10BD50000F931F93C0908004D0908104E0908204E0
:10BD6000F090830420E030E040E450E4C701B601E5
:10BD70000E94E0A518166CF420E030E04AEF54E48D
:10BD8000C701B6010E9400A30E948AA56B017C0135
:10BD900006C080E3C82E85E7D82EE12CF12C0E9446
:10BDA000927F60E080E00E94147B6FEF7BE08BEC81
:10BDB00093E10E94484F61E080E00E94147B67EFAE
:10BDC0007BE08BEC93E10E94484F64E670E080E0FA
:10BDD00090E00E94868D0E94BE8D6093F10C70935E
:10BDE000F20C8093F30C9093F40C0E94BE8D0091A2
:10BDF000F10C1091F20C2091F30C3091F40CDC0159
:10BE0000CB01801B910BA20BB30B8C159D05AE05CE
:10BE1000BF056CF483E090E00E9460800E94BE8DBC
:10BE200064E170E080E090E00E94868DDECF1F919B
:10BE30000F91FF90EF90DF90CF900895AF92BF9257
:10BE4000CF92DF92EF92FF920F931F93CF93DF93E6
:10BE5000C82FD62F10922C1310922D1310922E1340
:10BE600010922F131092301361E00E94008D60E059
:10BE70008C2F0E94D28C6D2F70E080E090E00E94A9
:10BE8000868D60E08C2F0E94008D8BE990E00197F9
:10BE9000F1F700E911E08C2F0E94AA8C892B31F474
:10BEA00001501109C1F78EEF9FEF4CC000E911E07E
:10BEB0008C2F0E94AA8C019709F43FC018E2D0E8A9
:10BEC00000E090E9E92EFF24F3948C2F0E94AA8CC5
:10BED000892B29F481E0E81AF108B9F7E4CF0E9430
:10BEE000618D6B017C0180E9A82EBB24B3948C2F5B
:10BEF0000E94AA8C019729F481E0A81AB108B9F729
:10BF0000D2CF0E94618DDC01CB018C199D09AE0955
:10BF1000BF098997A105B10538F0E02FF0E0EC5D8D
:10BF2000FC4E80858D2B8087D69511F40F5FD0E86D
:10BF3000115039F680E090E005C00150110909F078
:10BF4000B7CFB1CFDF91CF911F910F91FF90EF90BD
:10BF5000DF90CF90BF90AF900895EF92FF920F9334
:10BF60001F93CF93DF93C82F8B017A0183E50E9443
:10BF7000F97A6C2F8DED90E10E94D8850E94F27ABB
:10BF800083E50E94F97AB80183E590E0DFDBE70101
:10BF9000CE018E199F093091F90C2091FA0C3217BD
:10BFA00031F08DED90E10E9490858993F1CF0817D3
:10BFB000190729F01092321381E080933313DF9137
:10BFC000CF911F910F91FF90EF900C94F27ACF9345
:10BFD000DF934AE050E0BC0180E490E10E94C94F49
:10BFE000EC0180E490E10E94817A8C0F9D1FDF912B
:10BFF000CF9108951F93CF93DF931F92CDB7DEB7F4
:10C00000162FAE014F5F5F4F61E070E0A6DF8981C0
:10C0100090E002C0959587951A95E2F781700F9090
:10C02000DF91CF911F910895CF93DF93D82FC62F23
:10C0300083E50E94F97A6D2F8DED90E10E94D885FD
:10C040006C2F8DED90E10E94D885DF91CF910C94FB
:10C05000F27A0F931F93CF93DF9300D000D0CDB728
:10C06000DEB720911F0D2223A9F08C0164E87BE04C
:10C07000CE0101960E94DC4EB801CE0101960E94CD
:10C08000E94DBC0180E490E10E94857ACE010196E1
:10C090000E94984E26960FB6F894DEBF0FBECDBF15
:10C0A000DF91CF911F910F910895BF92CF92DF92B0
:10C0B000EF92FF920F931F93CF93DF93CDB7DEB72D
:10C0C00062970FB6F894DEBF0FBECDBF6C018B0137
:10C0D0007A0180918504882309F47CC080918404CE
:10C0E000882309F477C077FF07C00095109560E0BA
:10C0F000802F0E94147B4DC060E080E00E94147B82
:10C100000E94BE8D28EE33E040E050E00E94CDA3B7
:10C11000CA01B90120E831E541E050E00E94CDA319
:10C12000AB01BC01CE0107960E943F7BBE01695F57
:10C130007F4FCE0101960E94D44E66E576E0CE0197
:10C1400001960E94D24DBC01CE010D960E94D44EA4
:10C15000CE0101960E94984ECE0107960E94984EFD
:10C16000BE01635F7F4F8BEC93E10E943A4FB98829
:10C1700060E08B2D0E94147B0115110511F40B2D2D
:10C1800004C060E0802F0E94147BCE010D960E94B7
:10C19000984EB6018BEC93E10E943A4F61E27CE04D
:10C1A0008BEC93E10E94484FF601848160E0800FA0
:10C1B0000E94147B0E94BE8D60931B0D70931C0D1A
:10C1C00080931D0D90931E0DB701FF0C880B990BEA
:10C1D0000E94868D62960FB6F894DEBF0FBECDBF6B
:10C1E000DF91CF911F910F91FF90EF90DF90CF9053
:10C1F000BF900895AF92BF92CF92DF92EF92FF92DD
:10C200000F931F93CF93DF93CDB7DEB762970FB62F
:10C21000F894DEBF0FBECDBF20918504222309F420
:10C2200091C020918404222309F48CC06A017B010F
:10C230005C010E94BE8D00911B0D10911C0D209180
:10C240001D0D30911E0D0C591F4F2F4F3F4F0617DC
:10C2500017072807390708F075C0F7FE08C08701DF
:10C260000095109560E0802F0E94147B4AC060E02A
:10C2700080E00E94147B0E94BE8D28EE33E040E0F7
:10C2800050E00E94CDA3CA01B90120E831E541E0A8
:10C2900050E00E94CDA3AB01BC01CE0101960E94EB
:10C2A0003F7BBE016F5F7F4FCE0107960E94D44E49
:10C2B00066E576E0CE0107960E94D24DBC01CE0124
:10C2C0000D960E94D44ECE0107960E94984ECE0144
:10C2D00001960E94984EBE01635F7F4F8BEC93E105
:10C2E0000E943A4F09891A89E114F10431F00E0DC8
:10C2F0001F1D60E0802F0E94147BCE010D960E94CE
:10C30000984EB5018BEC93E10E943A4F60E17CE0DE
:10C310008BEC93E10E94484FF501848160E0800F2F
:10C320000E94147B0E94BE8D60931B0D70931C0DA8
:10C3300080931D0D90931E0DB601DD0C880B990B9B
:10C340000E94868D62960FB6F894DEBF0FBECDBFF9
:10C35000DF91CF911F910F91FF90EF90DF90CF90E1
:10C36000BF90AF9008954F925F926F927F92AF927D
:10C37000BF92CF92DF92EF92FF920F931F93CF93D2
:10C38000DF9300D000D0CDB7DEB781E080931202FA
:10C3900083E39DE00E942D37892B09F4A4C280918C
:10C3A0002714882319F01092271488C61092271496
:10C3B00080911F0D8823D1F164E87BE0CE010196C6
:10C3C0000E94DC4EBE016F5F7F4F80E490E10E94CF
:10C3D0003A4FBE016F5F7F4F89E69EE00E943A4F61
:10C3E000CE0101960E94984E4091370D5091380D24
:10C3F0006091390D70913A0D20E180E490E10E9446
:10C40000814F80E490E10E94817A4091370D5091F4
:10C41000380D6091390D70913A0D20E189E69EE06A
:10C420000E94814F89E69EE00E94817A8091370DBB
:10C430009091380DA091390DB0913A0D883025E0DA
:10C440009207A105B10509F4DDC108F08DC089345A
:10C4500021E09207A105B10509F4DDC1E0F58434BE
:10C4600021E09207A105B10509F4A8C1E8F48134DF
:10C4700021E09207A105B10509F485C138F48034A3
:10C480009140A105B10509F46FC11BC2823421E0BE
:10C490009207A105B10509F47FC183349140A1053C
:10C4A000B10509F482C10DC2863421E09207A105CD
:10C4B000B10509F495C108F48AC1873421E09207D7
:10C4C000A105B10509F495C188349140A105B105D4
:10C4D00009F498C1F6C1823025E09207A105B105A3
:10C4E00009F45AC1E8F4843721E09207A105B105A7
:10C4F00009F405C138F482379140A105B10509F46A
:10C5000009C1DFC1811525E09207A105B10509F434
:10C510002BC181309540A105B10509F434C1D1C1C9
:10C52000853025E09207A105B10509F450C170F4EA
:10C53000833025E09207A105B10509F436C18430A6
:10C540009540A105B10509F439C1BBC1863025E08C
:10C550009207A105B10509F443C187309540A105B3
:10C56000B10509F446C1ADC18D3B22E492072FEF1E
:10C57000A207B10509F4E9C008F04BC08F3E20E1E5
:10C5800092072FEFA207B10509F433C118F58233E2
:10C5900025E09207A105B10509F4BCC038F4893043
:10C5A0009540A105B10509F436C18BC1843325E05E
:10C5B0009207A105B10509F4A2C08D3F9240AF4F8B
:10C5C000B10509F07EC164E37BE082EE92E10E9456
:10C5D000344E90C08D3D22E292072FEFA207B105A5
:10C5E00009F48DC038F4873E9841AF4FB10509F486
:10C5F000EEC067C18F3C20E392072FEFA207B10581
:10C6000009F4DCC0873C9843AF4FB10509F4FAC088
:10C6100058C1873928E692072FEFA207B10509F420
:10C62000B2C040F58D3A22E592072FEFA207B1057F
:10C6300009F47CC038F4853B9A44AF4FB10509F446
:10C6400093C03FC1853A2AE592072FEFA207B105B3
:10C6500009F4E1C08D399246AF4FB10509F031C1FF
:10C6600064E37BE082EE92E10E94344E81E08093AD
:10C67000220D40C0873528EA92072FEFA207B105A7
:10C68000F1F078F485382AE792072FEFA207B10579
:10C6900009F4A6C087369849AF4FB10509F47CC0AC
:10C6A00010C18F3420EB92072FEFA207B10509F4D8
:10C6B0007CC08D33924CAF4FB10561F102C16CE289
:10C6C00071E080E090E00E94868D82E08093E91026
:10C6D0001092EC1000E010E083E29DE00E942D3704
:10C6E000892B09F0A1C00F5F1F4F0536110509F016
:10C6F000BEC49AC08BEF9FEF0E94B222E8C067E3EE
:10C700007BE082EE92E10E94344E1092220D8CEF7B
:10C710009FEFF2CF6AE37BE082EE92E10E94344E1B
:10C7200081E08093220D8DEF9FEFE6CF6DE37BE0FC
:10C7300082EE92E10E94344E6DE37BE082EE92E164
:10C740000E94344E8EEF9FEFD7CF60E47BE082EE05
:10C7500092E10E94344E60E47BE082EE92E10E941E
:10C76000344E8FEF9FEFC8CF65EA7BE086ED92E114
:10C770000E94344E65EA7BE082EE92E10E94344EE4
:10C7800080E090E0B9CF61E47BE086ED92E10E9429
:10C79000344E81E090E0B0CF6EE37BE086ED92E135
:10C7A0000E94344E82E090E0A7CF6BE37BE086ED01
:10C7B00092E10E94344E83E090E09ECF68E37BE0FC
:10C7C00086ED92E10E94344E84E090E095CF65E3DF
:10C7D0007BE086ED92E10E94344E85E090E08CCFC4
:10C7E00067E57BE086ED92E10E94344E86E090E0C2
:10C7F00083CF6AE57BE086ED92E10E94344E87E0CC
:10C8000090E07ACF6DE57BE086ED92E10E94344EB8
:10C8100088E090E071CF60E67BE086ED92E10E94D7
:10C82000344E89E090E068CF80911F0D8823B9F0E5
:10C830006DEB7CE080E490E10E94484F4091270D31
:10C840005091280D6091290D70912A0D2AE080E405
:10C8500090E10E94814F80E490E10E94817A809172
:10C86000270D9091280DA091290DB0912A0D8830A7
:10C8700025E09207A105B10509F4CFC308F0E8C28D
:10C88000893421E09207A105B10509F4CFC308F06E
:10C8900096C2843421E09207A105B10509F499C339
:10C8A00008F076C2813421E09207A105B10509F4B0
:10C8B00075C308F05FC280349140A105B10509F449
:10C8C00064C364E670E080E090E00E94868D6CE2D4
:10C8D00071E080E090E00E94868D82E08093E91014
:10C8E0001092EC1047C0CE0101960E949258BE01F2
:10C8F0006F5F7F4F82EE92E10E945E4ECE01019605
:10C900000E94984E6AE070E080E090E00E94868D80
:10C910008091E6129091E712892B19F00E94C408C9
:10C920001DC20E940E48182F882379F18091271488
:10C93000811139CD6AE37CE086ED92E10E94344EAC
:10C9400080911F0D882379F06BEE7CE080E490E10C
:10C950000E94484F612F80E490E10E94334F80E4B1
:10C9600090E10E94817A812F0E949E541A3211F028
:10C97000109227140E94BE8D6093860C7093870CD2
:10C980008093880C9093890CE9C18091BF11882312
:10C9900009F49AC18091C9119091CA1197FF04C0FE
:10C9A0001092CA111092C9118091C7119091C811AB
:10C9B000181619069CF42091C9113091CA11281734
:10C9C000390764F01092BF111092C4118CE291E00B
:10C9D0000E943F7F1092CA111092C911E091CB11B1
:10C9E0008091C611E817D4F18091220D811107C002
:10C9F0008091C7119091C8111816190634F50E943C
:10CA0000BE8D28EE33E040E050E00E94F9A3CA0159
:10CA1000B9010E949FA22091820C3091830C409119
:10CA2000840C5091850C0E942AA42091130230910D
:10CA3000140240911502509116020E94E0A51816AA
:10CA40000CF08CC11092CB1189C11092C4111092BC
:10CA5000BF118CE291E00E943F7F80C10E2F0E2E0D
:10CA6000000C110B8AE0E802F0011124EC53FE4E99
:10CA7000E7840E2C000CFF088091CC11A82E880FA3
:10CA8000BB080E94BE8D4090BB115090BC116090BD
:10CA9000BD117090BE11641975098609970928EEB9
:10CAA00033E040E050E00E94F9A3CA01B9010E94BE
:10CAB0009FA22B013C016701F7FE04C0CC24DD24BA
:10CAC000CE18DF08C501B7FE02C080E090E08C15EB
:10CAD0009D050CF098C08AE0809FF001819FF00DC9
:10CAE0001124EC53FE4E60897189072E000C880BCF
:10CAF000990B0E94A1A29B01AC01C301B2010E944B
:10CB0000E0A518160CF02AC1F7FE09C08091C911E2
:10CB10009091CA11B6010E946CA7892B71F48AE02A
:10CB2000809FF001819FF00D1124EC53FE4E86850D
:10CB3000082E000C990B0E94B2220E94BE8D6093B9
:10CB4000BB117093BC118093BD119093BE11809165
:10CB5000CC118F5F8093CC11082E000C990B8C1593
:10CB60009D050CF4FBC08091C611082E000C990B9A
:10CB70000197081719070CF4F1C08091C911909121
:10CB8000CA1101969093CA118093C9118091220D08
:10CB9000811108C08091C7119091C811181619060B
:10CBA0000CF08CC28CE291E00E943F7F60ED7CE053
:10CBB0008AEC92E10E940E4E6091C9117091CA11E7
:10CBC000CE0101968CD8BE016F5F7F4F8AEC92E157
:10CBD0000E94084ECE0101960E94984E6CED75E0C1
:10CBE00080E090E00E94868D6AEC72E1CE010196B1
:10CBF0000E94D44ECE0101960E948754CE01019628
:10CC00000E94984EABC03AE0F32EF09EF001F19EE8
:10CC1000F00D1124EC53FE4E62897389072E000C2F
:10CC2000880B990B0E94A1A29B01AC01C301B20128
:10CC30000E94E0A518160CF091C01092CC118091C2
:10CC4000CB118F5F8093CB11082E000C990B209194
:10CC5000C611022E000C330B8217930704F5F89EC1
:10CC6000F001F99EF00D1124EC53FE4E878587FDEF
:10CC700006C08685082E000C990B0E94B2220E94E5
:10CC8000BE8D6093BB117093BC118093BD119093C6
:10CC9000BE118091CC118F5F8093CC115FC00E9438
:10CCA000BE8D28EE33E040E050E00E94F9A3CA01B7
:10CCB000B9010E949FA26093820C7093830C8093B1
:10CCC000840C9093850C4AC08091220D882309F42E
:10CCD000D5C10E94BE8D28EEC22E23E0D22EE12CBB
:10CCE000F12CA70196010E94F9A3CA01B9010E9483
:10CCF0009FA22091820C3091830C4091840C509122
:10CD0000850C0E942AA420911302309114024091B4
:10CD10001502509116020E94E0A518160CF0AEC143
:10CD20000E94BE8DA70196010E94F9A3CA01B90114
:10CD30000E949FA26093820C7093830C8093840C5A
:10CD40009093850C8091200D9091210D0E94B2222C
:10CD500064E170E080E090E00E94868D8091220D79
:10CD6000882309F4ABC164E670E080E090E00E94A3
:10CD7000868DA4C1823421E09207A105B10509F492
:10CD800016C183349140A105B10509F419C199CDAB
:10CD9000863421E09207A105B10509F42CC108F4FD
:10CDA00021C1873421E09207A105B10509F42CC106
:10CDB00088349140A105B10509F42FC182CD82309C
:10CDC00025E09207A105B10509F4F1C0E8F4843724
:10CDD00021E09207A105B10509F434C138F4823786
:10CDE0009140A105B10509F436C16BCD811525E04F
:10CDF0009207A105B10509F4C8C081309540A1058D
:10CE0000B10509F4CBC05DCD853025E09207A105C1
:10CE1000B10509F4E7C070F4833025E09207A1055D
:10CE2000B10509F4CDC084309540A105B10509F4E0
:10CE3000D0C047CD863025E09207A105B10509F4A1
:10CE4000DAC087309540A105B10509F4DDC039CDC0
:10CE50008D3B22E492072FEFA207B10509F4FEC033
:10CE600008F045C08F3E20E192072FEFA207B105E1
:10CE700009F4CAC0E8F4823325E09207A105B105A0
:10CE800009F4E9C038F489309540A105B10509F4E9
:10CE9000CDC017CD843325E09207A105B10509F473
:10CEA000D1C08D3F9240AF4FB10509F410CD09CDEF
:10CEB0008D3D22E292072FEFA207B10509F4C2C00F
:10CEC00038F4873E9841AF4FB10509F48BC0F9CCD7
:10CED0008F3C20E392072FEFA207B10509F479C038
:10CEE000873C9843AF4FB10509F497C0EACC873926
:10CEF00028E692072FEFA207B10509F44FC000F50D
:10CF00008D3A22E592072FEFA207B10509F4DFCC95
:10CF100030F4853B9A44AF4FB105B9F1D2CC853A94
:10CF20002AE592072FEFA207B10509F47FC08D39DA
:10CF30009246AF4FB10509F0C4CC87EE9FEFDCCB32
:10CF4000873528EA92072FEFA207B10509F477C0C9
:10CF500070F485382AE792072FEFA207B10509F48C
:10CF60004AC087369849AF4FB10509F1AACC8F3432
:10CF700020EB92072FEFA207B10511F18D33924CF0
:10CF8000AF4FB10509F467C09CCC66E57BE086ED48
:10CF900092E10E94344E8AEF9FEFAECB69E57BE0D1
:10CFA00086ED92E10E94344E89EF9FEFA5CB6CE5B0
:10CFB0007BE086ED92E10E94344E88EF9FEF9CCBA0
:10CFC0006FE57BE086ED92E10E94344E87EF9FEFA4
:10CFD00093CB62E67BE086ED92E10E94344E86EFD1
:10CFE0009FEF8ACB66E67BE086ED92E10E94344EAD
:10CFF00085EF9FEF81CB6AE67BE086ED92E10E94B0
:10D00000344E84EF9FEF78CB6EE67BE086ED92E1C5
:10D010000E94344E83EF9FEF6FCB62E77BE086ED9B
:10D0200092E10E94344E82EF9FEF66CB66E77BE091
:10D0300086ED92E10E94344E81EF9FEF5DCB86EE4C
:10D040009FEF5ACB6AE77BE082EE92E10E94344E7A
:10D0500088EE9FEF51CB89EE9FEF4ECB6EE77BE0E2
:10D0600082EE92E10E94344E84E190E045CB6EE185
:10D0700070E080E090E00E94868D2ECB0E94BE8DF5
:10D080000091860C1091870C2091880C3091890CAE
:10D09000DC01CB01801B910BA20BB30B88349E4E9D
:10D0A000A105B10508F45ACE1092D61360E08BECBE
:10D0B00093E10E94BD861092840450CE26960FB64E
:10D0C000F894DEBF0FBECDBFDF91CF911F910F91BE
:10D0D000FF90EF90DF90CF90BF90AF907F906F90D8
:10D0E0005F904F900895BF92CF92DF92EF92FF92A0
:10D0F0000F931F93CF93DF93CDB7DEB762970FB631
:10D10000F894DEBF0FBECDBF8C016B0166EE7BE0F5
:10D11000CE010D960E94DC4E6BEB7CE0C8010E94B4
:10D12000CC4E76012FEFE21AF20AB701CE0101963A
:10D130000E946F5EBE016F5F7F4FCE0107960E9417
:10D14000D44E60E778E0CE0107960E94D24DBC0134
:10D15000C8010E94084ECE0107960E94984ECE014B
:10D1600001960E94984E8AE0B82EBE9CC001BF9CDA
:10D17000900D1124FC01EC53FE4E7F018081082E9E
:10D18000000C990B0E94D6A9892B09F4B2C0B701F3
:10D19000CE0101960E94DC4EBE016F5F7F4FCE0133
:10D1A00007960E94D44E69E176E0CE0107960E9470
:10D1B000D24DBC01C8010E94084ECE0107960E94C4
:10D1C000984ECE0101960E94984EBC9CC001BD9C19
:10D1D000900D11249C012C533E4E7901F901668576
:10D1E000062E000C770BCE0101960E946F5EBE01E9
:10D1F0006F5F7F4FCE0107960E94D44E61E87BE0BF
:10D20000CE0107960E94D24DBE01635F7F4F0E9400
:10D21000E94DBC01C8010E94084ECE0107960E944C
:10D22000984ECE0101960E94984E64EB7CE0C801B6
:10D230000E94764DF7016785062E000C770BCE0114
:10D2400001960E946F5EBE016F5F7F4FCE01079611
:10D250000E94D44EBE01635F7F4FCE0107960E94AD
:10D26000E94DBC01C8010E94084ECE0107960E94FC
:10D27000984ECE0101960E94984E6EEA7CE0C8015D
:10D280000E94764DF70160897189CE0101960E9456
:10D290006F5EBE016F5F7F4FCE0107960E94D44E36
:10D2A000BE01635F7F4FCE0107960E94E94DBC012E
:10D2B000C8010E94084ECE0107960E94984ECE01EA
:10D2C00001960E94984E69EA7CE0C8010E94764D62
:10D2D000F70162897389CE0101960E946F5EBE01DB
:10D2E0006F5F7F4FC8010E94084ECE0101960E94D9
:10D2F000984ECE010D960E94984EC80162960FB6C8
:10D30000F894DEBF0FBECDBFDF91CF911F910F917B
:10D31000FF90EF90DF90CF90BF900895EF92FF9233
:10D320000F931F93CF93DF93CDB7DEB768970FB6F8
:10D33000F894DEBF0FBECDBF8C0166EE7BE0CE0160
:10D340000D960E94DC4E63E87BE0CE0143960E947E
:10D35000DC4E65E87CE0C8010E94CC4EBE016D5EEB
:10D360007F4FC8010E94084E6CE77CE0C8010E9414
:10D37000764D84ECE82E81E1F82EF701608170E0B3
:10D38000CE0101960E946F5EBE016F5F7F4FCE019E
:10D3900007960E94D44EBE01635F7F4FCE01079671
:10D3A0000E94E94DBC01C8010E94084ECE010796BB
:10D3B0000E94984ECE0101960E94984E6FE67CE046
:10D3C000C8010E94764DF7016181062E000C770B93
:10D3D000CE0101960E946F5EBE016F5F7F4FCE014E
:10D3E00007960E94D44EBE01635F7F4FCE01079621
:10D3F0000E94E94DBC01C8010E94084ECE0107966B
:10D400000E94984ECE0101960E94984E65E67CE0FF
:10D41000C8010E94764DF7016281062E000C770B41
:10D42000CE0101960E946F5EBE016F5F7F4FCE01FD
:10D4300007960E94D44EBE01635F7F4FCE010796D0
:10D440000E94E94DBC01C8010E94084ECE0107961A
:10D450000E94984ECE0101960E94984E6DE57CE0A8
:10D46000C8010E94764DF70163817481CE01019657
:10D470000E946F5EBE016F5F7F4FCE0107960E94D4
:10D48000D44EBE016D5E7F4FCE0107960E94E94DDE
:10D49000BC01C8010E94084ECE0107960E94984E1A
:10D4A000CE0101960E94984E66E47CE0C8010E947D
:10D4B000764DF70165817681CE0101960E946F5EFF
:10D4C000BE016F5F7F4FCE0107960E94D44EBE0112
:10D4D000635F7F4FCE0107960E94E94DBC01C801F2
:10D4E0000E94084ECE0107960E94984ECE010196EA
:10D4F0000E94984E6DE37CE0C8010E94764DF701D2
:10D500006781062E000C770B6F5F7F4FCE0101966F
:10D510000E946F5EBE016F5F7F4FCE0107960E9433
:10D52000D44EBE01635F7F4FCE0107960E94E94D46
:10D53000BC01C8010E94084ECE0107960E94984E79
:10D54000CE0101960E94984E62E37CE0C8010E94E1
:10D55000764DF7016085062E000C770BCE01019603
:10D560000E946F5EBE016F5F7F4FC8010E94084E30
:10D57000CE0101960E94984ECE0143960E94984E8D
:10D58000CE010D960E94984EC80168960FB6F89489
:10D59000DEBF0FBECDBFDF91CF911F910F91FF90E6
:10D5A000EF9008950F931F9360E080912A040E94EA
:10D5B000D28C83E090E00197F1F761E080912A043A
:10D5C0000E94D28C83E290E00197F1F760E08091B5
:10D5D0002A040E94D28C80912804909129049927D2
:10D5E000FC01EE56FF4E6491FC01E45BFF4EE491BA
:10D5F000F0E0EE0FFF1FEE5CFF4E8591949100E48A
:10D6000012E42FE030E0462F0E9439916115710538
:10D610008105910549F0DC01CB010196A11DB11DE9
:10D62000BC01CD019F7003C060E070E0CB010E949F
:10D630009FA220E030E048EC52E40E94F1A4209147
:10D64000430D3091440D4091450D5091460D0E947F
:10D6500000A320E030E44CE156E40E94F1A420E075
:10D6600030E040E05FE30E9400A31F910F91089516
:10D6700023E333E948E853E40E94F1A420E030E0DA
:10D6800040E85FE30E942BA40E94EFA626E636EA5C
:10D6900045EA53E40E9400A36093430D7093440D48
:10D6A0008093450D9093460D0895CF92DF92EF92AF
:10D6B000FF9278DF6B017C0120E030E040E050E435
:10D6C0000E94E0A518161CF46DDF6B017C0120E0C0
:10D6D00030E040E050E4C701B6010E94E0A5181612
:10D6E0001CF460DF6B017C0120E030E040E050E49E
:10D6F000C701B6010E94E0A518161CF453DF6B01A8
:10D700007C0120E030E040E050E4C701B6010E9417
:10D71000E0A518162CF4FF90EF90DF90CF9042CF49
:10D72000C701B601FF90EF90DF90CF90089581E0A0
:10D730008093840480918504882341F088E080935D
:10D74000D61360E08BEC93E10C94BD860895809134
:10D75000850481110FC081E0809385048093840447
:10D760008091D113982F94609093D1138C600E9474
:10D77000037B18C0809184048823A1F01092D613F3
:10D7800060E08BEC93E10E94BD861092840480914E
:10D79000D1138B7F8093D11388600E94037B1092FA
:10D7A00085040895C4CF2F923F924F925F926F925B
:10D7B0007F928F929F92AF92BF92CF92DF92EF9221
:10D7C000FF920F931F93CF93DF93CDB7DEB766978A
:10D7D0000FB6F894DEBF0FBECDBF1C0183EA9FE0F9
:10D7E0000E94C85A40E855E260E070E083EA9FE09A
:10D7F0000E948F7E64E670E080E090E00E94868D5B
:10D800008CED95E0A0E0B0E08093A70F9093A80F77
:10D81000A093A90FB093AA0F64E670E080E090E0B7
:10D820000E94868D8FEF8A8781E08B8786E88C87C0
:10D830001D861E861F86188A198A89E78A8BC10170
:10D84000880F991F9E8B8D8BC12CD12CE12CF12C34
:10D85000412C512C320183EA9FE0E214F3046CF571
:10D86000ED89FE89CE16DF0644F50E943E4A0897F0
:10D870004CF049E050E0BE01665F7F4F83EA9FE0D5
:10D880000E94144A65E070E080E090E00E94868D7E
:10D8900000E010E0812C912C540183EA9FE00E946B
:10D8A0006F4A892B31F4F4E08F169104A104B1047E
:10D8B000ACF50230110594F535C00E94C85AE11448
:10D8C000F10409F47101C301B2010E94A1A24B014C
:10D8D0005C01B701FF0C880B990B0E94A1A29B0170
:10D8E000AC01C501B4010E94F1A466960FB6F8948C
:10D8F000DEBF0FBECDBFDF91CF911F910F91FF9083
:10D90000EF90DF90CF90BF90AF909F908F907F90DF
:10D910006F905F904F903F902F9008958FEFC81AAF
:10D92000D80A99CF83EA9FE00E946F4A892B69F059
:10D9300083EA9FE00E944D4AE1E0F0E0EC0FFD1F1A
:10D94000E00FF11F80830F5F1F4F65E070E080E004
:10D9500090E00E94868D0230110569F599818A85D3
:10D96000981329C09A818C85981325C0CE010396FF
:10D970009C8B8B8B83EA9FE00E946F4A892B31F44A
:10D9800094E089169104A104B1043CF50930110515
:10D99000C1F48B8190E0982F88272C81820F911DF4
:10D9A000092E000CAA0BBB0B480E591E6A1E7B1ECB
:10D9B000EFEFEE1AFE0AFFEF8F1A9F0AAF0ABF0AB7
:10D9C0006CCF83EA9FE00E944D4AEB89FC898193EA
:10D9D000FC8BEB8B0F5F1F4FCDCF0430110544F351
:10D9E000D8CF2F923F924F925F926F927F928F92F9
:10D9F0009F92AF92BF92CF92DF92EF92FF920F93DE
:10DA00001F93CF93DF936C01CDEED4E081E3882E9A
:10DA100084E0982E09E41DE0EE24E394F12C22E149
:10DA2000222E312C33E1432E512C40E1642E712CF7
:10DA300051E1A52EB12C80912F04909130048E15C8
:10DA40009F050CF4CFC021E0C216D10439F4F801CF
:10DA500082AD93ADF401918380830AC0F2E0CF16CA
:10DA6000D10431F4F40180819181F80193AF82AF48
:10DA7000F40180819181009739F48A819B81909390
:10DA80008D0480938C0422C08130910539F48A8101
:10DA90009B8190938B0480938A0418C082309105F7
:10DAA00039F48A819B8190938904809388040EC005
:10DAB000039761F48A819B81909387048093860405
:10DAC0006AE37CE08EE193E10E94344EF40181919F
:10DAD00091914F018430910539F42A813B81309333
:10DAE00011022093100221C08530910539F42A815A
:10DAF0003B81309307022093060217C086309105C0
:10DB000039F42A813B813093C7042093C60417C09F
:10DB10008730910539F42A813B81309305022093A7
:10DB2000040217C08A309105F1F18531910539F46D
:10DB30002A813B81309303022093020234C0863154
:10DB4000910539F42A813B81309301022093000230
:10DB50002AC08731910539F52A813B81283031056A
:10DB600049F470922B0460922A04B0922904A09286
:10DB7000280419C02730310549F430922B04209233
:10DB80002A0450922904409228040DC02630310501
:10DB900051F421E030E030932B0420932A041092BA
:10DBA0002904109228049C012B5031092A30310598
:10DBB00090F42A813B81309387042093860437E1D7
:10DBC000389FB001399F700D1124695E7D4F8EE141
:10DBD00093E10E94344E8FEFE81AF80A22960E5F06
:10DBE0001F4F29CFDF91CF911F910F91FF90EF90A1
:10DBF000DF90CF90BF90AF909F908F907F906F906D
:10DC00005F904F903F902F900895FF920F931F9336
:10DC1000CF93DF93F82E0AE010E0C0E0D0E08F2D24
:10DC20000E943C8DC80FD91F65E070E080E090E055
:10DC30000E94868D0150110991F7CE016AE070E0D3
:10DC40000E9458A7CB01DF91CF911F910F91FF90B8
:10DC500008954F925F926F927F92AF92BF92CF9250
:10DC6000DF92FF920F931F93CF93DF9300D000D0EA
:10DC7000CDB7DEB75C0183EA9FE00E94C85A40E05E
:10DC800052EC61E070E083EA9FE00E948F7E8CEDB1
:10DC900095E0A0E0B0E08093A70F9093A80FA09329
:10DCA000A90FB093AA0F64E670E080E090E00E94B4
:10DCB000868DC12CD12CF12CCA14DB040CF051C080
:10DCC00065E070E080E090E00E94868D00E010E06A
:10DCD000412C512C3201F1100FC083EA9FE00E94C9
:10DCE0006F4A892B31F485E14816510461047104AF
:10DCF0001CF40330110554F08FEFC81AD80A64E6FB
:10DD000070E080E090E00E94868DD6CF83EA9FE0AD
:10DD10000E946F4A892B69F083EA9FE00E944D4A76
:10DD2000E1E0F0E0EC0FFD1FE00FF11F80830F5FDB
:10DD30001F4F65E070E080E090E00E94868D023029
:10DD400011054CF089818B3B31F4FF24F3948A81D7
:10DD50008A3A09F0F12C8FEF481A580A680A780AB3
:10DD6000BACF8F2D26960FB6F894DEBF0FBECDBF6B
:10DD7000DF91CF911F910F91FF90DF90CF90BF90D7
:10DD8000AF907F906F905F904F9008951F93CF93C7
:10DD9000DF93182FCFECDDE0812F0E943C8D89931B
:10DDA00099936CE370E080E090E00E94868D8EE0B5
:10DDB000CF31D80789F70E948B7C20E030E040EA21
:10DDC00050E40E9400A320E030E040E85AE30E94C3
:10DDD00000A3DF91CF911F9108956F927F928F9250
:10DDE0009F92AF92BF92CF92DF92EF92FF920F93EA
:10DDF0001F93CF93DF93CDB7DEB768970FB6F89434
:10DE0000DEBF0FBECDBF7C018091BF0D9091C00DD4
:10DE1000019731F06AE37CE0C7010E94DC4E4DC1FE
:10DE200066E87BE0CE010D960E94DC4EBE01635F8A
:10DE30007F4F89E69EE00E943A4F6CE271E080E0FD
:10DE400090E00E94868DCE0143960E94D15964E6EF
:10DE500070E080E090E00E94868DC12CD12C85E09E
:10DE6000A82EB12C9AE0892E912C61E97BE0CE019D
:10DE700001960E94DC4E8F89988D892B69F06B8802
:10DE80007C8869817A81C3010E9412AA009721F0DF
:10DE90008C010619170902C00FEF1FEFCE01019682
:10DEA0000E94984EA8014F5F5F4FBE016D5E7F4F8D
:10DEB000CE0101960E945480BE016F5F7F4FCE015C
:10DEC0000D960E945E4ECE0101960E94984E898961
:10DED0009A89892B69F060E070E0CE010D960E946E
:10DEE000654D082E000C990BC0970A9708F4CEC018
:10DEF00010E069E17DE0CE0101960E94CC4E44E144
:10DF000050E06FEF7FEFCE0101960E94FA60CE01E4
:10DF100001960E94984E8FEFC81AD80A62E370E00B
:10DF200080E090E00E94868DC601B5010E946CA73A
:10DF3000019771F5CE0101960E9492588D819E81C4
:10DF4000892B59F0BE016F5F7F4F82EE92E10E94F4
:10DF5000494E0E94C40811E017C0E4E1CE16D10476
:10DF60009CF0C601B4010E946CA7892B69F4BE0124
:10DF7000635F7F4F89E69EE00E943A4F68EC70E055
:10DF800080E090E00E94868DCE0101960E94984E1E
:10DF9000CE0101960E94D159BE016F5F7F4FCE0125
:10DFA00043960E945E4ECE0101960E94984E62E317
:10DFB00070E080E090E00E94868DF4E6CF16D104F8
:10DFC00019F0112309F451CF80911F0D8823F1F02E
:10DFD00064E87BE0CE0101960E94DC4EBE01635FE7
:10DFE0007F4FCE0101960E94E94DBC01CE010796FC
:10DFF0000E94D44ECE0107960E948754CE01079608
:10E000000E94984ECE0101960E94984E89899A8965
:10E01000892B61F060E070E0CE010D960E94654DA5
:10E02000082E000C990BC0970A9730F063E97BE04B
:10E03000C7010E94DC4E21C06FE97BE0CE01019652
:10E040000E94DC4EBE016F5F7F4FCE010D960E9495
:10E05000F849182FCE0101960E94984E1111E6CF73
:10E06000F701118210821382128215821482BE017E
:10E07000635F7F4FC7010E945E4ECE0143960E94B0
:10E08000984ECE010D960E94984E17C06FE97BE026
:10E09000CE0101960E94DC4EBE016F5F7F4FCE0124
:10E0A0000D960E94F849082FCE0101960E94984EC5
:10E0B00011E0002309F41DCF1BCFC70168960FB6EE
:10E0C000F894DEBF0FBECDBFDF91CF911F910F91AE
:10E0D000FF90EF90DF90CF90BF90AF909F908F9088
:10E0E0007F906F9008954F925F926F927F92AF9260
:10E0F000BF92CF92DF92EF92FF920F931F93CF9335
:10E10000DF93CDB7DEB7EA970FB6F894DEBF0FBE48
:10E11000CDBFF82E6AE37CE0CE01C5960E94DC4EAE
:10E120008E010B5E1F4F6F2DC8010E9493861887CA
:10E130000F831D821E82198289E08A8381E08B838E
:10E140008C831C8A1B8ACE0101960E945D47CE01FA
:10E1500001960E94ED46CE0101960E9412460E8164
:10E1600010E00330110509F46EC16FE07DE0CE01CF
:10E17000C5960E940E4E6AE37CE08AEC92E10E9412
:10E18000344EBE016B5C7F4FCE0183960E94D44E0D
:10E190004AE050E060E070E0CE0183960E94556056
:10E1A000CE0183960E94984E61E080E00E94147B2D
:10E1B00066EB7BE0CE01C5960E94344E81EBA82E23
:10E1C0008CE0B82ECC24C394D12CE12CF12CE01699
:10E1D000F1060CF0EEC06E2DCE0101960E94A24514
:10E1E000F50121913191419151915F010E942BA440
:10E1F0002B013C0120E030E04CEF52EC0E949BA24E
:10E2000087FF24C0B601CE0189960E946F5E63EB42
:10E2100077E0CE0183960E94DC4EBE01675D7F4FA2
:10E22000CE0183960E94E94D67EA7BE00E94D24DC1
:10E23000BC018AEC92E10E94084ECE0183960E94B6
:10E24000984ECE0189960E94984E48C022E0B301B4
:10E25000A201CE018F960E949D4EB601CE018996F5
:10E260000E946F5E63EB77E0CE0183960E94DC4EE6
:10E27000BE01675D7F4FCE0183960E94E94D6FE23C
:10E2800076E00E94D24DBE01615D7F4F0E94E94D54
:10E29000BC018EEB92E10E94494ECE0183960E9412
:10E2A000984ECE0189960E94984ECE018F960E947C
:10E2B000984E6EEB72E1CE0183960E94D44E66EECC
:10E2C0007BE0CE0183960E94D24DBC018AEC92E1A4
:10E2D0000E94084ECE0183960E94984E013011058F
:10E2E00059F4E114F10409F05DC06AEC72E1CE0169
:10E2F000C5960E94494E56C00230110511F522E024
:10E30000B301A201CE0183960E949D4EBE016D5DB8
:10E310007F4FCE0189960E94D44E66EE7BE0CE01FF
:10E3200089960E94D24DBC01CE01C5960E94084E2E
:10E33000CE0189960E94984ECE0183960E94984EF7
:10E3400031C00330110571F16EEB72E1CE0183969D
:10E350000E94D44E44E150E06FEF7FEFCE018396F0
:10E360000E94C07FCE0183960E94984E64E47BE0B9
:10E37000CE0183960E94DC4ECE0183960E94AA5A5B
:10E38000CE0183960E94984E80918504882351F097
:10E3900080918404882331F060ED77E080E090E0A4
:10E3A0000E94868DFFEFEF1AFF0A8FEFC81AD80A76
:10E3B0000ECFCE01C5960E94054D8AEC92E10E94D7
:10E3C000054D01151105C9F46CEF7CE08AEC92E172
:10E3D0000E940E4E61EF7CE0CE0183960E94CC4EEF
:10E3E0004AE050E06FEF7FEFCE0183960E94C07F3E
:10E3F000CE0183960E94984EEBC0043011050CF0BC
:10E4000000C1BE016B5C7F4FCE0183960E94D44E4B
:10E410004AE050E06FEF7FEFCE0183960E94C07F0D
:10E42000CE0183960E94984E64E47BE0CE018396F1
:10E430000E94DC4ECE0183960E94AA5ACE0183969A
:10E440000E94984EDEC063EB7BE0CE01C5960E9431
:10E45000344EBE016B5C7F4FCE0183960E94D44E3A
:10E460004AE050E060E070E0CE0183960E94556083
:10E47000CE0183960E94984E6AE37CE08AEC92E19A
:10E480000E94344E6AEC72E1CE01C5960E94494E5C
:10E4900000E010E0602FCE0101960E94A2456B01C2
:10E4A0007C0122E0AB01BC01CE0183960115110570
:10E4B00051F40E949D4EBE016D5D7F4F8BEC93E148
:10E4C0000E943A4F18C00E949D4EBE016D5D7F4F65
:10E4D000CE0189960E94D44E66EE7BE0CE018996ED
:10E4E0000E94D24DBC01CE01C5960E94084ECE01BD
:10E4F00089960E94984ECE0183960E94984E22E003
:10E50000B701A601CE0183960E949D4EBE016D5DAE
:10E510007F4FCE0189960E94D44E66EE7BE0CE01FD
:10E5200089960E94D24DBC018AEC92E10E94084E6D
:10E53000CE0189960E94984ECE0183960E94984EF5
:10E540000F5F1F4F0330110509F0A4CFCE01C59610
:10E550000E94054DBE016B5C7F4FCE0183960E94E9
:10E56000D44E4AE050E06FEF7FEFCE0183960E94D9
:10E57000C07FCE0183960E94984E64E47BE0CE017A
:10E5800083960E94DC4ECE0183960E94AA5ACE0149
:10E5900083960E94984E8AEC92E10E94054D69EBA9
:10E5A0007BE0CE0183960E94DC4E6AEC72E1CE01E4
:10E5B00083960E94E94D63EC7BE00E94D24DBC0142
:10E5C0008AEC92E10E94494ECE0183960E94984EB9
:10E5D000CE01C5960E94984EEA960FB6F894DEBF1B
:10E5E0000FBECDBFDF91CF911F910F91FF90EF90A4
:10E5F000DF90CF90BF90AF907F906F905F904F90E3
:10E60000089563EC7BE08AEC92E10E94FA4DE0CF42
:10E61000AF92BF92CF92DF92EF92FF920F931F9330
:10E62000CF93DF93CDB7DEB72C970FB6F894DEBF4C
:10E630000FBECDBF8091220D811102C00E94927F3A
:10E6400080912D0490912E04029751F08091AF0C8F
:10E650009091B00C009709F48DC1039709F48AC119
:10E6600068E57DE084EC92E10E940E4E64EC72E17C
:10E67000CE0101960E94D44E44E150E060E070E08B
:10E68000CE0101960E945560CE0101960E94984EDF
:10E6900069E47DE084EC92E10E940E4E64EC72E14C
:10E6A000CE0101960E94D44E44E150E06FEF7FEF1F
:10E6B000CE0101960E94C07FCE0101960E94984E25
:10E6C00087E00E947C458C0186E00E947C45BC016D
:10E6D00080E090E00E949FA22AE037ED43EA5CE3ED
:10E6E0000E9400A323E333E948E853E40E942AA4EC
:10E6F0006B017C0184E0A82EB12C20E030E048ECD6
:10E7000052E4C701B6010E94E0A5181614F581E095
:10E71000A81AB10809F4F4C064E670E080E090E063
:10E720000E94868D86E00E947C45BC0180E090E0DE
:10E730000E949FA22AE037ED43EA5CE30E9400A317
:10E7400023E333E948E853E40E942AA46B017C01E7
:10E75000D4CFB80180E090E00E949FA22AE037ED7C
:10E7600043EA5CE30E9400A323E333E948E853E46F
:10E770000E942AA4AB01BC0121E0CE0101960E94B7
:10E780009D4E68EE7BE0CE0107960E94DC4EBE01F6
:10E790006F5F7F4FCE0107960E94E94DBC018AEC66
:10E7A00092E10E94494ECE0107960E94984ECE01FA
:10E7B00001960E94984E6AEC72E1CE0101960E9489
:10E7C000D44E42E350E06FEF7FEFCE0101960E94FE
:10E7D000C07FCE0101960E94984E64E47BE0CE019A
:10E7E00001960E94DC4ECE0101960E94AA5ACE01EB
:10E7F00001960E94984E63E47BE08AEC92E10E94CD
:10E80000FA4D21E0B701A601CE0101960E949D4E6E
:10E8100066EB7BE0CE0107960E94DC4EBE016F5F87
:10E820007F4FCE0107960E94E94DBC0180ED92E139
:10E830000E94494ECE0107960E94984ECE01019645
:10E840000E94984E66EE7BE0CE0101960E94DC4E5F
:10E8500060ED72E1CE0101960E94E94DBC0184ECAD
:10E8600092E10E94494ECE0101960E94984E64ECBE
:10E8700072E1CE0101960E94D44E4AE050E060E081
:10E8800070E0CE0101960E94FA60CE0101960E94CE
:10E89000984E64E47BE0CE0101960E94DC4ECE01EE
:10E8A00001960E94AA5ACE0101960E94984E63E4F6
:10E8B0007BE080ED92E10E94FA4D60ED72E1CE01C5
:10E8C00001960E94D44E66EE7BE0CE0101960E9436
:10E8D000D24D6AEC72E10E94E94DBC018AEC92E1F2
:10E8E0000E94494ECE0101960E94984E8091AF0C35
:10E8F0009091B00C039709F006C184E090E0FFC04E
:10E900006EE37DE084EC92E10E940E4E64EC72E1D5
:10E91000CE0101960E94D44E4AE050E060E070E0E3
:10E92000CE0101960E945560CE0101960E94984E3C
:10E9300066ED7BE0CE0101960E94DC4E64EC72E154
:10E94000CE0101960E94E94DBC018AEC92E10E9441
:10E95000494ECE0101960E94984E8091AF0C909145
:10E96000B00C049721F41092B00C1092AF0C81E01F
:10E9700090E018C186E09FE00E94C85A64E670E00B
:10E9800080E090E00E94868D6EE77DE084EC92E16D
:10E990000E940E4E64EC72E1CE0101960E94D44EAC
:10E9A00044E150E060E070E0CE0101960E945560C5
:10E9B000CE0101960E94984E6FE67DE084EC92E1D4
:10E9C0000E940E4E64EC72E1CE0101960E94D44E7C
:10E9D00044E150E06FEF7FEFCE0101960E94C07FCF
:10E9E000CE0101960E94984E8CE40E94E65A6B017B
:10E9F0007C0104E010E0A7019601C701B6010E9466
:10EA000030A7811192C021E0B701A601CE0107967F
:10EA10000E949D4E68EE7BE0CE0101960E94DC4E86
:10EA2000BE01695F7F4FCE0101960E94E94DBC0196
:10EA30008AEC92E10E94494ECE0101960E94984EC6
:10EA4000CE0107960E94984E6AEC72E1CE010196C3
:10EA50000E94D44E42E350E06FEF7FEFCE0101966B
:10EA60000E94C07FCE0101960E94984E64E47BE034
:10EA7000CE0101960E94DC4ECE0101960E94AA5A58
:10EA8000CE0101960E94984E63E47BE08AEC92E10D
:10EA90000E94FA4D86E60E94E65A6B017C0104E072
:10EAA00010E0A7019601C701B6010E9430A7882394
:10EAB00009F47DC00150110909F0E2C06AE37CE06D
:10EAC00080ED92E10E94344E60ED72E1CE0101963C
:10EAD0000E94D44E66EE7BE0CE0101960E94D24D9C
:10EAE0006AEC72E10E94E94DBC018AEC92E10E945D
:10EAF000494ECE0101960E94984E83E090E090939B
:10EB0000B00C8093AF0C64E670E080E090E00E946F
:10EB1000868D8091220D882309F4BEC060E273E0E7
:10EB200080E090E00E94868DB7C00150110909F085
:10EB30009BC064E67DE084EC92E10E940E4E64ECA2
:10EB400072E1CE0101960E94D44E4AE050E060E0AE
:10EB500070E0CE0101960E945560CE0101960E94A0
:10EB6000984E66ED7BE0CE0101960E94DC4E64EC8F
:10EB700072E1CE0101960E94E94DBC018AEC92E15E
:10EB80000E94494ECE0101960E94984E8091AF0C92
:10EB90009091B00C039721F41092B00C1092AF0C2E
:10EBA00082E090E090932E0480932D04ACCF21E07E
:10EBB000B701A601CE0107960E949D4E66EB7BE051
:10EBC000CE0101960E94DC4EBE01695F7F4FCE01EF
:10EBD00001960E94E94DBC0180ED92E10E94494EF0
:10EBE000CE0101960E94984ECE0107960E94984E43
:10EBF00066EE7BE0CE0101960E94DC4E60ED72E194
:10EC0000CE0101960E94E94DBC0184EC92E10E9484
:10EC1000494ECE0101960E94984E64EC72E1CE01FD
:10EC200001960E94D44E4AE050E06FEF7FEFCE0194
:10EC300001960E94FA60CE0101960E94984E64E40B
:10EC40007BE0CE0101960E94DC4ECE0101960E942F
:10EC5000AA5ACE0101960E94984E63E47BE080EDB3
:10EC600092E10E94FA4D30CF68EC70E080E090E0D5
:10EC70000E94868D8CE40E94E65A6B017C01BBCE1B
:10EC800068EC70E080E090E00E94868D86E60E944D
:10EC9000E65A6B017C0105CF2C960FB6F894DEBFC7
:10ECA0000FBECDBFDF91CF911F910F91FF90EF90DD
:10ECB000DF90CF90BF90AF9008952F923F924F92E8
:10ECC0005F926F927F928F929F92AF92BF92CF92FC
:10ECD000DF92EF92FF920F931F93CF93DF93CDB705
:10ECE000DEB7C554D1090FB6F894DEBF0FBECDBF55
:10ECF0002B013C0169017A010E94BE8D22966CAF06
:10ED00007DAF8EAF9FAF229720E9421621E05206D9
:10ED10006104710434F090E9492E55245394612C18
:10ED2000712C30E1C31637E2D306E104F1042CF470
:10ED3000CDA6DEA6EFA6F8AA08C080E197E2A0E083
:10ED4000B0E08DA79EA7AFA7B8AB8091220D882316
:10ED500021F0CDA6DEA6EFA6F8AA22966CAD7DAD79
:10ED60008EAD9FAD229728EE33E040E050E00E9448
:10ED7000CDA326962CAF3DAF4EAF5FAF269791E067
:10ED80009DAB19A61AA61BA61CA68E01035F1F4FDA
:10ED9000CC24DD247601C418D508E608F708C9AAF2
:10EDA000DAAAEBAAFCAAC9A4DAA4EBA4FCA42DA5B8
:10EDB0003EA54FA558A9C216D306E406F5060CF0E9
:10EDC0002AC3C701B6010E94A1A220E030E04AE7B1
:10EDD00054E40E94F1A4AB01BC0123E0C8010E94ED
:10EDE0009D4EB80184EC92E10E945E4EC8010E94E3
:10EDF000984E8DA59EA5AFA5B8A90A97A105B10506
:10EE000084F426964CAD5DAD6EAD7FAD2697C801FE
:10EE100036D4B80184EC92E10E945E4EC8010E9493
:10EE2000984ECE0101960E94184561E37DE08AEC80
:10EE300092E10E940E4EDE0111961D01C12CD12CD3
:10EE40007601F10181909190A190B1901F01A501EF
:10EE50009401C501B4010E9400A39B01AC01C7014C
:10EE6000B6010E942BA46B017C0123E0B501A40133
:10EE7000C8010E949D4EB801CE0143960E94D44E17
:10EE800066EE7BE0CE0143960E94D24DBC018AEC37
:10EE900092E10E94084ECE0143960E94984EC8010E
:10EEA0000E94984E0215130561F6C701B6010E9433
:10EEB000EFA66B017C01FDE24F16F1E05F066104F5
:10EEC00071042CF00E94927F60E080E0ADD323E0DB
:10EED000B701A601CE0143960E949D4E61EF7BE0F3
:10EEE000C8010E94DC4E64EC72E1C8010E94E94D49
:10EEF00064EF7BE00E94D24DBE016D5E7F4F0E94A9
:10EF0000E94D69EF7BE00E94D24DBC018AEC92E1B1
:10EF10000E94084EC8010E94984ECE0143960E945E
:10EF2000984E2DEC3CEC4CE45FE3C701B6010E9427
:10EF3000E0A529813A814B815C812DA33EA34FA39B
:10EF400058A718160CF0ABC12AE939E949E95FE383
:10EF5000C701B6010E949BA287FFA1C1CDA8CC200A
:10EF600009F49DC189849A84AB84BC8420E030E09C
:10EF7000A901C501B4010E949BA2CD80DE80EF8073
:10EF8000F884882309F12DA13EA14FA158A5CA01FB
:10EF9000B9010E9400A36EAB7FAB88AF99AFA70108
:10EFA0009601C701B6010E9400A39B01AC016EA9A6
:10EFB0007FA988AD99AD0E942BA40E94EFA6A50160
:10EFC00094010E949EA404C06BED7FE089EC9FE356
:10EFD00020EE3EE245E652E40E9400A36EAB7FAB1A
:10EFE00088AF99AF20E030E0A901C701B6010E94C7
:10EFF0009BA2882309F12DA13EA14FA158A5CA01CA
:10F00000B9010E9400A36AAF7BAF8CAF9DAFA50191
:10F010009401C501B4010E9400A39B01AC016AAD3B
:10F020007BAD8CAD9DAD0E942BA40E94EFA6A701E5
:10F0300096010E949EA404C06BED7FE089EC9FE3E3
:10F0400020EE3EE245E652E40E9400A36AAF7BAFA9
:10F050008CAF9DAF20E030E0A9016DA17EA18FA112
:10F0600098A50E949BA28823F9F0A5019401C501EF
:10F07000B4010E9400A34B015C01A7019601C701E6
:10F08000B6010E9400A39B01AC01C501B4010E941E
:10F090002BA40E94EFA62DA13EA14FA158A50E942E
:10F0A0009EA46B017C0108C08BEDC82E8FE0D82E8A
:10F0B00089ECE82E8FE3F82E62EF7BE0C8010E9416
:10F0C000DC4E64EC72E1C8010E94E94D6CEF7BE01C
:10F0D0000E94D24DBC018AEC92E10E94494EC801C7
:10F0E0000E94984E62EF7BE0C8010E94DC4E64EC07
:10F0F00072E1C8010E94E94D66E17CE00E94D24DB8
:10F10000BC0184EC92E10E94494EC8010E94984ED5
:10F1100021E04EA95FA968AD79ADCE014F960E945E
:10F120009D4E21E04AAD5BAD6CAD7DADCE01499603
:10F130000E949D4E20EE3EE245E652E4C701B60134
:10F140000E9400A3AB01BC0121E0C8010E949D4EBA
:10F15000B801CE0143960E94D44E66EE7BE0CE010C
:10F1600043960E94D24DBE01675E7F4F0E94E94DDB
:10F1700066EE7BE00E94D24DBE01615E7F4F0E9431
:10F18000E94DBC018EEB92E10E94494ECE014396BF
:10F190000E94984EC8010E94984ECE0149960E9446
:10F1A000984ECE014F960E94984E2DE2421621E0D5
:10F1B00052066104710474F469A57AA58BA59CA517
:10F1C00025E030E040E050E00E94CDA3672B682BA3
:10F1D000692BB9F564EC72E1C8010E94D44E45E098
:10F1E00050E06FEF7FEFC8010E94FA60C8010E94F3
:10F1F000984E6FE17CE0C8010E94DC4E45E050E093
:10F2000061EF7FEFC8010E945560C8010E94984ECF
:10F210006AE37CE0C8010E94DC4EC8010E94AA5A41
:10F22000C8010E94984E6EEB72E1C8010E94D44E54
:10F2300045E050E060E070E0C801A2D6C8010E943D
:10F24000984E6EEB72E18AEC92E10E94084E3FE12B
:10F25000431651046104710434F4C9A4DAA4EBA484
:10F26000FCA4F7FC11C06AEC72E1C8010E94D44E04
:10F27000C8010E948754C8010E94984E6AE37CE04E
:10F280008AEC92E10E94344EB201C30177FE04C0C1
:10F2900069A97AA98BA99CA90E94868DA9C023E09F
:10F2A0004DA15EA16FA178A5CE0143960E949D4E0F
:10F2B00062EF7BE0C8010E94DC4E64EC72E1C801A1
:10F2C0000E94E94D61E27CE00E94D24DBE016D5E7C
:10F2D0007F4F0E94E94D6AEF7BE00E94D24DBC0156
:10F2E00084EC92E10E94494EC8010E94984ECE01E2
:10F2F00043960E94984E49855A856B857C8523E00C
:10F30000CE0149960E949D4E4D815E816F81788528
:10F3100023E0C8010E949D4EB801CE0143960E9491
:10F32000D44E66E27CE0CE0143960E94D24DBE01EF
:10F33000675E7F4F0E94E94D6AEF7BE00E94D24DED
:10F34000BC018EEB92E10E94494ECE0143960E9491
:10F35000984EC8010E94984ECE0149960E94984E40
:10F360002DE2421621E052066104710474F469A58D
:10F370007AA58BA59CA525E030E040E050E00E94F6
:10F38000CDA3672B682B692BE9F464EC72E1C8010B
:10F390000E94D44E4AE050E06FEF7FEFC8010E9418
:10F3A000FA60C8010E94984E6EEB72E1C8010E949B
:10F3B000D44E4AE050E060E070E0C801E1D5C801F9
:10F3C0000E94984E6AEC72E1C8010E94D44EC801B6
:10F3D0000E948754C8010E94984E6AE37CE08AEC40
:10F3E00092E10E94344EC301B2010E94868D1DAA93
:10F3F0000E94BE8D6B017C0122962CAD3DAD4EADC1
:10F400005FAD2297C21AD30AE40AF50AC9A6DAA6A2
:10F41000EBA6FCA6C8CC64EC72E1CE010D960E946E
:10F42000D44E4AE050E06FEF7FEFCE010D960E9480
:10F430005560CE010D960E94984ECDA8CC20B1F11A
:10F440006FE17CE0CE010D960E94DC4E45E050E07D
:10F4500061EF7FEFCE010D960E945560CE010D96B3
:10F460000E94984E8091220D882391F069E27DE000
:10F47000CE010D960E94CC4E45E050E060E070E079
:10F48000CE010D960E945560CE010D960E94984EB9
:10F490006AE37CE0CE010D960E94DC4ECE010D9613
:10F4A0000E94AA5ACE010D960E94984E6EEB72E110
:10F4B000CE010D960E94D44E4AE050E06FEF7FEFF0
:10F4C000CE010D965DD5CE010D960E94984ECB5B78
:10F4D000DF4F0FB6F894DEBF0FBECDBFDF91CF91E7
:10F4E0001F910F91FF90EF90DF90CF90BF90AF9062
:10F4F0009F908F907F906F905F904F903F902F9054
:10F50000089568E37CE00C946C4F0F931F93CF93A6
:10F51000DF93EC010E943A4F8C01CE01F2DF800FA5
:10F52000911FDF91CF911F910F910895282F309156
:10F53000680E313208F04AC08091450E8111FCCF2F
:10F540009091D71342E04093450E2093440E2FEF45
:10F550002093430E1092420E3093410EE8E4FEE0F9
:10F56000A1E2BEE020E0321721F041914D932F5FE0
:10F57000FACF1092200E2091200E990F922B90938B
:10F58000200E90911F0E913061F410921F0E9091F9
:10F59000200E9093BB009091BC0093FDF8CF95ECAA
:10F5A00001C095EE9093BC009091450E9230E1F32E
:10F5B0009091430E9F3F79F08091430E803241F04D
:10F5C0008091430E803331F084E005C081E003C0B8
:10F5D00082E001C083E01092470E1092680E1092F4
:10F5E000460E089581E0A2CF682F8DED90E10C9436
:10F5F000D88591E09093460E8093D7131092470ED2
:10F600001092680E0895CF93C82F682F607F8BECFF
:10F6100093E10E94D08680E1C89FB00111248BEC59
:10F6200093E1CF910C94D086CF93DF93CDB7DEB723
:10F6300028970FB6F894DEBF0FBECDBF98E0EFEF6E
:10F64000F4E0DE01119601900D929A95E1F7909108
:10F65000D413961710F46FEF690FFE013196E60F81
:10F66000F11DE60FF11D9081890F806828960FB675
:10F67000F894DEBF0FBECDBFDF91CF91C4CF0F9303
:10F680001F93CF93DF93CDB7DEB7A2970FB6F89451
:10F69000DEBF0FBECDBF8C01CB01BA01F8011182D4
:10F6A000108213821282158214822AE0AE014F5F0B
:10F6B0005F4F0E946D9EBE016F5F7F4FC8010E9429
:10F6C000344EA2960FB6F894DEBF0FBECDBFDF91C9
:10F6D000CF911F910F9108950F931F93CF93DF93B5
:10F6E000EC010E946C4F8C01CE010BDF800F911F4B
:10F6F000DF91CF911F910F910895CF92DF92EF92FA
:10F70000FF92CF93DF936B017C0197FF15C06DE2F1
:10F7100080E490E10E94334FEC0144275527BA0161
:10F720004C195D096E097F092AE080E490E10E948E
:10F73000814FC80FD91F08C02AE0AB01BC0180E48B
:10F7400090E10E94814FEC0180E490E1DADE8C0FC1
:10F750009D1FDF91CF91FF90EF90DF90CF900895A4
:10F760008F929F92AF92BF92CF92DF92EF92FF92D1
:10F770000F931F93CF93DF936B017C01142F9B0199
:10F78000AC010E9430A7882319F06BE37CE027C00E
:10F7900046015701E894B7F82FEF3FEF4FE75FE7D7
:10F7A000C501B4010E9430A781110DC02FEF3FEFBA
:10F7B0004FE75FE7C501B4010E949BA218161CF435
:10F7C0006FE37CE00CC02FEF3FEF4FE75FE4C70132
:10F7D000B6010E94E0A5181694F463E47CE080E48E
:10F7E00090E1DF91CF911F910F91FF90EF90DF900B
:10F7F000CF90BF90AF909F908F900C946C4F2FEF55
:10F800003FEF4FE75FECC701B6010E949BA287FD67
:10F81000E4CF20E030E0A901C701B6010E949BA21D
:10F8200087FF0BC06DE280E490E10E94334FEC0152
:10F83000F7FAF094F7F8F09402C0C0E0D0E000E0EE
:10F8400060E070E080E09FE3101741F020E030E0DE
:10F8500040E251E40E94F1A40F5FF6CFA7019601A8
:10F860000E942BA46B017C010E948FA54B015C01BF
:10F870002AE0AB01BC0180E490E10E94814FC80FF7
:10F88000D91F1123C9F1C501B4010E949FA29B0198
:10F89000AC01C701B6010E942AA46B017C016EE293
:10F8A00080E490E10E94334FC80FD91F20E030E080
:10F8B00040E251E4C701B6010E9400A34B015C0184
:10F8C0000E948FA56B01E12CF12C2AE0B701A60163
:10F8D00080E490E10E94814FC80FD91FC701B60193
:10F8E0000E949FA29B01AC01C501B4010E942AA401
:10F8F0006B017C011150D1F6CE01DF91CF911F91A8
:10F900000F91FF90EF90DF90CF90BF90AF909F90BE
:10F910008F90089525CF2F923F924F925F926F92D2
:10F920007F928F929F92AF92BF92CF92DF92EF928F
:10F93000FF920F931F93CF93DF93CDB7DEB7289736
:10F940000FB6F894DEBF0FBECDBFC090CF0DD090E4
:10F95000D00D4091D10D5091D20DC416D5062CF486
:10F960003C2D2D2D6A01432F522FE3EDFDE060E089
:10F9700070E0CB01019111910417150754F44A016D
:10F98000550FAA08BB08680D791D8A1D9B1DA8018B
:10F9900015C0C016D10654F40D2C000CEE08FF085B
:10F9A0006C0D7D1D8E1D9F1D680108C0012E000C71
:10F9B000220B330B600F711F821F931F2EE0EF315C
:10F9C000F207C1F60E94A1A220E030E048E152E433
:10F9D0000E94F1A48B0188879F838FECE82E8DE035
:10F9E000F82E812C912C5401D7016D917D917D01D0
:10F9F000072E000C880B990B0E94A1A29801488544
:10FA00005F810E942AA49B01AC010E9400A39B017C
:10FA1000AC01C501B4010E942BA44B015C01EFE1D4
:10FA2000FEE0EE15FF0501F720E030E04CE152E486
:10FA30000E94F1A40E94EFA66B017C0120E030E05F
:10FA400040E85FE30E94E0A518160CF069C02FECB7
:10FA50003DE03A832983212C312C412C512C320159
:10FA6000A981BA818D919D91BA83A9839C01990F37
:10FA7000440B550B2B833C834D835E83CA01B90134
:10FA80000E94A1A2980148855F810E942AA44B018F
:10FA90005C0120E030E0A9010E94E0A5181624F0E6
:10FAA000B7FAB094B7F8B094A7019601C501B401B4
:10FAB0000E949BA287FF0BC08B819C81AD81BE8180
:10FAC000480E591E6A1E7B1E9FEF291A390AAFE1A4
:10FAD000BEE0E981FA81AE17BF0711F620E030E001
:10FAE00040EC5FE3C701B6010E9400A36B017C01FB
:10FAF000F5E02F1631040CF4AACFC301B2010E9425
:10FB0000A1A26B017C01B101330C880B990B0E94FF
:10FB1000A1A29B01AC01C701B6010E94F1A403C0E0
:10FB2000B80188859F816B017C01C701B6012896C9
:10FB30000FB6F894DEBF0FBECDBFDF91CF911F91FE
:10FB40000F91FF90EF90DF90CF90BF90AF909F907C
:10FB50008F907F906F905F904F903F902F9008957F
:10FB60004F925F926F927F928F929F92AF92BF92CD
:10FB7000CF92DF92EF92FF921F93CF93DF93CDB797
:10FB8000DEB728970FB6F894DEBF0FBECDBF4B018E
:10FB90005C0111E0612E712C9301220F331F220FA3
:10FBA000331F3A832983F901EA55FB4FC080D18086
:10FBB000E280F380A5019401C701B6010E949BA2D7
:10FBC00087FF02C01F5FE6CFA5019401C701B60100
:10FBD0000E949BA249815A8142575B4F5E834D83AD
:10FBE000811106C0FA0160817181828193814DC0CB
:10FBF000F1E06F1AF0EC7F0AC301880F991F880F9C
:10FC0000991FFC01EA55FB4F2081318142815381CC
:10FC100029833A834B835C83FC01E257FB4F40808E
:10FC2000518062807380A3019201ED81FE81608129
:10FC30007181828193810E942AA46D837E838F8348
:10FC4000988729813A814B815C81C501B4010E946A
:10FC50002AA49B01AC016D817E818F8198850E94D1
:10FC600000A34B015C0129813A814B815C81C70172
:10FC7000B6010E942AA49B01AC01C501B4010E94F7
:10FC8000F1A4A30192010E942BA428960FB6F89428
:10FC9000DEBF0FBECDBFDF91CF911F91FF90EF90E0
:10FCA000DF90CF90BF90AF909F908F907F906F909C
:10FCB0005F904F9008950F931F930E94BE8D6093A5
:10FCC0000E0F70930F0F8093100F9093110F86E01B
:10FCD0009FE00E944D4A97FF1FC00E94BE8D009179
:10FCE0000E0F10910F0F2091100F3091110FDC01AA
:10FCF000CB01801B910BA20BB30B00910A0F10914B
:10FD00000B0F20910C0F30910D0F80179107A20758
:10FD1000B307E8F28FEF9FEF1F910F910895CF92F5
:10FD2000DF92EF92FF92CF93DF93EC016A017B01A8
:10FD3000E889F98982E080834115514E610571059A
:10FD4000B1F060E079E08DE390E0A70196010E94B8
:10FD5000F9A3DA01C9010197A109B109B695A795DF
:10FD6000979587959C01211580E13807A8F0E889CF
:10FD7000F989108260E874E88EE190E0A7019601AD
:10FD80000E94F9A3DA01C9010197A109B109B69549
:10FD9000A795979587959C01EC85FD853083EE8529
:10FDA000FF852083188EEC89FD8986E08083EA89AF
:10FDB000FB89808180618083EA89FB8980818860FA
:10FDC0008083EA89FB89808180688083EA89FB8956
:10FDD00080818F7D8083DF91CF91FF90EF90DF90C6
:10FDE000CF900895EF92FF920F931F93CF93DF93DD
:10FDF0001F921F92CDB7DEB709E41DE089549D40E4
:10FE00007C01C701800F911FF80161918F019A83D6
:10FE10008983CE0101962FD1FDE00F3C1F0789F7A2
:10FE200089E49DE00F900F90DF91CF911F910F918A
:10FE3000FF90EF9008950F931F93CF93DF931F923E
:10FE40001F92CDB7DEB707E41DE0F80160818EEDAB
:10FE500093E09A838983CE0101960DD1F8016181E7
:10FE60008FED93E09A838983CE01019604D1C80176
:10FE70000F900F90DF91CF911F910F910895EF9206
:10FE8000FF920F931F93CF93DF931F921F92CDB7D3
:10FE9000DEB704EC11E1845C91417C01C701800F65
:10FEA000911FF80161918F019A838983CE01019698
:10FEB000E2D0F1E10E3C1F0789F784EC91E10F904D
:10FEC0000F90DF91CF911F910F91FF90EF900895C8
:10FED000EF92FF920F931F93CF93DF931F921F9286
:10FEE000CDB7DEB704EC11E1845C91417C01C70120
:10FEF000800F911FF80161918F019A838983CE0150
:10FF00000196B9D0F2E10E3B1F0789F784EC91E12D
:10FF10000F900F90DF91CF911F910F91FF90EF9075
:10FF200008950895809185048823E1F080918404E8
:10FF30008823C1F081E067DB8BE39FE10197F1F754
:10FF400060E080E071DB68E77EE08BEC93E10E948B
:10FF5000484F61E080E068DB68E67EE08BEC93E18F
:10FF60000C94484F089580918504882341F0809136
:10FF70008404882321F060E08BEC93E127C7089587
:10FF80008F929F92AF92BF92EF92FF920F931F9327
:10FF9000CF93DF9320918504222309F461C020913F
:10FFA0008404222309F45CC08A01EB017C0177FF01
:10FFB00016C0C095D09561E08C2F36DBB7018BEC75
:10FFC00093E10E943A4F67E57EE08BEC93E10E945B
:10FFD000484FF701848161E08C0F26DB31C00E941D
:10FFE000BE8D80908A0C90908B0CA0908C0CB09061
:10FFF0008D0C24E6820E911CA11CB11C861697065E
:020000021000EC
:10000000A806B90668F561E08C2F0EDBB7018BEC12
:1000100093E10E943A4F66E47EE08BEC93E10E940C
:10002000484FF701848161E08C0FFEDA0E94BE8D9B
:1000300060938A0C70938B0C80938C0C90938D0C36
:10004000B801110F880B990BDF91CF911F910F9180
:10005000FF90EF90BF90AF909F908F900C94868D03
:10006000DF91CF911F910F91FF90EF90BF90AF90D4
:100070009F908F900895FF920F931F93CF93DF93DC
:10008000EC01F62E08811981C8010E94B7A3F81669
:1000900021F06F2DC8010E94BFA3CE01DF91CF9147
:1000A0001F910F91FF900895CF93DF93EC01FB0117
:1000B000248135810E94F04ECE01DF91CF910895C9
:1000C0004F925F926F927F928F929F92AF92BF9268
:1000D000CF92DF92EF92FF920F931F93CF93DF9314
:1000E000CDB7DEB7C654D1090FB6F894DEBF0FBE48
:1000F000CDBF8C016AE37CE0CE01C7960E94DC4E46
:100100006AE37CE0CE01CD960E94DC4EBE016F5FBB
:100110007F4F8FEF92E10E94FE4B8D889E88AF88C3
:10012000B88C498C5A8C6B8C7C8C8D8D9E8DAF8D50
:10013000B8A127968CAF9DAFAEAFBFAF2797C801D0
:100140000197039708F0BCC1A3019201C501B40156
:1001500090580E949EA42BED3FE049EC5FE30E9483
:100160002BA4209167043091680440916904509158
:100170006A040E942BA46B017C0120E030E0A901FD
:100180000E949BA287FD09C0C092E013D092E113A8
:10019000E092E213F092E31310C02BED3FE049EC44
:1001A00050E4C701B6010E942BA46093E013709342
:1001B000E1138093E2139093E313C090E013D09087
:1001C000E113E090E213F090E3132BED3FE049ECF4
:1001D00050E4C701B6010E94E0A5181684F42BED87
:1001E0003FE049EC50E4C701B6010E942AA46093A5
:1001F000E0137093E1138093E2139093E31320E0F4
:1002000030E044E353E46091E0137091E113809196
:10021000E2139091E3130E9400A32BED3FE049E429
:1002200050E40E94F1A46093DC137093DD1380937B
:10023000DE139093DF130E948AA5CE018B960E9455
:100240006F5E67E47CE0CE0185960E94DC4EBE01C5
:10025000655D7F4FCE0185960E94E94D61E57CE0AA
:100260000E94D24DBC0180ED92E10E94494ECE0128
:1002700085960E94984ECE018B960E94984EC09013
:10028000DC13D090DD13E090DE13F090DF1320E05C
:1002900030E044EB52E4C701B6010E949BA218165D
:1002A0008CF020E030E040E05FE3C701B6010E943F
:1002B0002BA40E948AA5CE018B960E946F5E68E5F2
:1002C0007CE022C020E030E044E353E4C701B60103
:1002D0000E949BA218169CF1A701960160E070E8AD
:1002E00084E393E40E942AA46093DC137093DD13EB
:1002F0008093DE139093DF130E948AA5CE018B9624
:100300000E946F5E6BE57CE0CE0185960E94DC4E1C
:10031000BE01655D7F4FCE0185960E94E94DBC010F
:10032000CE01C7960E94494ECE0185960E94984EF6
:10033000CE018B960E94984E69E27AE061C020E07F
:1003400030E047E853E4C701B6010E949BA21816AB
:10035000FCF020E030E044E353E4C701B6010E9422
:100360002AA420E030E040E05FE30E942BA46093E9
:10037000DC137093DD138093DE139093DF130E94E0
:100380008AA5CE018B960E946F5E6BE57CE01EC055
:10039000A701960160E070E084EB93E40E942AA438
:1003A00020E030E040E05FE30E942BA46093DC1388
:1003B0007093DD138093DE139093DF130E948AA560
:1003C000CE018B960E946F5E68E57CE0CE0185963B
:1003D0000E94DC4EBE01655D7F4FCE0185960E9476
:1003E000E94DBC01CE01C7960E94494ECE018596CB
:1003F0000E94984ECE018B960E94984E6EE57CE04E
:10040000CE01CD960E94344EBE01695C7F4FCE0175
:1004100085960E94D44E4AE050E060E070E0CE0144
:1004200085960E945560CE0185960E94984E0E9446
:10043000BE8DC0901B0DD0901C0DE0901D0DF09056
:100440001E0DA4E6CA0ED11CE11CF11CC616D7066F
:10045000E806F90608F423C20E94BE8D0E949FA2FE
:100460006B017C0160911B0D70911C0D80911D0D25
:1004700090911E0D0E94A1A220E030E048EC51E4D2
:100480000E942BA49B01AC01C701B6010E949BA254
:1004900087FD05C266EE7BE0CE0185960E94DC4EAC
:1004A000BE01635C7F4FCE0185960E94E94DBC0181
:1004B000CE01C7960E94084ECE0185960E94984EA6
:1004C000C8010297029708F0C4C120E030E040E282
:1004D00051E4C501B4010E9400A36B017C0120E03E
:1004E00030E040E251E4C301B2010E9400A34B019D
:1004F0005C0120E030E040E251E427966CAD7DAD38
:100500008EAD9FAD27970E9400A32B013C010E9456
:10051000BE8D2091F10C3091F20C4091F30C509172
:10052000F40C621B730B840B950B0E949FA220E0BE
:1005300030E04AE754E40E94F1A4AB01BC0123E09F
:10054000CE018B960E949D4E62EF7BE0CE01859698
:100550000E94DC4EBE01655D7F4FCE0185960E94F4
:10056000E94D66E576E00E94D24DBC018EEB92E14A
:100570000E94494ECE0185960E94984ECE018B96E0
:100580000E94984E6EEB72E1CE0185960E94D44E89
:1005900060ED72E1CE0185960E94E94DBE01695C75
:1005A0007F4F0E94E94DBC01CE01C7960E94494E83
:1005B000CE0185960E94984E6BE37EE08AEC92E134
:1005C0000E940E4E21E0B701A601CE0185960E9441
:1005D0009D4EBE016B5D7F4F8AEC92E10E94084EFA
:1005E000CE0185960E94984E21E0B301A201CE0172
:1005F000C1960E949D4E21E0B501A401CE018B96CB
:100600000E949D4E66EE7BE0CE0185960E94DC4EF8
:10061000BE01655D7F4FCE0185960E94E94D66EE75
:100620007BE00E94D24DBE016F5C7F4F0E94E94D7E
:1006300060E67CE00E94D24DBC018AEC92E10E940F
:10064000084ECE0185960E94984ECE018B960E9450
:10065000984ECE01C1960E94984EA7019601C701FF
:10066000B6010E9400A36B017C01A5019401C501A4
:10067000B4010E9400A39B01AC01C701B6010E9416
:100680002BA46B017C01A3019201C301B2010E9462
:1006900000A39B01AC01C701B6010E942BA40E94DC
:1006A000EFA66B017C016093D8137093D9138093EC
:1006B000DA139093DB1364E67CE08AEC92E10E940B
:1006C000FA4D21E0B701A601CE0185960E949D4E0C
:1006D000BE016B5D7F4FCE018B960E94D44E62E7C8
:1006E0007CE0CE018B960E94D24DBC0180ED92E160
:1006F0000E94494ECE018B960E94984ECE0185965F
:100700000E94984E60ED72E18AEC92E10E94084EE0
:10071000C090D813D090D913E090DA13F090DB1387
:1007200020E030E04AE754E4C701B6010E94E0A5AA
:1007300087FD29C020E030E04AE754E4C701B60154
:100740000E94F1A4AB01BC0123E0CE0185960E947A
:100750009D4EBE016B5D7F4FCE018B960E94D44EA5
:1007600063E77CE0CE018B960E94D24DBC0180ED08
:1007700092E10E94494ECE018B960E94984ECE0186
:1007800085960E94984E20E030E64AE656E4609155
:10079000D8137091D9138091DA139091DB130E94D2
:1007A0009BA2BE01695C7F4F87FF4FC0CE0185963B
:1007B0000E94D44E61EF7BE0CE0185960E94D24D1F
:1007C0006AEC72E10E94E94DBC018AEC92E10E9460
:1007D000494ECE0185960E94984E03301105A1F432
:1007E0006AEC72E1CE0185960E94D44ECE018596C8
:1007F0000E948754CE0185960E94984E6AE37CE061
:100800008AEC92E10E94344E68E67CE0CE01859647
:100810000E94DC4E60ED72E1CE0185960E94E94DAA
:10082000BC01CE018B960E94D44E4AE050E06FEF9F
:100830007FEFCE018B96A4DBCE018B960E94984E63
:10084000CE0185960E94984E04C08AEC92E10E94E7
:10085000494E6AE070E080E090E00E94868DCE0113
:10086000CD960E94984ECE01C7960E94984ECA5BC4
:10087000DF4F0FB6F894DEBF0FBECDBFDF91CF9133
:100880001F910F91FF90EF90DF90CF90BF90AF90AE
:100890009F908F907F906F905F904F9008956AE344
:1008A0007CE0CE0185960E94DC4ECE0185960E94AA
:1008B000AA5ACE0185960E94984EBE01635C7F4F76
:1008C0008BEC93E10E943A4FE5CD1F93CF93DF93DA
:1008D000CDB7DEB7A8970FB6F894DEBF0FBECDBF79
:1008E000182F0E943D5E8EE10E94F97A62E08DED44
:1008F00090E15ED160E08DED90E15AD10E94F27AF4
:100900008EE10E94F97A61E08DED90E151D160E2D3
:100910008DED90E14DD10E94F27A80E290E09093CB
:1009200003138093021380E090E8A9E8B4E4809375
:100930007C0490937D04A0937E04B0937F0480E0B8
:1009400090E0A5E7B4E48093780490937904A093B1
:100950007A04B0937B04BE016F5F7F4F8FEF92E10B
:100960000E94B14B112309F487C060E17EE080E46E
:1009700090E10E94484F80E490E10E94817A60E01B
:100980007EE080E490E10E94484FBE016F5F7F4FA0
:1009900080E490E10E946C7B60EF7DE080E490E178
:1009A0000E94484F6D857E858F8598890E947D7B4A
:1009B00060EE7DE080E490E10E94484F69897A8989
:1009C0008B899C890E947D7B60ED7DE080E490E1D5
:1009D0000E94484F20E030E040E251E4698D7A8D7A
:1009E0008B8D9C8D0E9400A342E050E00E948A7C87
:1009F00061E77CE080E490E10E946C7B60EC7DE04C
:100A000080E490E10E94484F20E030E040E251E471
:100A10006D8D7E8D8F8D98A10E9400A342E050E0E5
:100A20000E948A7C61E77CE080E490E10E946C7B1C
:100A300060EB7DE080E490E10E94484F20E030E0F0
:100A400040E251E469A17AA18BA19CA10E9400A37C
:100A500042E050E00E948A7C61E77CE080E490E123
:100A60000E946C7B6AE87DE080E490E10E94484F40
:100A700080E490E10E94817A64EF71E080E090E090
:100A80000E94868DA8960FB6F894DEBF0FBECDBF2C
:100A9000DF91CF911F91089585ED8093BC008091E7
:100AA000BC0084FDFCCF1092450E089540910414C3
:100AB000262F30E0240F311D21323105DCF4209146
:100AC000450E2430C9F4FC0180E090E0861758F40C
:100AD000309104142191DC01AC51BC4EA30FB11D27
:100AE0002C930196F3CF80910414680F6093041443
:100AF00080E0089581E0089582E0089508950895C2
:100B00000895E091FA0C8091F90CE81730F4F0E0C8
:100B1000E550F34F808190E008958FEF9FEF0895A7
:100B20009091FA0C8091F90C981750F4E92FF0E0AD
:100B3000E550F34F208130E09F5F9093FA0C02C0A4
:100B40002FEF3FEFC90108958091F90C90E02091BB
:100B5000FA0C821B91090895CF92DF92EF92FF92D7
:100B60000F931F93CF93DF937C01CB018A012091D8
:100B7000460E222389F0EB016B01C40ED51ECC1565
:100B8000DD0561F06991D701ED91FC910190F08153
:100B9000E02DC7011995F3CF642F88DFC801DF91DD
:100BA000CF911F910F91FF90EF90DF90CF9008951C
:100BB000CF93DF931F92CDB7DEB769832091460EA6
:100BC0002223D1F02091680E203240F021E030E065
:100BD000FC013383228380E090E014C08091470EB3
:100BE000E82FF0E0E85BF14F998190838F5F80936D
:100BF000470E8093680E04C061E0CE01019656DF77
:100C000081E090E00F90DF91CF91089580E090E037
:100C10000895FC0190810180F281E02DF89481819A
:100C2000892B81832281892F809528232283A7E025
:100C3000B0E01197F1F7218182238183A3E2B0E034
:100C40001197F1F780817894EFECF0E03197F1F7AC
:100C5000982381E009F480E00895FC0190810180EF
:100C6000F281E02D892F809560FF12C0F8942281D7
:100C7000822382838181892B8183A3E2B0E0119753
:100C8000F1F78281982B9283789487ED90E011C0E0
:100C9000F8942281822382838181892B8183AFEF23
:100CA000B0E01197F1F78281982B928378948FE0CE
:100CB00090E00197F1F70895DC012C911196ED91E8
:100CC000FC911297F8948181922F909589238183CA
:100CD00078948DE743E050E0815021F1DA011197DB
:100CE000F1F730813223C1F3F89482818923828322
:100CF0008181822B81837894ABE7B7E01197F1F77C
:100D0000F89481819823918383E191E00197F1F731
:100D10008081282381E009F080E07894E3E6F6E022
:100D20003197F1F708951F93CF93DF93EC01162FBE
:100D300060E0812F65D6612F70E0FB01EE56FF4E1B
:100D4000E491E883FB01E45BFF4EE491F0E0EE0FF9
:100D5000FF1FEE5CFF4E859194919A8389831B86D9
:100D60001D861C86FE013B9623961292EC17FD070A
:100D7000E1F7DF91CF911F9108951F93CF93DF93F8
:100D8000EC01162F8C810E94F97A6B85812F862BBE
:100D900090E00E94F47ADF91CF911F910C94F27A47
:100DA0000F931F93CF938C01C62FE7DF6C2F6460E6
:100DB000C801E3DF6C2F6B7FC801DFDF83EC90E0BD
:100DC0000197F1F7CF911F910F9108950F931F9302
:100DD000CF938C01C62F607F6160E2DF80E1C89F06
:100DE000B00111246160C801DBDF81E090E0CF91A8
:100DF0001F910F9108951F920F920FB60F92112419
:100E00000BB60F922F933F934F935F936F937F9304
:100E10008F939F93AF93BF93EF93FF938091EA10CB
:100E200099D52091ED103091EE102F5F3F4F309308
:100E3000EE102093ED109091EC10953618F096E09E
:100E40009093E9109091E9109430C9F128F4923010
:100E500069F09330D1F05EC0953009F451C09630FE
:100E600009F058C091E09093B91151C0811152C05E
:100E70002091ED103091EE102436310508F442C077
:100E80001092B9111092EC101CC0813009F042C0D0
:100E9000E091EC1091E09E0F9093EC10F0E0209127
:100EA000ED103091EE10EE0FFF1FE151FF4E318338
:100EB00020831092EE101092ED1094E029C0811161
:100EC00017C0E091EC1091E09E0F9093EC10F0E0D1
:100ED0002091ED103091EE10EE0FFF1FE151FF4E0B
:100EE000318320831092EE101092ED1093E010C029
:100EF0002091ED103091EE102536310558F007C0E5
:100F0000811108C01092EE101092ED1003C095E010
:100F10009093E9109091EB10992329F0811102C070
:100F20002F9A01C02F98FF91EF91BF91AF919F91A0
:100F30008F917F916F915F914F913F912F910F9082
:100F40000BBE0F900FBE0F901F901895CF92DF929F
:100F5000EF92FF92CF93DF93EC01072E000C880BEA
:100F6000990B0E94A1A26B017C0120E030E040E4DB
:100F70005FE30E9400A320E030E048E452E40E94D6
:100F8000F1A40E948AA5C617D707D4F020E030E06C
:100F900040EA5FE3C701B6010E9400A320E030E011
:100FA00048E452E40E94F1A420E030E040E85FE32E
:100FB0000E942BA40E948AA521E06C177D070CF4E7
:100FC00020E0822F90E0DF91CF91FF90EF90DF90B3
:100FD000CF9008950F931F93CF93DF93082F6EEB5D
:100FE00079E080E490E10E941350C7E0D0E010E087
:100FF000B8010C2E02C0759567950A94E2F76170EE
:10100000772742E050E080E490E10E94C94F2197A9
:1010100078F7DF91CF911F910F9108951F920F9252
:101020000FB60F9211240BB60F922F933F934F934D
:101030005F936F937F938F939F93AF93BF93EF9340
:10104000FF938091B900887F803609F49CC068F5D1
:10105000883209F45BC090F4803109F454C038F44C
:10106000882309F4F6C0883009F44DC0F5C08831F2
:1010700009F44CC0803209F45DC0EEC0803409F43C
:1010800068C048F4803309F455C0883309F0E4C0DF
:101090008093430ED8C0803509F44FC0883509F4D9
:1010A0005DC0883409F0D8C0D6C0883909F4C7C0FB
:1010B000A8F4883709F467C038F4883609F463C0A7
:1010C000803709F460C0C8C0883809F4B8C08039D6
:1010D00009F45FC0803809F0BFC05BC0803B09F4F1
:1010E00086C038F4803A09F466C0883A09F47FC0B3
:1010F000B3C0803C09F4A7C0883C09F4A4C0883B75
:1011000009F48AC0A9C08091200E10C09091420EAF
:101110008091410E981770F5E091420E81E08E0F9C
:101120008093420EF0E0EF5DF14F80818093BB0031
:1011300085EC86C08093430E8EC0E091420E81E024
:101140008E0F8093420E8091BB00F0E0EF5DF14F77
:1011500080839091420E8091410E6EC0E091420ECC
:1011600081E08E0F8093420E8091BB00F0E0EF5D36
:10117000F14F80838091440E81116DC081E0809396
:101180001F0E84EA61C083E08093450E10922614FE
:10119000CFCF80912614803208F051C0E091261400
:1011A00081E08E0F809326148091BB00F0E0EA5F0F
:1011B000FB4E8083BDCF85EC8093BC001092450E22
:1011C00080912614803230F4E0912614F0E0EA5F3A
:1011D000FB4E10826091261470E0E091F50CF091C6
:1011E000F60C86E094E119951092261435C084E03F
:1011F0008093450E1092051410920414E091F70CA0
:10120000F091F80C199580910414811105C081E0CA
:10121000809304141092E413E091051481E08E0F82
:1012200080930514F0E0EC51FC4E80818093BB006C
:101230009091051480910414981708F479CF85E8EB
:101240008093BC0009C085EC8093BC001092450ED1
:1012500003C01092430E20DCFF91EF91BF91AF913C
:101260009F918F917F916F915F914F913F912F91BE
:101270000F900BBE0F900FBE0F901F9018950C94FF
:1012800056A808953F924F925F926F927F928F92ED
:101290009F92AF92BF92CF92DF92EF92FF920F9305
:1012A0001F93CF93DF93CDB7DEB7A4970FB6F89413
:1012B000DEBF0FBECDBF81E08093271400E010E0B9
:1012C00082E0382E0E30110508F0AAC2F8018827F6
:1012D000E855FF4F8F4F0C947FA78091BF0D9091E1
:1012E000C00D892B09F566E17AE0CE0107960E94D0
:1012F000DC4E6FEB73E1CE0107960E94E94DBC0115
:10130000CE0101960E94D44E48EC50E06FEF7FEF83
:10131000CE0101960E945560CE0101960E94984E22
:10132000CE0107960E94984E8091BF0D9091C00DFE
:10133000019709F562E07AE0CE0107960E94DC4E43
:101340006FEB73E1CE0107960E94E94DBC01CE011F
:1013500001960E94D44E48EC50E06FEF7FEFCE0133
:1013600001960E945560CE0101960E94984ECE01D2
:1013700007960E94984E8091BF0D9091C00D0297E4
:1013800009F56BE27AE0CE0107960E94DC4E6FEB26
:1013900073E1CE0107960E94E94DBC01CE01019692
:1013A0000E94D44E48EC50E06FEF7FEFCE010196E3
:1013B0000E945560CE0101960E94984ECE0107967C
:1013C0000E94984E60E37AE0CE0107960E94DC4EC0
:1013D00069EB73E1CE0107960E94E94DBC01CE0195
:1013E00001960E94D44E40ED57E06FEF7FEFCE01A3
:1013F00001960E94C07FCE0101960E94984ECE01B8
:1014000007960E94984E8091BF0D9091C00D019754
:10141000E9F5CE0107960E94ED6E8B859C850097BD
:1014200089F1EF81F8852081222361F1079750F13E
:1014300065EF7FE0CE0101960E94CC4E48EC50E073
:101440006FEF7FEFCE0101960E94FA60CE01019608
:101450000E94984EBE01695F7F4FCE0101960E94A7
:10146000D44E48EC50E06FEF7FEFCE0101960E9422
:10147000C07FCE0101960E94984E60ED77E080E03B
:1014800090E044D3CE0107960E94984E64E670E047
:1014900080E090E03BD33092E9101092EC10C0C194
:1014A00069EE7FE0CE0101960E94CC4E48EC50E000
:1014B0006FEF7FEFCE0101960E94FA60CE01019698
:1014C0000E94984E5BD36B017C0158D328EE33E029
:1014D00040E050E00E94F9A3CA01B90120E831E5DB
:1014E00041E050E00E94F9A320E13EE040E050E0FE
:1014F0000E94CDA349015A012CE330E040E050E0C6
:101500000E94CDA329013A01AB01BC01CE01019695
:101510000E943F7BB301A201CE0107960E943F7B50
:10152000B501A401CE010D960E943F7BC701B60113
:1015300020E03CE546E255E00E94F9A3BA01A9018A
:10154000CE0149960E943F7BBE01675E7F4FCE0170
:1015500043960E94D44E65E77CE0CE0143960E94FC
:10156000D24DBE01635F7F4F0E94E94D68E77CE08A
:101570000E94D24DBE01695F7F4F0E94E94D6BE62C
:1015800079E00E94D24DBE016F5F7F4F0E94E94D0E
:1015900064E379E00E94D24DBC01CE014F960E94D7
:1015A000D44ECE0143960E94984ECE0149960E9499
:1015B000984ECE010D960E94984ECE0107960E943D
:1015C000984ECE0101960E94984E40ED57E06FEF85
:1015D0007FEFCE014F960E94C07FCE014F961EC175
:1015E0008091AF0C9091B00C019719F46AED7FE0F7
:1015F00002C06CEC7FE0CE0101960E94CC4E48EC1C
:1016000050E06FEF7FEFCE0101960E94FA60CE01AD
:1016100001960E94984E6CEB7FE0F2C06CEA7FE08E
:10162000CE0101960E94CC4E48EC50E06FEF7FEF68
:10163000CE0101960E94FA60CE0101960E94984E5A
:101640006FE97FE0DDC062E97FE0CE0101960E9494
:10165000CC4E48EC50E06FEF7FEFCE0101960E9438
:10166000FA60CE0101960E94984E67E87FE0C8C0FC
:101670006BE77FE0CE0101960E94CC4E48EC50E033
:101680006FEF7FEFCE0101960E94FA60CE010196C6
:101690000E94984E6AE67FE0B3C08091AF0C9091B3
:1016A000B00C039719F46FE57FE002C065E57FE0B9
:1016B000CE0101960E94CC4E48EC50E06FEF7FEFD8
:1016C000CE0101960E94FA60CE0101960E94984ECA
:1016D0006AE47FE095C06DE37FE0CE0101960E9451
:1016E000CC4E48EC50E06FEF7FEFCE0101960E94A8
:1016F000FA60CE0101960E94984E6EE27FE080C0B3
:1017000063E27FE0CE0101960E94CC4E48EC50E0AF
:101710006FEF7FEFCE0101960E94FA60CE01019635
:101720000E94984E66E17FE06BC08091AF0C909173
:10173000B00C029719F465E07FE002C065EF7EE02F
:10174000CE0101960E94CC4E48EC50E06FEF7FEF47
:10175000CE0101960E94FA60CE0101960E94984E39
:1017600068EE7EE04DC06CED7EE0CE0101960E94F9
:10177000CC4E48EC50E06FEF7FEFCE0101960E9417
:10178000FA60CE0101960E94984E6CEC7EE038C063
:1017900061EC7EE0CE0101960E94CC4E48EC50E018
:1017A0006FEF7FEFCE0101960E94FA6035C061EBCA
:1017B0007EE0CE0101960E94CC4E48EC50E06FEFE7
:1017C0007FEFCE0101960E94FA60CE0101960E9441
:1017D000984E64EA7EE014C068E97EE0CE0101968E
:1017E0000E94CC4E48EC50E06FEF7FEFCE010196A7
:1017F0000E94FA60CE0101960E94984E68E87EE051
:10180000CE0101960E94CC4E40ED57E06FEF7FEF86
:10181000CE0101960E94C07FCE0101960E94984E93
:101820000E940E48882319F0109227140CC00E94C1
:10183000B36180912714882331F00F5F1F4F0F3061
:10184000110509F03FCDA4960FB6F894DEBF0FBE88
:10185000CDBFDF91CF911F910F91FF90EF90DF905F
:10186000CF90BF90AF909F908F907F906F905F9040
:101870004F903F90089590E0FC013197E231F105DF
:1018800008F04EC08827EA54FF4F8F4F0C947FA773
:10189000809180008F7703C0809180008F7D80933E
:1018A0008000089580918000877FF9CF84B58F777D
:1018B00002C084B58F7D84BD08958091B0008F777C
:1018C00003C08091B0008F7D8093B0000895809117
:1018D00090008F7707C0809190008F7D03C080912A
:1018E0009000877F8093900008958091A0008F776B
:1018F00007C08091A0008F7D03C08091A000877FEA
:101900008093A0000895809120018F7707C0809177
:1019100020018F7D03C080912001877F809320016B
:101920000895FC01A089B1898C91A689B78982FDAF
:101930000FC09C91818D8F5F8F73228D821749F02C
:10194000218DDF01A20FB11D5D969C93818F0895BB
:101950008C910895CF93DF93282F30E0F901E8525E
:10196000FF4E8491F901EE56FF4ED491F901E45BEC
:10197000FF4EC491CC2389F081117DDFEC2FF0E084
:10198000EE0FFF1FEE5CFF4EA591B491EC91ED239D
:1019900081E090E021F480E002C080E090E0DF91FF
:1019A000CF9108951F93CF93DF93282F30E0F90153
:1019B000E852FF4E8491F901EE56FF4ED491F901A1
:1019C000E45BFF4EC491CC23B9F0162F811153DF95
:1019D000EC2FF0E0EE0FFF1FE85EFF4EA591B491F3
:1019E0009FB7F894111104C08C91D095D82302C0F0
:1019F000EC91DE2BDC939FBFDF91CF911F91089577
:101A0000CF93DF9390E0FC01EE56FF4E2491FC0152
:101A1000E45BFF4E8491882361F190E0880F991F69
:101A2000FC01E250F04FC591D491FC01E85EFF4EFD
:101A3000A591B491611109C09FB7F8948881209550
:101A400082238883EC912E230BC0623061F49FB710
:101A5000F8948881322F309583238883EC912E2B44
:101A60002C939FBF06C08FB7F894E8812E2B288354
:101A70008FBFDF91CF910895863308F08653909100
:101A80007B00282F2870977F922B90937B002091CA
:101A9000E00490E4299F900111248770822B8093A9
:101AA0007C0080917A00806480937A0080917A0033
:101AB00086FDFCCF809178002091790090E0922BF8
:101AC00008953FB7F89480912D1490912E14A09111
:101AD0002F14B091301426B5A89B05C02F3F19F0E4
:101AE0000196A11DB11D3FBFBA2FA92F982F88279E
:101AF000820F911DA11DB11DBC01CD0142E0660FF9
:101B0000771F881F991F4A95D1F708958F929F924A
:101B1000AF92BF92CF92DF92EF92FF926B017C0166
:101B2000D0DF4B015C01C114D104E104F104E9F000
:101B3000C8DFDC01CB0188199909AA09BB09883ED5
:101B40009340A105B10578F321E0C21AD108E1085C
:101B5000F10888EE880E83E0981EA11CB11CC11408
:101B6000D104E104F10421F7DECFFF90EF90DF9084
:101B7000CF90BF90AF909F908F9008952FB7F8941B
:101B80006091291470912A1480912B1490912C1437
:101B90002FBF08951F920F920FB60F9211242F930B
:101BA0003F938F939F93AF93BF938091291490910C
:101BB0002A14A0912B14B0912C143091281423E0F6
:101BC000230F2D3720F40196A11DB11D05C026E875
:101BD000230F0296A11DB11D209328148093291470
:101BE00090932A14A0932B14B0932C1480912D144D
:101BF00090912E14A0912F14B09130140196A11D34
:101C0000B11D80932D1490932E14A0932F14B09394
